:020000040800F2
:10800000002000205DA500081582000839820008C4
:1080100045820008558200086582000800000000C3
:108020000000000000000000000000004D8100087A
:1080300089820008000000009181000805D6000830
:10804000D7A50008D7A50008D7A50008D7A5000820
:10805000D7A50008D7A50008D7A50008D7A5000810
:10806000D7A50008D7A50008D7A50008D7A5000800
:10807000D7A50008D7A50008D7A50008D7A50008F0
:10808000D7A50008D7A50008D7A50008D7A50008E0
:10809000D7A50008D7A50008D7A50008D7A50008D0
:1080A000D7A50008D7A50008D7A50008D7A50008C0
:1080B000D7A5000811B10008D7A50008D7A500086A
:1080C000D7A50008D7A50008D7A50008D7A50008A0
:1080D000D7A5000825C4020801C40208DBC30208B2
:1080E000D7A50008D7A50008D7A50008D7A5000880
:1080F000D7A50008D7A50008D7A50008D7A5000870
:10810000D7A50008D7A50008D7A50008D7A500085F
:10811000954C0308D7A5000883B10008D7A500082F
:10812000D7A50008D7A50008D7A50008D7A500083F
:10813000DFF80CD03BF066FD0048004787E20208FC
:108140000020002080F3088870470000224B196847
:108150000868B0E8F00F80F30988BFF36F8F4FF025
:10816000000080F311884EF00D0E704700000000F3
:1081700006480068006880F3088862B661B6BFF3FD
:108180004F8FBFF36F8F00DF00BF00BF08ED00E02F
:10819000EFF30980BFF36F8F0F4B1A6820E9F00FE0
:1081A000106008B54FF0BF0080F31188BFF34F8F08
:1081B000BFF36F8F04F054FA4FF0000080F3118882
:1081C000BDE8084019680868B0E8F00F80F3098836
:1081D000BFF36F8F704700BF44000060EFF305806E
:1081E00070470000014800687047000030000060E0
:1081F000A0F16101192900D82038704770470000AC
:1082000054656D636F4D696E695F61726D000099B1
:108210001A00000024A03CF0A7B810B504464FF4A3
:10822000E13005F09BFA234B01221A602146BDE89C
:10823000104021A03CF098B82348C18AE8202CF0D7
:1082400036FBFEE71421E8202CF031FB1FA03CF0A8
:108250008BF8FBE71E21E8202CF029FB1EA03CF048
:1082600083F8FBE72821E8202CF021FB1DA03CF03F
:108270007BF8FBE710B53221E8202CF018FBBDE8B5
:1082800010401CA03CF070B810B53C21E8202CF048
:108290000EFBBDE8104019A03CF066B819A03CF0F8
:1082A00063B81AA03CF060B84E4D49206661756C09
:1082B000740000008801224264656275673A2025D7
:1082C00073200D0A00000000508204604D656D208F
:1082D0004661756C74200000427573204661756CB0
:1082E000742000005573616765204661756C7420C9
:1082F00000000000535643200000000044656275F2
:108300006720000050656E20000000005379735410
:1083100069636B20000000000CB5002201920092FE
:108320005248016841F4803101604FF4A063016854
:1083300001F4003100910199491C0191009911B992
:1083400001999942F3D10168890302D50121009175
:1083500000E000920099012930D145490A6842F0B5
:1083600010020A600A6822F003020A600A6842F0FA
:1083700002020A604168416041684160416841F41D
:1083800080614160416821F47C114160416841F4A1
:10839000E8114160016841F0807101600168890164
:1083A000FCD5416821F003014160416841F00201C0
:1083B00041604168C1F381010229FAD10CBDABE7EC
:1083C00010B52A48016841F0010101604168294A5D
:1083D000114041600168284A11400160016821F4A0
:1083E00080210160416821F4FE0141604FF41F01CA
:1083F0008160FFF7E4FF21494FF00060086010BD85
:1084000010B51A4A506800F00C011D4B1D48002998
:108410000ED004290ED008290ED003605168194AE5
:10842000C1F30311121D515C0268CA40026010BD05
:108430000360F3E70360F1E7516801F470115368DA
:1084400003F48033022404EB914133B153689B035E
:1084500007D50D4B59430160E0E70B4B59430160D1
:10846000DCE7074B59430160D8E7000000100240E9
:10847000002002400000FFF8FFFFF6FE08ED00E0DC
:1084800000127A000000006000093D002A490843FC
:108490002A490860704770B50F23C2780126017819
:1084A000002A1ED0254A126802F4E062C2F5E0629A
:1084B000120AC2F10404D3404578A54082781A40DC
:1084C0002A43120101F1E02181F80024007800F034
:1084D0001F018E404009800000F1E020C0F80061DB
:1084E00070BD01F01F0086404809800000F1E020C7
:1084F000C0F8806170BD124A114001430F48001F4F
:10850000016070470D4A121D002903D01168014314
:108510001160704711688143116070474FF0E0218E
:10852000042804D0086920F0040008617047086935
:1085300040F00400086170470000FA050CED00E00F
:1085400080FFFF1F10B5DD4988420AD14415012183
:10855000204600F056FD2046BDE81040002100F006
:1085600050BDD74988420AD104150121204600F0A8
:1085700048FD2046BDE81040002100F042BDD14931
:1085800088420AD10121CC03204600F03AFD204662
:10859000BDE81040002100F034BD10BD10B54268A8
:1085A000C94B1A400C790B6842EA0422134343601A
:1085B0008268C64B1A40D1F80A30D1F806402343EE
:1085C0004C7942EA440213438360C26A22F4700287
:1085D000897B491EC9B242EA0151C16210BD002126
:1085E000016001714171C0F80610C0F80A10012144
:1085F00081737047002904D0816841F001018160D6
:108600007047816821F0010181607047002904D022
:10861000816841F4807181607047816821F48071C4
:1086200081607047C9B2002A03D042680A434260A1
:10863000704742688A4342607047816841F0080190
:1086400081607047014600208968090700D5012034
:108650007047816841F00401816070470146002045
:108660008968490700D501207047002904D0816836
:1086700041F4A00181607047816821F4A00181600C
:108680007047014600208968490200D501207047E3
:10869000426822F46042491E42EA4131416070471B
:1086A000002904D0416841F400614160704741688D
:1086B00021F400614160704770B5072609290AD985
:1086C000C568A1F10A0404EB4404A640B543A340E5
:1086D0001D43C56007E0056901EB4104A640B543B1
:1086E000A3401D4305611F23072A09D2446B521E74
:1086F00002EB820293409C4391400C43446370BD63
:108700000D2A09D2046BD21F02EB820293409C43D4
:1087100091400C43046370BDC46A0D3A02EB8202BF
:1087200093409C4391400C43C46270BD002904D027
:10873000816841F4801181607047816821F4801163
:1087400081607047C06C80B270475C484C300068F4
:108750007047002904D0416841F48061416070474E
:10876000416821F4806141607047002904D041686C
:1087700041F4805141607047416821F4805141606B
:108780007047826822F4E0420A4382607047002901
:1087900004D0816841F4004181607047816821F410
:1087A000004181607047002904D0816841F40211C2
:1087B00081607047816821F4021181607047014631
:1087C00000208968890200D50120704770B507260E
:1087D00009290AD9C568A1F10A0404EB4404A6409A
:1087E000B543A3401D43C56007E0056901EB4104A3
:1087F000A640B543A3401D430561836BC3F30154F9
:10880000121B921C02EB82021F249440A34391404E
:108810000B43836370BD826B22F44012491E42EA0F
:1088200001518163704708B500900098084400909A
:108830000098026008BD08B50090009808442830F0
:1088400000900098006880B208BD4268204B1A4032
:108850000A4342607047416282627047426822F078
:108860001F020A434260704714490831002804D0AF
:10887000086840F4000008607047086820F40000B1
:10888000086070470246002012680A4200D00120AA
:108890007047C9430160704710B5024600200B0ABB
:1088A0005468C9B20C401168194202D0002C00D0A3
:1088B000012010BD090AC94301607047002401402E
:1088C00000280140003C0140FFFEF0FFFDF7F1FFF2
:1088D000FFFD3FFF01684FF6FE721140016000216D
:1088E000016041608160C1607249724A08399042FA
:1088F00004D1486840F00F00486070476D4A143258
:10890000904204D1486840F0F00048607047694ADE
:108910002832904204D1486840F470604860704743
:10892000644A3C32904204D1486840F47040486048
:108930007047604A5032904204D1486840F4702039
:10894000486070475B4A6432904204D1486840F402
:10895000700048607047574A7832904204D14868A6
:1089600040F0706048607047534A111F904204D134
:10897000086840F00F00086070474F4A1432904278
:1089800004D1086840F0F000086070474A4A283275
:10899000904204D1086840F4706008607047464A0D
:1089A0003C32904204D1086840F47040086070473F
:1089B000414A50329042FAD1086840F47020086071
:1089C000704730B5026847F6F0739A438B680C6ABB
:1089D0004D6923430C692C4323438C692343CC69A1
:1089E00023434C6A23438C6A234313430360CA68BE
:1089F00042600A6882604968C16030BD0021016040
:108A000041608160C160016141618161C161016258
:108A1000416281627047002904D0016841F0010180
:108A20000160704701684FF6FE72114001607047A7
:108A3000002A03D002680A430260704702688A4332
:108A40000260704741607047406880B270470246DC
:108A50000020D10003D518490839096802E01549FA
:108A600008390968114200D001207047C10003D5C0
:108A70001149091F086070470E490839486070475E
:108A800002460020D10003D50B490839096802E0ED
:108A9000084908390968114200D001207047C10017
:108AA00003D50549091F0860704702490839486025
:108AB00070470000080002400804024010B59C49BD
:108AC000884209D10121042000F09BFA0021BDE871
:108AD0001040042000F095BA9649884209D101213E
:108AE000082000F08EFA0021BDE81040082000F0B8
:108AF00088BA9149884209D10121102000F081FAF9
:108B00000021BDE81040102000F07BBA8B4988425C
:108B100009D10121202000F074FA0021BDE81040A5
:108B2000202000F06EBA8649884209D101214020F8
:108B300000F067FA0021BDE81040402000F061BA63
:108B40008049884209D10121802000F05AFA002191
:108B5000BDE81040802000F054BA7B4988420AD119
:108B600084150121204600F04CFA2046BDE8104053
:108B7000002100F046BA10BD10B50121084600F0F2
:108B800040FA0021BDE81040012000F03ABA2DE97A
:108B9000F0410022CC7804F00F03E40601D58C7874
:108BA00023430C784FF00F0714F0FF0F4FF0010C28
:108BB0001CD005680CFA02F40E882640A64211D19A
:108BC000960007FA06F825EA080503FA06F848EAC7
:108BD0000505CE78282E02D0482E02D002E044614E
:108BE00000E00461521C082AE4D305600A88FF2AC9
:108BF0001ED94568002202F108060CFA06F40E8818
:108C00002640A64210D1960007FA06F825EA080584
:108C100003FA06F848EA0505CE78282E00D144610B
:108C2000CE78482E00D10461521C082AE3D3456057
:108C3000BDE8F0814FF6FF710180022181700421AF
:108C4000C17070470246002092680A4200D001209D
:108C50007047806880B2704702460020D2680A429E
:108C600000D001207047C06880B270470161704732
:108C700041617047002A01D001617047416170472E
:108C8000C160704741F48032826181618261816993
:108C90008069704710B52D4B1A684FF680742240DA
:108CA00042EA00100843186010BD2949C8617047A6
:108CB000F0B5264C002801DAE36900E06368C0F3F0
:108CC0000346420D120185B2C0F301579540032FB0
:108CD00007D0C2020CD50322B240934343F0706226
:108CE00009E023F07062636823F07063636002E060
:108CF000AB4343F0706201B12A43002801DAE2611C
:108D0000F0BD6260F0BD10B58A07120F0F239340CB
:108D100021F003040D4921448C689C438C608B68CE
:108D2000904003438B6010BD0949DC3108607047F7
:108D300000080140000C01400010014000140140F7
:108D400000180140001C01400020014000000140CB
:108D5000000020420D49086070470C494860704788
:108D60000A498860704709494AF6AA200860704796
:108D700006494CF6CC400860704701460020034A83
:108D8000D2680A4200D00120704700000030004045
:108D9000B448016841F0010101604168B24A1140E4
:108DA00041600168B14A11400160016821F48021ED
:108DB0000160416821F4FE0141604FF41F018160B0
:108DC0007047A8490A6822F480320A600A6822F4CF
:108DD00080220A60B0F5803F07D0B0F5802F03D124
:108DE000086840F4A02008607047086840F48030AC
:108DF000086070470346002059099A4A01290AD0A1
:108E000002290AD0516A03F01F02012393400B424A
:108E100000D0012070471168F5E7116AF3E718B533
:108E2000002000904FF4A0643120FFF7E3FF009989
:108E3000491C00910099A14201D00028F4D03120B2
:108E4000FFF7D8FF08B1012018BD002018BD854AE2
:108E5000116821F0F80141EAC000106070478449B0
:108E6000086070477F4B5A6822F47C120843104315
:108E7000586070477E49086670477A4A516821F009
:108E800003010143516070477648406800F00C00D0
:108E90007047744A516821F0F001014351607047F6
:108EA000704A516821F4E0610143516070476D4A96
:108EB000516821F4605141EAC00050607047694A2E
:108EC000002903D0517A014351727047517A81438E
:108ED000517270476649D83108607047614A5168DD
:108EE00021F440410143516070475E490022203126
:108EF0000A7001F82029012805D0042802D1052094
:108F000081F820007047012081F8200070475949FE
:108F10000860704753490A6A02430A62704755491C
:108F200044390860704710B54E4A516801F00C0191
:108F3000514B002927D0042927D0082927D00360C6
:108F4000516801F0F00109094C4B5C5C0168E1409B
:108F50004160546804F4E064240A1C5D21FA04F4BE
:108F60008460546804F46054E40A1B5DD940C16015
:108F7000526802F44042920B404B1B1F9A5CB1FBBB
:108F8000F2F1016110BD0360DAE70360D8E75168D0
:108F900001F47011536803F48033022404EB91410F
:108FA00033B153689B0307D5354B59430160C7E77D
:108FB000334B59430160C3E72F4B59430160BFE76F
:108FC000284A002903D05169014351617047516912
:108FD000814351617047234A002903D091690143BD
:108FE0009161704791698143916170471D4A0029E1
:108FF00003D0D1690143D1617047D1698143D16107
:109000007047184A002903D0D1680143D1607047E6
:10901000D1688143D1607047124A002903D0116999
:109020000143116170471169814311617047114912
:109030004039086070470E49C86470470949C871D3
:1090400070470848416A41F08071416270470146AB
:109050000020044A92680A4200D00120704701496A
:1090600088727047001002400000FFF8FFFFF6FE14
:10907000000042428004424200127A001800006060
:1090800000093D00434A002903D0118801431180A3
:10909000704711888143118070473E48001D018848
:1090A00041F01001018070473A48001D018821F00D
:1090B00010010180704737481C300088354918314D
:1090C000098840EA0140704700B50246FFF7E5FF16
:1090D0003049100C18310880081D02805DF804EB3F
:1090E000E2E700B50246FFF7D8FF2A49C2F3034082
:1090F00008310880081D02805DF804EBD4E700B554
:109100000246FFF7CAFF2349100C20310880081DD2
:1091100002805DF804EBC7E71E48103000880007A6
:10912000010B1C4814300088084370471948001D83
:1091300001888906FCD570471648001D018821F07A
:109140000801018001880907FCD57047014600200D
:10915000104A121D12880A4200D0012070470D49A2
:10916000091D0A8882430A8070470A49091D098837
:10917000C2B21140074A1288024202D009B101204E
:109180007047002070470349091D0A8882430A80FE
:10919000704700000028004010B5A94988420AD154
:1091A000841401212046FFF72CFF2046BDE8104023
:1091B0000021FFF726BFA34988420AD104140121E8
:1091C0002046FFF729FF2046BDE810400021FFF7A9
:1091D00023BF9D4988420AD1C41301212046FFF7CD
:1091E0001BFF2046BDE810400021FFF715BF10BD52
:1091F00030B5028802F441530A884C88CD88224356
:109200008C882C4322430C8922434C8922438C892D
:109210002243CC8922431A430280828B22F40062CB
:109220008283098A018230BDF0B585B005460C46BF
:10923000022000210126AA8B4FF240031A40AA8384
:1092400002222A84AF8BA268022A21D0A08800B112
:1092500002266846FFF767FE0098E188B1F5007FB7
:109260002CD07101B0FBF1F000EB8000A168400050
:10927000B0FBF1F0401D80B20A21B0FBF1F000F02C
:109280000101401AC0F34F004FF6FF7202EA0121BC
:10929000821EFE2A01D302200021E28808430243F5
:1092A0002A8420886188A2890843A1881143084341
:1092B000384340F40060A88305B0F0BD000A00EB1D
:1092C0008000A1684000B0FBF1F0401D80B2D3E700
:1092D0000021018041808180C180018141818181A3
:1092E000C181072101827047002101804180818076
:1092F000C1800222826081817047002904D00188E8
:1093000041F0400101807047018821F04001018057
:109310007047002904D0818B41F4806181837047BC
:10932000818B21F4806181837047090901238B407F
:1093300099B2002A03D082880A43828070478288CB
:109340008A4382807047002A03D082880A43828041
:10935000704782888A438280704781817047808904
:109360007047A1F57E42FF3A04D0018841F4807134
:1093700001807047018821F48071018070470029C5
:1093800004D0818841F0040181807047818821F0F8
:10939000040181807047028822F400620280028802
:1093A0000A4302807047018841F480510180704770
:1093B000002904D0018841F40051018070470188E0
:1093C00021F4005101807047012901D0008B7047C2
:1093D000808A7047008A7047B1F5804F04D00188B9
:1093E00021F4804101807047018841F4804101806F
:1093F00070470246002012890A4200D001207047BF
:10940000C9430181704730B50246002001F00F03C7
:10941000012505FA03F4A3B2090905FA01F4A4B27F
:109420009188214012891A4202D0002900D00120DF
:1094300030BD01F00F0201219140C9430181704705
:109440000030014000380040003C004010B5FE49AB
:1094500088420AD1C41401212046FFF7D2FD2046DC
:10946000BDE810400021FFF7CCBDB0F1804F0CD01B
:10947000F649884213D101210220FFF7CDFD0021DA
:10948000BDE810400220FFF7C7BD01210846FFF7E5
:10949000C3FD0021BDE810400120FFF7BDBDEC4930
:1094A000884209D101210420FFF7B6FD0021BDE863
:1094B00010400420FFF7B0BDE649884209D10121E0
:1094C0000820FFF7A9FD0021BDE810400820FFF7A4
:1094D000A3BDE149884209D101211020FFF79CFD7D
:1094E0000021BDE810401020FFF796BDDB498842FF
:1094F00009D101212020FFF78FFD0021BDE8104098
:109500002020FFF789BDD64988420AD144140121A1
:109510002046FFF776FD2046BDE810400021FFF70A
:1095200070BDD04988420AD10121CC042046FFF702
:1095300068FD2046BDE810400021FFF762BDCA4922
:1095400088420AD101210C052046FFF75AFD20462A
:10955000BDE810400021FFF754BDC44988420AD13C
:1095600001214C052046FFF74CFD2046BDE8104088
:109570000021FFF746BDBE49884209D101214020A4
:10958000FFF74AFD0021BDE810404020FFF744BD31
:10959000B849884209D101218020FFF73DFD002113
:1095A000BDE810408020FFF737BDB34988420AD19B
:1095B000841501212046FFF72FFD2046BDE810400D
:1095C0000021FFF729BDAD4988420AD101210C04D1
:1095D0002046FFF716FD2046BDE810400021FFF7AA
:1095E00010BDA74988420AD101214C042046FFF74B
:1095F00008FD2046BDE810400021FFF702BDA1494B
:1096000088420AD101218C042046FFF7FAFC20464B
:10961000BDE810400021FFF7F4BC10BD30B5028852
:10962000894C8F4DA0420DD0A8420BD0B0F1804F95
:1096300008D0864B984205D0854B984202D0854B86
:10964000984203D122F070034A881A43824B984211
:1096500006D0824B984203D022F44073CA881A4342
:1096600002808A8882850A880285A0420AD0A842A0
:1096700008D0824A904205D0814A904202D0814A65
:10968000904201D1097A01860121818230BD30B535
:10969000028C22F001020284028C8388048B24F065
:1096A000700424F003050C882C4322F002020D897B
:1096B00015434A882A43644DA8420BD0684DA842FE
:1096C00008D06E4DA84205D06D4DA84202D06D4D18
:1096D000A8420FD122F008054A892A4322F0040546
:1096E0008A882A4323F4807323F400738D891D43F1
:1096F000CB892B4383800483C9888186028430BD53
:1097000070B5028C22F010020284028C8388048BD4
:1097100024F4E04424F440760D884FF6FF7404EA04
:109720000525354322F020020E8904EA0616164369
:109730004A8804EA02123243434EB04202D0484EF5
:10974000B04217D122F080024E8904EA0616164371
:1097500026F040068A8804EA0212324323F480632A
:1097600023F400638E8904EA86061E43CB8904EA4B
:109770008303334383800583C9880187028470BDD6
:1097800070B5028C22F480720284028C8388848BF0
:1097900024F0700424F003040D88254322F40072A1
:1097A0000E894FF6FF7404EA062616434A8804EA37
:1097B00002223243244EB04202D0294EB04217D189
:1097C00022F400664A8904EA0222324322F48066C7
:1097D0008A8804EA0222324323F4805323F400539C
:1097E0008E8904EA06161E43CB8904EA0313334329
:1097F00083808583C9888187028470BD70B5028C9F
:1098000022F480520284058C8288838B23F4E04307
:1098100023F440760C884FF6FF7303EA04243443A4
:1098200025F400550E8903EA06362E434D8803EAD7
:1098300005353543044EB04202D0094EB04226D120
:1098400022F480468A891FE0002C01400004004079
:1098500000080040000C00400010004000140040D0
:1098600000340140004C01400050014000540140D0
:1098700000180040001C0040002000400040014053
:10988000004401400048014003EA821232438280D2
:109890008483C988A0F84010058470BD828B22F4AF
:1098A00040628283828B4FF6FF7303EA01210A43F1
:1098B00082837047F0B5048C24F480540484868B32
:1098C000048C4FF6FF7505EA013726F4734605EA66
:1098D0000222324305EA03331343F74A90420ED083
:1098E000F64A90420BD0B0F1804F08D0F44A904233
:1098F00005D0F44A904202D0F34A904205D124F4B4
:109900000051394341F4805104E024F402420A43F7
:1099100042F4805183830184F0BD828B22F00C02DB
:109920008283828B0A4382837047F0B5048C24F4CF
:1099300080740484858B048C4FF6FF7707EA012638
:1099400025F0F30507EA031313432B43DA4A904249
:109950000ED0DA4A90420BD0B0F1804F08D0D84AEE
:10996000904205D0D74A904202D0D74A904205D1C2
:1099700024F40071314341F4807104E024F4206246
:109980000A4342F4807183830184F0BD028B22F488
:1099900040620283028B4FF6FF7303EA01210A4300
:1099A00002837047F0B5048C24F010040484068B05
:1099B000048C4FF6FF7505EA011726F4734605EA95
:1099C0000333334305EA02221A43BB4B98420ED0BD
:1099D000BA4B98420BD0B0F1804F08D0B84B9842A8
:1099E00005D0B84B984202D0B74B984205D124F02D
:1099F0002001394341F0100104E024F0A0030B439F
:109A000043F0100102830184F0BD028B22F00C02AE
:109A10000283028B0A430283704770B5048C24F0E2
:109A200001040484058B048C25F0F3054FF6FF76C2
:109A300006EA031313432B439F4A90420ED09F4ADA
:109A400090420BD0B0F1804F08D09D4A904205D093
:109A50009C4A904202D09C4A904205D124F00202D6
:109A60000A4342F0010104E024F00A020A4342F0F2
:109A700001010383018470BD70B505460C468E4814
:109A8000854209D08D48854206D0B5F1804F03D07C
:109A90008B48854200D08B4820886188A288238922
:109AA00058B1042811D0082817D02846FFF702FF24
:109AB000E1882846BDE87040F0E62846FFF7ADFF94
:109AC000E1882846BDE870409FE72846FFF76AFF17
:109AD000E1882846BDE8704058E72846FFF725FF93
:109AE000E1882846BDE8704017E72DE9F0410746B8
:109AF0000C46002501266188002900D10225A28894
:109B0000012A00D102262088238988B13846FFF730
:109B100049FFE1883846FFF739FF23893246294655
:109B20003846FFF77AFFE1883846BDE8F0416CE738
:109B30003846FFF772FFE1883846FFF766FF238952
:109B4000324629463846FFF72DFFE1883846BDE802
:109B5000F0411BE710B50A884B88CC881A438B88E4
:109B600023431A430B891A434B8989891A430A43B1
:109B7000A0F8442010BD4FF6FF71818000210180C4
:109B8000C180418001727047002101804180818045
:109B9000C180018141818181C181704700210180A3
:109BA000418001228280C1800181704700210180B3
:109BB00041808180C180018141818181704700297C
:109BC00004D0018841F0010101807047018821F033
:109BD000010101807047002905D030F8441F41F48D
:109BE00000410180704730F8441FC1F30E0101802D
:109BF0007047002A03D082890A4382817047828994
:109C00008A4382817047818270471143A0F84810CF
:109C10007047002A03D082890A4382817047828973
:109C20008A4382817047018921F0070101817047D1
:109C3000028922F070020A430281704700B5034690
:109C40001846FFF7F5FF188940F00700188100BD9E
:109C500070B50D4604461146602D0CD001222046F9
:109C6000FFF7DBFE29462046FFF7E2FF208940F0A0
:109C70000700208170BD01222046FFF793FEF1E727
:109C800030B50489E4B24FF6FF7505EA03231343A8
:109C90000B432343038130BD10B504462046FFF734
:109CA000EFFF208920F0070040F0070020F070004F
:109CB00040F07000208110BD002C014000340140B4
:109CC0000004004000080040000C004010B50446AD
:109CD0002046FFF7D5FF208940F480402081EAE745
:109CE000018582827047028822F070020A43028056
:109CF000704770B50589048B068C25F007050D4368
:109D00004FF6FC410C4040F201110C4326F02206B4
:109D10004FF6FF7101EA03111143314305810483BA
:109D2000018470BD028B22F070020A4302837047E7
:109D3000028B22F4E0424FF6FF7303EA0121114344
:109D400001837047828B22F070020A43828370473E
:109D5000828B22F4E0424FF6FF7303EA01211143A4
:109D600081837047002904D0018841F0800101807F
:109D70007047018821F0800101807047002904D0DC
:109D8000818841F0040181807047818821F00401BD
:109D900081807047002904D0818841F008018180CA
:109DA0007047818821F0080181807047002904D024
:109DB000818841F0010181807047818821F0010193
:109DC00081807047028B22F008020A4302837047A9
:109DD000028B22F400624FF6FF7303EA0121114364
:109DE00001837047828B22F008020A438283704706
:109DF000828B22F400624FF6FF7303EA01211143C4
:109E000081837047028B22F004020A430283704769
:109E1000028B22F480624FF6FF7303EA01211143A3
:109E200001837047828B22F004020A4382837047C9
:109E3000828B22F480624FF6FF7303EA0121114303
:109E400081837047028B22F080020A4302837047AD
:109E5000028BC2F30E024FF6FF7303EA0121114396
:109E600001837047828B22F080020A43828370470D
:109E7000828BC2F30E024FF6FF7303EA01211143F6
:109E800081837047028C22F002020A4302847047E9
:109E9000028C22F008020A4302847047028C22F0EE
:109EA00020024FF6FF7303EA01111143018470474A
:109EB000028C22F080024FF6FF7303EA0111114376
:109EC00001847047028C22F400724FF6FF7303EA9C
:109ED0000121114301847047028C22F400624FF685
:109EE000FF7303EA0121114301847047028C22F4BD
:109EF00000524FF6FF7303EA0131114301847047AA
:109F000010B501238B40048C9C430484038C8A404D
:109F100013430384CFE610B504238B40048C9C4389
:109F20000484038C8A4013430384C4E630B500F1F3
:109F3000180301248C40058CA5430584002911D009
:109F400008290FD0091FC1F34E001844016821F4FD
:109F5000E041016001684FF6FF7303EA02221143FA
:109F6000016030BD03EB5100016821F07001016018
:109F700001681143016030BD002904D0018841F01F
:109F8000020101807047018821F0020101807047C1
:109F9000002904D0018841F0040101807047018844
:109FA00021F0040101807047002904D0818841F02C
:109FB000800181807047818821F080018180704715
:109FC000028822F00802028002880A430280704759
:109FD000828822F07002828082880A4382807047E1
:109FE000028922F00702028102890A430281704736
:109FF000028922F08002028102890A4302817047AD
:10A0000081847047818570478186704701877047DA
:10A0100081877047A0F840107047028822F4407290
:10A02000028002880A4302807047808E7047008F4A
:10A030007047808F7047B0F840007047808C704741
:10A04000008D704702460020128A0A4200D001208B
:10A050007047C9430182704702460020138A0B40B3
:10A0600092890A40002B02D0002A00D001207047BC
:10A07000C94301827047000010B5E14988420AD106
:10A0800001218C032046FEF7BCFF2046BDE81040AE
:10A090000021FEF7B6BFDB4988420AD101214C04FA
:10A0A0002046FEF7B9FF2046BDE810400021FEF72C
:10A0B000B3BFD54988420AD101218C042046FEF75E
:10A0C000ABFF2046BDE810400021FEF7A5BFCF49F9
:10A0D00088420AD10121CC042046FEF79DFF20468C
:10A0E000BDE810400021FEF797BFC94988420AD158
:10A0F00001210C052046FEF78FFF2046BDE81040E9
:10A100000021FEF789BF10BD30B585B004460D466D
:10A11000208A4CF6FF710840E98801432182A0891A
:10A120004EF6F3110840A9882A8911436A8902432F
:10A130001143A181A08A4FF6FF410840A98901433C
:10A14000A1826846FEF7EFFEAD48844201D1039834
:10A1500000E00298A189090408D500EBC00101EBD9
:10A16000001029684900B0FBF1F007E000EBC001E6
:10A1700001EB001029688900B0FBF1F06422B0FB0C
:10A18000F2F109010B096FF018056B4300EB830036
:10A19000A3891D044FF0320307D503EBC000B0FBC9
:10A1A000F2F000F00700084306E003EB0010B0FBFC
:10A1B000F2F000F00F000843208105B030BD4FF4ED
:10A1C0001651016000218180C18001810C224281F1
:10A1D0008181704710B5038A4FF2FF0213400A884D
:10A1E0004C8822438C88C9880C4322431A4302823C
:10A1F00010BD0021018041808180C180704700290D
:10A2000004D0818941F4005181817047818921F412
:10A2100000518181704710B540F66A13C1F34213B3
:10A2200001F01F040121A140012B07D0022B07D010
:10A2300014303AB102680A43026010BD0C30F8E7EE
:10A240001030F6E702688A43026010BD002A03D08E
:10A25000828A0A4382827047828A8A438282704756
:10A26000028A22F00F020282028A0A4302827047A7
:10A27000828922F40062828182890A438281704746
:10A28000002904D0818941F00201818170478189D0
:10A2900021F0020181817047028A22F020020282AD
:10A2A000028A0A4302827047002904D0018A41F4DD
:10A2B000804101827047018A21F480410182704708
:10A2C000C1F30801818070478088C0F3080070479F
:10A2D000818941F0010181817047028BD2B20283F2
:10A2E000028B42EA012101837047028B02F47F4214
:10A2F0000283028B0A4302837047002904D0818ABB
:10A3000041F0200181827047818A21F02001818201
:10A310007047002904D0818A41F010018182704782
:10A32000818A21F0100181827047002904D0818A3E
:10A3300041F0080181827047818A21F00801818201
:10A340007047002904D0818941F400418181704720
:10A350008189C1F30E0181817047002904D0818A6F
:10A3600041F4006181827047818A21F40061818219
:10A370007047828A22F004028282828A0A438282A1
:10A380007047002904D0818A41F002018182704720
:10A39000818A21F0020181827047024600201288E2
:10A3A0000A4200D0012070478A05C94301807047E6
:10A3B00070B5002440F66A12C1F3421301F01F0584
:10A3C000012606FA05F2012B0CD0022B0DD0838A50
:10A3D0001340090A8E40008830400BB100B10124BF
:10A3E000204670BD83891340F3E7038A1340F0E7EA
:10A3F00040F66A120A0A01219140C9430180704760
:10A40000003801400044004000480040004C00403B
:10A410000050004010B50120FEF709FEBDE81040D5
:10A420000020FEF704BE2049086070471E49091F3E
:10A43000086070471C498431086070471B4A1188C6
:10A4400021F46071014311807047184A118821F08E
:10A450007F0101431180704708B5144A2C3A10441B
:10A4600000900098016008BD08B510492C390844D7
:10A4700000900098008808BD0B489C300068C0B26E
:10A4800070470A480830018841F001010180704797
:10A490000548A0300068C0B2704704480830018801
:10A4A00041F002010180704704860D422C6C00408F
:10A4B00010B501210C072046FEF7AEFD2046BDE891
:10A4C00010400021FEF7A8BD2149086270472049CD
:10A4D000086170471F4A116821F0E00101431160D3
:10A4E00070471B49A031086070471A4B1A6822F068
:10A4F000030202431A601848026842F00402026034
:10A50000012905D020BF016821F0040101607047D6
:10A5100030BFF8E70F48016841F0040101600168AD
:10A5200041F0020101600C48016841F00401016042
:10A5300030BF704701460020064A52680A4200D0E8
:10A540000120704703490A6842EA800008607047AA
:10A5500000000E420070004010ED00E04FF48070EB
:10A560001D4908604FF4F0701C4908601C481D49E3
:10A5700008604FF0BB301C4908601C481C4908604B
:10A580004FF0BB301B4908601B481C4908601C4841
:10A590001C49086018481C4908604FF044301B49AA
:10A5A000086041F201004FF0204108604FF4407014
:10A5B000174908606FF070401649086016488047D8
:10A5C00016480047FEE7FEE7FEE7FEE7FEE7FEE788
:10A5D000FEE7FEE7FEE7FEE7141002401810024017
:10A5E000BB44BBB40014014004140140BB4444B458
:10A5F0000018014004180140BBBBBB44001C0140D3
:10A600004444BBBB041C0140002001400420014025
:10A61000040000A0040100A0C183000831810008EB
:10A6200038B54FF48074ADF8004048208DF8030031
:10A630009D4D69462846FEF7AAFA21462846FEF7B0
:10A6400015FB38BD38B54FF48074ADF800401020CC
:10A650008DF8030003208DF80200934D69462846CB
:10A66000FEF795FA21462846FEF700FB38BD8E4AD4
:10A670004FF40041002802D01046FEF7F7BA10460A
:10A68000FEF7F6BA884A4FF48071002802D01046CF
:10A69000FEF7ECBA1046FEF7EBBA4FF48071824831
:10A6A000FEF7D0BA4FF400417F48FEF7CBBA38B579
:10A6B00001212420FEF78FFC4FF40144ADF8004047
:10A6C00010208DF8030003208DF80200764D6946B6
:10A6D0002846FEF75CFA21462846FEF7C7FA38BD41
:10A6E00010B5FFF7AFFF0120FFF7CCFF0120FFF708
:10A6F000BEFF042003F0D0F90020FFF7C3FF0420C1
:10A7000003F0CAF9BDE810400020B0E710B5FFF72C
:10A7100099FF0020FFF7ABFF0020FFF7B3FF0420F5
:10A7200003F0BAF90120FFF7A2FF0120FFF7AAFF0B
:10A73000BDE81040042003F0AFB910B50120FFF7C9
:10A7400096FF022003F0A8F90020FFF790FF0024F5
:10A75000FFF778FF0120FFF795FFFFF761FFFFF795
:10A760009CFF40B1641CE4B2642CF1D30020FFF7DD
:10A770007EFF012010BD052003F08EF9002010BDE2
:10A7800010B500240120FFF77DFFFFF749FF0120EE
:10A7900003F082F90120FFF76AFF012003F07CF942
:10A7A00007E0641CE4B2FA2C03D9FFF7AFFF0120E5
:10A7B00010BDFFF772FF0028F3D1FFF758FF00200C
:10A7C00010BD10B50020FFF752FFFFF73BFF002040
:10A7D000FFF758FF022003F05FF90120FFF747FF62
:10A7E000022003F059F9BDE8104000203FE710B502
:10A7F0000020FFF73CFFFFF725FF0120FFF742FF96
:10A80000022003F049F90120FFF731FF022003F095
:10A8100043F9BDE81040002029E770B50546FFF771
:10A8200011FF0020FFF723FF0024E809FFF72AFFAC
:10A830006806050E022003F02FF90120FFF717FF2D
:10A84000022003F029F90020FFF711FF022003F096
:10A8500023F9641CE4B2082CE7D370BD70B506463A
:10A860000024FFF7DDFE00250020FFF700FF022097
:10A8700003F012F90120FFF7FAFE6006040EFFF75D
:10A880000CFF08B1641CE4B2012003F005F96D1C53
:10A89000EDB2082DE8D31EB1FFF793FF204670BD3F
:10A8A000FFF7A5FFFAE7000000080140FFF7FFBE31
:10A8B00010B50446FFF714FF200AA02101EB400069
:10A8C000C0B2FFF7AAFFFFF75BFFE0B2FFF7A5FFFB
:10A8D000FFF756FFFFF704FFA120FFF79EFFFFF7EA
:10A8E0004FFF0020FFF7BAFF0446FFF70FFF204697
:10A8F00010BD70B504460D46FFF7F2FE200AA021F8
:10A9000001EB4000C0B2FFF788FFFFF739FFE0B26C
:10A91000FFF783FFFFF734FF2846FFF77EFFFFF7BF
:10A920002FFFFFF7F3FEBDE87040052003F0D4B819
:10A930002DE9F04106460D461746002409E0E000E7
:10A9400025FA00F0C1B2301980B2FFF7D2FF641CC3
:10A95000E4B2BC42F3D3BDE8F0812DE9F0410246F8
:10A960000E4600200024971908E00502381B401EFF
:10A9700080B2FFF79DFF2844641CE4B2B442F4D3D4
:10A98000E9E710B5FF20FFF793FF55280AD05521BE
:10A99000FF20FFF7AEFFFF20FFF78AFF552803D007
:10A9A000012010BD002010BD002010BD70B5044670
:10A9B0000E46154608E02046641CA4B2FFF778FF57
:10A9C00006F8010B6D1EADB2002DF4D170BD70B54F
:10A9D00006460D46144606E029783046FFF789FF03
:10A9E000761CB6B26D1C641EA4B2F5D270BD000018
:10A9F0000146FE48028822F03802028002880A439B
:10AA000002800121FEF779BC2DE9F04107460024C0
:10AA10004FF48055F54E06E0641CA4B2AC4202D35C
:10AA20000020BDE8F08102213046FEF7E2FC00285C
:10AA3000F2D039463046FEF790FC002405E0641C55
:10AA4000A4B2AC4201D30020EBE701213046FEF76F
:10AA5000D0FC0028F3D03046FEF781FCC0B2E0E71E
:10AA60002DE9F04F87B00446012141F23400FEF792
:10AA7000B2FAE020ADF818004FF018088DF81B80EE
:10AA800003268DF81A60DA4D06A92846FEF77FF8EE
:10AA9000E0212846FEF7EAF84FF00209ADF81890D9
:10AAA0008DF81A604FF0100A8DF81BA006A9D14846
:10AAB000FEF76DF8D04D95F82300022801D0062846
:10AAC0000AD10820ADF818008DF81A608DF81BA087
:10AAD00006A9CA48FEF75BF895F8230001274FF056
:10AAE000000B092801D00B2818D101210802FEF71C
:10AAF00072FA4FF48050ADF818008DF81A608DF896
:10AB00001BA006A9BE48FEF742F8ADF80A90ADF8C2
:10AB10000C70ADF81080BB48C0F8B0B1ADF804B00F
:10AB20004FF48270ADF80600ADF808B0B649B74AE8
:10AB300014B1012C12D021E0ADF80AB0ADF80CB080
:10AB40003820ADF8100095F82300022801D006281F
:10AB500014D1C1F884B1C2F88C710FE0ADF80A903D
:10AB6000ADF80C70ADF8108095F82300022801D0E4
:10AB7000062803D1C1F88471C2F88CB14FF400707B
:10AB8000ADF80E00ADF812B00720ADF81400974DE7
:10AB900001A92846FEF72CFB01212846FEF7ADFB54
:10ABA000FF20FFF731FFFF20FFF72EFFFF20FFF709
:10ABB0002BFF012C05D01820FFF71AFF07B0BDE8C6
:10ABC000F08F3820FFF714FFF8E70146904802881D
:10ABD00022F03802028002880A4302800121FEF737
:10ABE0008CBB2DE9F041074600244FF48055884E78
:10ABF00005E0641CA4B2AC4201D3002011E702219D
:10AC00003046FEF7F6FB0028F3D039463046FEF713
:10AC1000A4FB002405E0641CA4B2AC4201D30020D4
:10AC2000FFE601213046FEF7E4FB0028F3D0304672
:10AC3000FEF795FBC0B2F4E670B586B0012138206E
:10AC4000FEF7C9F90121C803FEF7D0F93820ADF8A5
:10AC5000140018268DF8176003248DF816406D4DEA
:10AC600005A92846FDF793FF38212846FDF7FEFF8A
:10AC700061481022550190F8230001280AD00528C8
:10AC800008D0042817D0072815D00C2813D008287E
:10AC900011D01FE02020ADF814008DF816408DF87B
:10ACA0001720544C05A92046FDF771FF20212046AE
:10ACB000FDF7DEFF0EE0ADF814508DF816408DF86C
:10ACC00017204E4C05A92046FDF761FF2946204676
:10ACD000FDF7CEFF0020ADF800004FF48271ADF813
:10ACE0000210ADF804000221ADF806100121ADF804
:10ACF0000810ADF80C60ADF80A50ADF80E00072052
:10AD0000ADF81000424C69462046FEF771FA012169
:10AD10002046FEF7F2FAFF20FFF763FF3820FFF727
:10AD200054FF06B070BD01463B48028822F038024D
:10AD3000028002880A4302800121FEF7DEBA2DE973
:10AD4000F041074600244FF48055334E05E0641C63
:10AD5000A4B2AC4201D3002063E602213046FEF7E4
:10AD600048FB0028F3D039463046FEF7F6FA0024B7
:10AD700005E0641CA4B2AC4201D3002051E60121DD
:10AD80003046FEF736FB0028F3D03046FEF7E7FAF0
:10AD9000C0B246E630B587B001210820FEF71BF9A6
:10ADA00001218803FEF722F94FF46044ADF8184002
:10ADB00018208DF81B0003208DF81A00154D06A9E8
:10ADC0002846FDF7E4FE21462846FDF74FFF01A87F
:10ADD000FEF77EFA0020ADF804004FF48271ADF862
:10ADE0000610ADF80800ADF80A0017E00030014089
:10ADF000000801400010014062730460001401402B
:10AE00000020014000002442000022420080224233
:10AE1000003C0040000C014000380040ADF80C0040
:10AE20006915ADF80E103821ADF81010ADF812000C
:10AE30000720ADF81400084C01A92046FEF7D8F908
:10AE400001212046FEF759FAFF20FFF778FF102076
:10AE5000FFF769FF07B030BD00380040A548A4499E
:10AE60004160A54941607047A248016941F08001F5
:10AE7000016170479F48C068C10701D00120704739
:10AE8000410701D502207047C00601D50320704755
:10AE90000020704770B50446FFF7ECFF0546012D12
:10AEA00005D102F0F9FD641EA4B2002CF4D104B95E
:10AEB000FF25284670BD70B5054645F6FF7630463D
:10AEC000FFF7E8FF002812D18A4C206940F0020009
:10AED00020616561206940F0400020613046FFF745
:10AEE000D9FF012803D0216921F00201216170BD41
:10AEF0002DE9F04106460D4640F6FF773846FFF74C
:10AF0000C9FF00280ED17B4C206940F00100206170
:10AF100035803846FFF7BEFF012803D0216921F0B4
:10AF200001012161BDE8F08100887047C10703D0AD
:10AF300030F8010C000A70470088C0B270472DE954
:10AF4000F04105460E461746002407E036F8141077
:10AF50002846FFF7CDFFAD1C641CA4B2BC42F5D35C
:10AF6000E0E710B50446002307E02046FFF7DCFFCA
:10AF700021F81300A41C5B1C9BB29342F5D310BDB7
:10AF80002DE9F05F82460F461546AAF10060B0F544
:10AF9000002F4DD24FEAD028C0F34906C6F5806491
:10AFA000A54200D82C46DFF854B134E032183BF803
:10AFB00012208A4203D1401C80B2A042F6D3A042A4
:10AFC00014D24846FFF777FF002006E0821937F8D1
:10AFD00010102BF81210401C80B2A042F6D3484645
:10AFE0004FF480624549FFF7AAFF04E02246394644
:10AFF0005046FFF7A4FFA5421AD008F10108002629
:10B0000007EB44070AEB440A281B85B24FF480641F
:10B01000A54200D82C464FF0006000EBC82942142E
:10B0200036494846FFF79DFF00204FF6FF71C4E701
:10B03000BDE8F09F70B504460D460023304E08E091
:10B04000B44208D22046FFF771FFE854641C5B1C31
:10B050009BB29342F4D370BD13B5012201A9FFF74F
:10B060008FFF1CBD2DE9F0470D4690460024074692
:10B07000A0F10060B0F5002F25D200264FF48069C2
:10B08000DFF880A015E06878000215F8021B08447C
:10B090002146641CA4B22AF811004A46944206D103
:10B0A000002418493846FFF76BFF07F50067B61C08
:10B0B000B6B24645E7D3002C05D022463846BDE857
:10B0C000F04710495CE7BDE8F08710B501680E4A0B
:10B0D0001140B1F1005F09D141680C4C216000685A
:10B0E000FDF730F82068BDE81040004710BD0000B3
:10B0F0002301674500200240AB89EFCD10100060AE
:10B1000000000880100800600000FE2F280000608A
:10B1100010B5514C01212046FEF794FF2046BDE8B2
:10B1200010400121FEF795BF7FB504460D46012171
:10B130000220FDF75BFFADF80840ADF80450002495
:10B14000ADF80A40ADF80640434D01A92846FEF788
:10B1500065FA1D218DF800108DF8014002218DF84F
:10B16000021001218DF803106846FDF794F90122C1
:10B1700011462846FEF73DFD01212846FEF71FFD3A
:10B180007FBD2DE9F041BF20EFF3118580F31188D9
:10B19000BFF34F8FBFF36F8F26F0CAFC2F4E0121F4
:10B1A0003046FEF74FFF2E4C012802D16068401C4C
:10B1B00060602C480168491C016021880027B1F5B6
:10B1C0007A7F02D2491C218007E027490868401C89
:10B1D0000860012032F018FF278024490888401CAD
:10B1E0000880088842F21072904200D90F80012135
:10B1F0003046FEF72EFF85F31188BDE8F0817FB55C
:10B2000004460D4601211020FDF7F0FEADF8084080
:10B21000ADF804500020ADF80A00ADF806000F4C60
:10B2200001A92046FEF7FAF936218DF80010012118
:10B230008DF8011003228DF802208DF80310684666
:10B24000FDF729F9012211462046FEF7D2FC012123
:10B250002046FEF7B4FC7FBD000400400010004013
:10B260002C00006028020060B8030060E407006062
:10B27000F8B501215820FDF7AEFE4020ADF80000E2
:10B2800010258DF8035003248DF80240FE4E6946C8
:10B290003046FDF77CFC2902ADF800108DF8035014
:10B2A0008DF802406946F948FDF771FCADF8005091
:10B2B00048208DF803008DF802406946F448FDF7F8
:10B2C00066FC40213046FDF7D3FC0A2002F004FC66
:10B2D00040213046FDF7CAFC0A2002F0FDFB402168
:10B2E0003046FDF7C5FC0A2002F0F6FB402130464F
:10B2F000FDF7BCFC0A2002F0EFFB40213046FDF7D1
:10B30000B7FC0A2002F0E8FB40213046FDF7AEFC16
:10B310000A2002F0E1FB40213046FDF7A9FC0A209B
:10B3200002F0DAFB40213046FDF7A0FC0A2002F0D3
:10B33000D3FBF8BD2DE9F04104460D46D34F4FF441
:10B34000805631463846FDF793FC05F01F00204338
:10B35000FFF7F5FCFF20FFF7F2FC0446280603D5B3
:10B36000FF20FFF7ECFC044631463846FDF77EFC33
:10B370002046BDE8F0812DE9F04104460D46904697
:10B38000C24F4FF4805631463846FDF771FC05F048
:10B390001F002043FFF7D3FC4046FFF7D0FC3146A7
:10B3A0003846BDE8F041FDF761BC2DE9F0410546A6
:10B3B0000C46B64F4FF4805631463846FDF758FCE0
:10B3C0003A20FFF7BCFC05E06D1E0020FFF7B7FC3C
:10B3D00004F8010B002DF7D10020207031463846CB
:10B3E000BDE8F041FDF742BC2DE9F04104460D46B1
:10B3F000A64F4FF4805631463846FDF739FC7A2087
:10B40000FFF79DFC04E0641E2878FFF798FC6D1C94
:10B41000002CF8D131463846BDE8F041FDF726BC96
:10B4200070B505469B4E05F06004307884420BD021
:10B4300003221F21A020FFF79EFFC5F341121F2109
:10B440008020FFF798FF347070BD10B50446204689
:10B45000FFF7E6FF2146BDE8104000206AE770B51F
:10B4600005460C462846FFF7DBFF22462946BDE885
:10B47000704040207FE770B50D4600240146D4207F
:10B48000FFF7EDFFE9B2D620FFF7E9FFC5F307218B
:10B49000D720FFF7E4FF40F6FF7501E0641CA4B27B
:10B4A000EA20FFF7D2FFC00701D0AC42F6D370BD4F
:10B4B00070B505460024FFF7DBFE4FF4FA7609E08D
:10B4C000FF2200211046FFF756FF641CA4B20A2099
:10B4D00002F002FB1D20FFF7B8FFC00701D1B44204
:10B4E000EED3B44201D3012070BD6A490020486008
:10B4F00000210820FFF7B3FF00210920FFF7AFFF6D
:10B5000000210C20FFF7ABFF00210D20FFF7A7FF64
:10B5100010210A20FFF7A3FF1A210B20FFF79FFF3E
:10B5200011210420FFF79BFF1A210520FFF797FF49
:10B53000FF210620FFF793FF1F210720FFF78FFF52
:10B54000A1213820FFF78BFF3F212820FFF787FF3D
:10B5500030212920FFF783FFF9213020FFF77FFFFB
:10B56000F7213120FFF77BFF0D21C020FFF777FF88
:10B570000021C120FFF773FF3322C2218020FFF793
:10B58000FAFE1221C620FFF76AFF0C21C720FFF741
:10B5900066FF1521C420FFF762FFEE21CA20FFF7E6
:10B5A0005EFF0521CB20FFF75AFF2978E420FFF743
:10B5B00056FF6978E520FFF752FFA978E220FFF7F0
:10B5C0004EFFE978E320FFF74AFF2979E020FFF7F3
:10B5D00046FF6979E120FFF742FF4FF4807421466E
:10B5E0000020FFF748FF21461020FFF744FF1F20EF
:10B5F000FFF716FFC0221B218020FFF7BCFE0422AC
:10B600001F218020FFF7B7FEE420FFF71EFF2978F7
:10B61000884201D1002070BD012070BD722014E766
:10B6200070B505460E4611210220FFF718FF1A21BA
:10B630000320FFF714FF41F611202C18E1B2062079
:10B64000FFF70DFFC4F307210720FFF708FF0022D3
:10B6500011467A20FFF78FFE31462846FFF7C4FED9
:10B6600008221F218020FFF786FE1C20FFF7EDFE39
:10B67000084C800719D508221F21A020FFF77BFE68
:10B68000A078401CC0B207E000180140000C014047
:10B690000010014034000060A070142801D91BF094
:10B6A0006FF904F08BFE002070BD0020A070012017
:10B6B00070BD2DE9F04107460E463920FFF7C5FE63
:10B6C000E8B3354C00202179FFF7C9FEA088C0F30C
:10B6D00007210120FFF7C3FE00213A20FFF72AFED1
:10B6E000606000213A20FFF725FE616841EA0020F2
:10B6F000606000213A20FFF71DFE054600213A2038
:10B70000FFF718FE45EA00252D1F00213A20FFF71C
:10B7100011FE804600213A20FFF70CFE48EA002087
:10B720007F1EBD420ED96078401CC0B260701428E4
:10B7300001D91BF025F904F041FE002019E6FFE7CE
:10B74000002016E600060FD46078401CC0B260707E
:10B75000142801D91BF014F91049488F401C488760
:10B7600004F02CFE002004E60020607031462846DC
:10B77000FFF71BFE21790C20FFF771FEA088C0F3B4
:10B7800007210D20FFF76BFE40221E218020FFF7CE
:10B79000F2FD2846EDE500003400006050820460B0
:10B7A000704730B56423B0FBF3F4E4B2B0FBF3F5BB
:10B7B00003FB1500132C01D96430C0B200EB9003D9
:10B7C0000724B3FBF4F504FB1533BC4D1A440D44B8
:10B7D00015F8015C2A4492B2800703D1032901D2F3
:10B7E000521E92B2B2FBF4F004FB102030BD810770
:10B7F00001D0002070476421B0FBF1F201FB12017F
:10B8000009B1012070474FF4C871B0FBF1F201FBA0
:10B81000120008B100207047012070472DE9F04761
:10B8200007460C461646DFF89882B7FBF8F3A548A2
:10B83000002E01D1002101800188994235D003807A
:10B8400040F2B2754FF4B7794FF4B67A0CE028465F
:10B85000FFF7CDFF20B14B4508D3A3F5B77301E047
:10B86000A3F26D136D1CADB25345F0D8A5F5FA6582
:10B87000A571581CA4F807000025DFF8409209F1D3
:10B880000C090CE0A079FFF7B2FF08B1012D44D0FC
:10B8900019F80500984204D81B1A6D1CADB21C2B78
:10B8A000F0D26D1C65715B1CE370B7FBF8F008FB10
:10B8B00010704FF46161B0FBF1F2A270B0FBF1F2D5
:10B8C00001FB12033C22B3FBF2F36370B0FBF1F314
:10B8D00001FB1300B0FBF2F102FB11002070A07914
:10B8E000E278617900F5FA60FFF75BFF2071012EC5
:10B8F00011D1A179744801F5FA61018061798170F3
:10B90000E178C170217901717048A1780170617886
:10B91000417021788170BDE8F0871D2BC1D31D3B9C
:10B92000BBE710B5FDF7C7FB01226949FFF776FFBA
:10B93000002010BD2DE9F05F8846DDF828A0914673
:10B94000002400F11E01822902D30120BDE8F09FEE
:10B9500040F2B27500F5FA665E4FDFF87CB108E0A0
:10B960002846FFF744FF08B13C4400E05C446D1CEE
:10B97000ADB2B542F4D3A8F1010808F0FF070025E5
:10B98000DFF83881DFF838B108F10C080FE018F85B
:10B99000050040F2A321484304EBC014B0B2FFF706
:10B9A00026FF10B1012D00D15C446D1CADB2BD422B
:10B9B000EDD3A9F1010940F2A32009FB00F904EB42
:10B9C000C910C3EB4311C1EB032100EB0110CAEB1B
:10B9D0000A1100EB81000B99441801214FF0C0506F
:10B9E000FDF704FB0120FEF76FFD0C9911B920460D
:10B9F000FDF76AFBFDF79AFB2046A7E73EB500245A
:10BA00000420FEF731FD45F25005A84247D0012140
:10BA10004FF0C050FDF7EAFA0120FEF755FDFEF7A2
:10BA2000F9FC0120FDF761FA08E0641CE4B20A2089
:10BA300002F052F8FA2C01D300203EBD4120FDF760
:10BA4000D9F90028F1D04FF48070FDF763FA012096
:10BA5000FDF765FAFDF76AFBFDF76EFB012108466D
:10BA6000FDF710FBFDF762FBFDF717FB47F6FF70D4
:10BA7000FDF737FBFDF75AFB37212A22CDE90021DC
:10BA8000002002900F231B2208211020FFF752FFF5
:10BA9000FDF70AFB29460420FEF7DEFC07E0FDF770
:10BAA0004BFB01210846FDF7EDFAFDF73FFBFFF7E1
:10BAB00077FEFFF736FF01203EBD0000705B0408F3
:10BAC000805101003E0000609E020060A302006001
:10BAD000101800600085E2018033E101FE4991F811
:10BAE0002310012913D0052911D004290FD00729CB
:10BAF0000DD00C290BD0082909D0022905D0062920
:10BB000003D0092901D00B2903D1FEF77DBFFFF730
:10BB100068B87047F04890F82300012814D0052831
:10BB200012D0042810D007280ED00C280CD00828DA
:10BB30000AD0022805D0062803D0092801D00B28F6
:10BB400005D13820FEF754BF3820FFF73EB87047C4
:10BB5000E14890F82300012814D0052812D00428C9
:10BB600010D007280ED00C280CD008280AD00228A4
:10BB700005D0062803D0092801D00B2805D11820AC
:10BB8000FEF736BF1820FFF720B87047D2480121D2
:10BB900090F82300012813D0052811D0CF4A04289B
:10BBA00011D007280FD00C280DD008280BD0022860
:10BBB0000CD006280AD009280BD00B2809D00AE09F
:10BBC000C748016007E0C2F8A41104E0C2F88C1174
:10BBD00001E0C4480160FF2080E770B5002441F611
:10BBE000FF75FF20FFF77AFFFF2806D0641CFDF7E2
:10BBF000BAF8AC42F5D3012070BD002070BD10B57D
:10BC0000B548002190F82300012813D0052811D051
:10BC1000B24A042811D007280FD00C280DD00828CC
:10BC20000BD002280CD006280AD009280BD00B28EC
:10BC300009D00AE0AA48016007E0C2F8A41104E0B4
:10BC4000C2F88C1101E0A7480160FFF7C6FF18B1E8
:10BC5000FFF79CFF012010BD002010BD70B5054608
:10BC60004FF6FF7401E0641EA4B2FF20FFF736FF19
:10BC7000A84201D0002CF6D10CB1002070BDFF20ED
:10BC800070BD70B504460D46FE20FFF7E7FF30B1EA
:10BC9000012070BDFF20FFF721FF04F8010B6D1E8E
:10BCA000ADB2F7D2FF20FFF719FFFF20FFF716FF15
:10BCB000002070BD70B505460C46FFF78EFF08B139
:10BCC000012070BD2046FFF709FFFD2C18D000248D
:10BCD0004FF40076285DFFF701FF641CA4B2B44264
:10BCE000F8D3FF20FFF7FAFEFF20FFF7F7FEFF2053
:10BCF000FFF7F4FE00F01F00052801D0022070BD00
:10BD0000002070BD70B505460C461646FFF73EFF95
:10BD1000FFF775FF08B1FF2070BD45F04000FFF749
:10BD2000DDFE200EFFF7DAFEC4F30740FFF7D6FE74
:10BD3000C4F30720FFF7D2FEE0B2FFF7CFFE304694
:10BD4000FFF7CCFE0C2D02D1FF20FFF7C7FE1F240A
:10BD5000FF20FFF7C3FE0106DED5641EE4B2F7D272
:10BD600070BD70B50546012200210A20FFF7CAFF09
:10BD7000044624B910212846FFF783FF0446FFF745
:10BD800005FF0CB1012070BD002070BD70B50546E7
:10BD9000012200210920FFF7B5FF044624B9102134
:10BDA0002846FFF76EFF0446FFF7F0FE0CB10120B6
:10BDB00070BD002070BD1FB56846FFF7E7FF10B1EA
:10BDC000002004B010BD9DF800100120B0EB911FC1
:10BDD00009D19DF808209DF8091000EB02200844C5
:10BDE00080B28002EDE79DF805009DF80A1000F092
:10BDF0000F0000EBD1109DF8091001F0030100EBDA
:10BE000041019DF808009DF80720800900EB8200A1
:10BE10009DF8062002F0030200EB8220401CC91F9F
:10BE20008840CEE72DE9F8432B4890F823000128FD
:10BE300012D0052810D004280ED007280CD00C28CA
:10BE40000AD0082808D0022809D0062807D00928D7
:10BE500005D00B2803D005E0FEF7EEFE02E001203E
:10BE6000FEF7FEFDFFF756FE0024FF20FFF736FE2B
:10BE7000641CA4B20A2CF8D302240021952208469F
:10BE8000FFF740FF0546012D02D0641EA4B2F4D294
:10BE9000154F00263E70012D6DD187224FF4D571CC
:10BEA0000820FFF72FFF4FF6FE74012829D001224A
:10BEB00000213720FFF726FF012200212920FFF76C
:10BEC00021FF01285BD80220387001220021372091
:10BED000FFF718FF012209E062730460008022422C
:10BEE00094012242B0012442400000600021292038
:10BEF000FFF708FF054628004ED0641EA4B2E4D226
:10BF00004AE00026E846FF20FFF7E8FD08F80600B3
:10BF1000761CB6B2042EF6D39DF80200012843D158
:10BF20009DF80300AA283FD14607012200213720AF
:10BF3000FFF7E8FE012231462920FFF7E3FE054620
:10BF400015B1641EA4B2F0D2ACB1012200213A2096
:10BF5000FFF7D8FE78B90024FF20FFF7BFFD08F8EF
:10BF60000400641CA4B2042CF6D39DF80000400623
:10BF700002D50620387017E00420387014E0012044
:10BF80003870012200211046FFF7BCFE054628004C
:10BF900002D0641EA4B2F4D22CB1012251021020AE
:10BFA000FFF7B0FE00B13E70FFF7F0FDFFF7D0FDE8
:10BFB000387810B10020BDE8F8830DB12846FAE7C3
:10BFC000AA20F8E72DE9F0410646154638480078E2
:10BFD000062800D049024FF40077012D1AD0012223
:10BFE0001220FFF78FFE39463046FFF74AFE04461F
:10BFF00006F500766D1E15F0FF0501D0002CF2D07D
:10C00000012200210C20FFF77DFEFFF7BFFD204637
:10C01000BDE8F08101221120FFF774FE04462000E4
:10C02000F3D139463046FFF72CFE0446EDE770B5F4
:10C0300006460C4615461E480078062800D06402C5
:10C04000012D13D0012809D0012200213720FFF74C
:10C0500059FE012229461720FFF754FE01222146EE
:10C060001920FFF74FFE04466CB11DE00122214666
:10C070001820FFF747FE0446B4B9FE213046FFF70B
:10C0800019FE044610E0FC213046FFF713FE06F5CA
:10C0900000766D1E15F0FF0501D00028F3D0FD21BC
:10C0A0000020FFF707FE0446FFF770FD204670BD35
:10C0B0004000006070B50024FE4D04EB840005EBE9
:10C0C000800000F0EFFE641C142CF6D3FA4800F058
:10C0D000E9FEF948143000F0E5FEF748283000F09A
:10C0E000E1FEF5483C3000F0DDFEF348503000F052
:10C0F000D9FEF248F04941631431816370BD70B5D7
:10C10000044601F06AFAED4DA868401CA860286852
:10C1100010B1686938B10CE02C60A868012808D11A
:10C12000FFF7C8FF05E02868E16AC06A884200D8C6
:10C130002C60686A401C6862E06A01212A698140BB
:10C1400011432961DB4900EB800001EB8000211DD8
:10C1500000F0B6FE01F04DFA686900280CD028689E
:10C16000E16AC06A884207D2D5494FF08050086022
:10C17000BFF34F8FBFF36F8F70BD2DE9F04781463E
:10C18000DDE908570A9C0E4690469A464FEA880118
:10C19000A522206B36F0EEFD206BA8F1010800EB24
:10C1A000880020F0070800202218315C82F8341043
:10C1B000315C11B1401C1028F6D3002684F843608E
:10C1C000142D00D31325E5626564A664201D00F0DC
:10C1D00074FE04F1180000F070FE2461C5F1140033
:10C1E000A0616462E66484F8506052464946404665
:10C1F00001F0CCF92060002F00D03C60BDE8F08752
:10C200002DE9FF5F8146DDE90E788A4616469B469A
:10C21000B00001F022FA054628000AD0542001F0AF
:10C220001CFA04460CB1256304E0284601F060FACC
:10C2300000E000248CB10020CDE90240CDE9007877
:10C240005B46324651464846FFF797FF2046FFF7C8
:10C2500056FF012004B0BDE8F09F4FF0FF30F9E732
:10C260009648416B0968002905D0416BC968C968C7
:10C270004968816270474FF0FF318162704710B5A5
:10C280000446206B01F034FA2046BDE8104001F06E
:10C290002FBA70B5044601F0A0F9884D04B92C6896
:10C2A000201D00F031FE58B9E06A824A00EB80019F
:10C2B00052F8211021B90121814028698843286161
:10C2C000A06A18B104F1180000F01EFE686A401C54
:10C2D00068622868844208D17748211D3C3000F00C
:10C2E000EFFD6868401C686007E0A868401EA86011
:10C2F0002046FFF7C4FFFFF7B3FF01F07AF9686942
:10C3000000280AD02868844207D16D494FF0805038
:10C310000860BFF34F8FBFF36F8F70BD2DE9F04101
:10C320000026664F386B002808D0B869401CB861F9
:10C33000F86900B101263046BDE8F081FD686D1C4A
:10C34000FD6045B9786BB96B7963B863386A401C96
:10C350003862FFF785FFB86ADFF8588185420DD350
:10C36000786B006838B1786BC068C46860688542D3
:10C370000ED2B86202E04FF0FF30B8623868C06A8F
:10C3800000EB800058F820000128D1D90126CFE722
:10C39000201D00F0B9FDA06A18B104F1180000F0EA
:10C3A000B3FDE06A01213A6981401143396100EB34
:10C3B000800008EB8000211D00F082FDE06A3968F2
:10C3C000C96A8842CCD30126CAE72DE9F04100248E
:10C3D000002701F002F9394D286B401E2863286BB5
:10C3E000F0BBA868E0B3DFF8D080012608F1280888
:10C3F0001DE0D8F80C00C46804F1180000F084FDBA
:10C40000201D00F081FDE06A2A6906FA00F111435F
:10C410002961284900EB800001EB8000211D00F01C
:10C420004FFDE06A2968C96A884200D3EE61D8F8F6
:10C4300000000028DDD10CB1FFF712FFAC6944B158
:10C44000FFF76CFF00B1EE61641E002CF8D10020F4
:10C45000A861E86920B1012719493807086000E0A0
:10C4600003E0BFF34F8FBFF36F8F01F0C2F8384680
:10C4700062E72DE9F04104460F46104EF56830683A
:10C48000001D00F041FD38B9306890F82C100120F3
:10C490008840316981433161601C08D13FB1316806
:10C4A000BDE8F0410448091D503000F009BD2C449E
:10C4B000306807E01C180060AC19006044000060A0
:10C4C00004ED00E04460AC4206D23168B06B091D57
:10C4D000BDE8F04100F000BD3168706B091D00F04F
:10C4E000FBFCB06A844200D2B46225E7FA48016BD3
:10C4F000491C0163704770B505460E460023FFF7DF
:10C50000F5FFF548C2682C68A119944205D98C4200
:10C5100008D9914206D9012304E08C4201D8914206
:10C5200000D9012329601BB1881A0021FFF7A1FF60
:10C53000FFF74BFF002807D1E8494FF08050086013
:10C54000BFF34F8FBFF36F8F70BD10B50246002051
:10C55000002A07D0FFF7CAFF00211046FFF789FF26
:10C56000FFF733FF002807D1DC494FF08050086007
:10C57000BFF34F8FBFF36F8F10BD10B5044601F0AE
:10C580002CF80CB9D4480468E46A01F032F820466B
:10C5900010BDBF22EFF3118182F31188BFF34F8FDB
:10C5A000BFF36F8F002801D1CB480068C06A81F3C8
:10C5B000118870472DE9F04104460D460026142DE0
:10C5C00000D3132501F009F8C34F04B93C68606C2F
:10C5D000A84241D0854208D939688C4209D03968CF
:10C5E000C96AA94205D8012603E039688C4200D106
:10C5F0000126D4F82C80404500D1E5626564A0692D
:10C60000002802DBC5F11400A061B54D08EB8801DC
:10C61000606905EB8101884215D1201D00F074FC92
:10C62000012120B93A6901FA08F082433A61E06ACF
:10C630003A6981401143396100EB800005EB8000CD
:10C64000211D00F03DFC3EB1A4494FF08050086030
:10C65000BFF34F8FBFF36F8FBDE8F04100F0C9BF4C
:10C660009D4A106B002802D00120D0617047002045
:10C67000D0611069B0FA80F0C0F11F00984900EB5A
:10C68000800001EB800041684968416000F10803C7
:10C69000994201D1496841604068C06810607047A4
:10C6A00070B5044600F099FF8B4D04B92C68201D2D
:10C6B00000F02AFC58B9E06A894A00EB800152F880
:10C6C000211021B901218140286988432861A06A8D
:10C6D00018B104F1180000F017FC211D814800F08A
:10C6E000EFFB00F086FF686928B100F076FFFFF7E6
:10C6F000B7FD00F07EFF2868844209D1686940B127
:10C7000076494FF080500860BFF34F8FBFF36F8FB3
:10C7100070BD7448A9680068884202D10020286072
:10C7200070BDBDE870409BE700216E4B42699A42A4
:10C7300006D1806AA3F12802904201D000B90121FC
:10C740000846704770B50446002C2BD0624D28680F
:10C75000844227D000F041FF2046FFF7E5FFE8B113
:10C76000201D00F0D1FBE06A01212A6981401143BC
:10C7700029615B4900EB800001EB8000211D00F086
:10C780009FFBE06A2968C96A884207D353494FF082
:10C7900080500860BFF34F8FBFF36F8FBDE87040CC
:10C7A00000F027BF70BD2DE9F04104460026BF20F0
:10C7B000EFF3118580F31188BFF34F8FBFF36F8FB5
:10C7C0002046FFF7B1FF40B1434F386B48B14548B1
:10C7D00004F11801283800F073FB85F31188304606
:10C7E000AAE5E06A3968C96A884200D30126201D9B
:10C7F00000F08AFBE06A01213A6981401143396106
:10C80000374900EB800001EB8000211D00F058FB50
:10C81000E3E770B5334E304D143E1CE0FFF766FE83
:10C82000306820B10024FFF7D0FDA4B901E0012455
:10C83000F9E700F0D2FEF068C468201D00F064FB48
:10C84000A868401EA8606868401E686000F0D1FEBD
:10C850002046FFF714FD68680028DFD170BD204E28
:10C860004FF080541D4DFFF7D4FF30680128FAD9EE
:10C870002C60BFF34F8FBFF36F8FF4E71CB51648E2
:10C8800000242C30CDE900402346802216A1184810
:10C89000FFF7B6FC012811D1BF2080F31188BFF348
:10C8A0004F8FBFF36F8F0C484FF0FF318162012132
:10C8B0004161C460BDE81C4000F07BBE1CBDBF20D0
:10C8C00080F31188BFF34F8FBFF36F8F02490020B1
:10C8D000486100F081BE00004400006004ED00E00B
:10C8E0001C180060FC19006049444C450000000021
:10C8F0005FC80008FE48C0687047FD48C0687047C0
:10C90000FB4880687047002801D1F948006834303E
:10C91000704710B50C46F6490968183100F0DCFA8A
:10C920002046BDE810400121A3E570B5154641F051
:10C930000043EF490C68A3610968183100F0C0FAA0
:10C940002846BDE87040012193E52DE9F041C0681B
:10C95000C46804F11800074600F0D6FAE44D2A6BCB
:10C9600001265AB13946E34800F0AAFAE06A29687C
:10C97000C96A884214D90120EE61DDE4201D00F06F
:10C98000C3FAE06A2A6906FA00F111432961DA491B
:10C9900000EB800001EB8000211D00F091FAE5E73B
:10C9A0000020C9E470B541F000410160C46800F0A6
:10C9B000ABFA201D00F0A8FACD4DE06A01262A69E5
:10C9C00006FA00F111432961CB4900EB800001EB2D
:10C9D0008000211D00F074FAE06A2968C96A884263
:10C9E00002D90120EE6170BD002070BDC0490A6A05
:10C9F0000260C9684160704770B504460D4600F09A
:10CA0000ECFDBB49C8682A68531C08D02368096A32
:10CA10008B4206D06168814203D801240DE00024D6
:10CA20000BE06168401A904206D2101A2860204636
:10CA3000FFF7DCFF002400E0012400F0DAFD2046CF
:10CA400070BDAB490120C8617047002101E0401C66
:10CA5000491C0278A52AFAD0880880B270470028BD
:10CA600001D1A3480068006BEFE7A1480068704758
:10CA70009F484169002903D0006B18B1002070471E
:10CA8000012070470220704770B50446002839D055
:10CA9000974DE06A2968C96A884233D2A0690028A4
:10CAA00004DB2868C06AC0F11400A061E06A924EFD
:10CAB00000EB8000616906EB800081421FD1201DE0
:10CAC00000F022FA012150B9E06A00EB800256F82A
:10CAD000222022B92A6901FA00F082432A612868DB
:10CAE000C06AE0622A6981401143296100EB80003D
:10CAF00006EB8000211DBDE8704000F0E1B9286818
:10CB0000C06AE06270BD70B504460020002C2CD0D5
:10CB1000A16C491EA164636CE26A9A4225D0002987
:10CB200023D1201D00F0F0F9734A7149012350B957
:10CB3000E06A00EB800552F8255025B90D6903FA2B
:10CB400000F085430D61606CE062C0F11400A061EB
:10CB5000E06A0D6983402B430B6100EB800002EB20
:10CB60008000211D00F0ACF9012070BD604908680B
:10CB700080690A680968D26AC2F114028A61704742
:10CB80005B490868002803D00868826C521C8264E4
:10CB90000868704770B506460C4600F01EFD544DFF
:10CBA0002868C06C80B92A68012082F850005CB106
:10CBB00001212046FFF75DFC50494FF0805008608E
:10CBC000BFF34F8FBFF36F8F00F013FD00F005FD33
:10CBD0002868C46C002034B116B12968C86402E02A
:10CBE0002A68611ED164296881F8500000F001FDB7
:10CBF000204670BD2DE9F04781460F4616469846FF
:10CC000000F0EBFC3A4D286890F85000022817D04D
:10CC10002C68E06C20EA0900E0642968012081F8B2
:10CC20005000B8F1000F0BD001214046FFF721FC66
:10CC300032494FF080500860BFF34F8FBFF36F8FC2
:10CC400000F0D7FC00F0C9FC16B12868C06C306059
:10CC5000286890F8500001280DD02868C16CB943AD
:10CC6000C16401242968002081F8500000F0C1FC53
:10CC70002046BDE8F0870024F4E72DE9F0410446A2
:10CC80000D4690461F46012600F0A7FC0FB1E06C50
:10CC9000386094F85000022184F85010B8F1050F64
:10CCA00013D2DFE808F01203070B0D00E16C2943F3
:10CCB000E1640AE0E16C491CE16406E0E56404E03B
:10CCC000022801D0E56400E00026012827D1201DBC
:10CCD00000F01AF9064DE06A01212A6981401143EA
:10CCE0002961054900EB800001EB8000211D07E070
:10CCF00044000060D41900601C18006004ED00E0DE
:10CD000000F0DEF8E06A2968C96A884207D96149FB
:10CD10004FF080500860BFF34F8FBFF36F8F00F06C
:10CD200068FC30465CE52DE9F0470446089F012683
:10CD3000BF20EFF3118580F31188BFF34F8FBFF34E
:10CD40006F8F002B01D0E06C186094F85000022324
:10CD500084F85030052A13D2DFE802F01203070BE3
:10CD60000D00E26C0A43E2640AE0E16C491CE164F4
:10CD700006E0E16404E0022801D0E16400E000265E
:10CD800001282BD1DFF81081D8F830004FF00109CD
:10CD900070B104F11801414800F092F8E06AD8F847
:10CDA0000010C96A884219D9B7B1C7F8009015E0D8
:10CDB000201D00F0A9F8E06AD8F8102009FA00F167
:10CDC0001143C8F8101000EB8001354800EB8100DA
:10CDD000211D00F075F8E1E7C8F81C9085F3118873
:10CDE000304646E72DE9F04104468846BF20EFF380
:10CDF000118780F31188BFF34F8FBFF36F8F94F8C3
:10CE00005010022084F85000E06C401CE0640129BE
:10CE100026D1214D286B012678B104F118011F4855
:10CE200000F04EF8E06A2968C96A884218D9B8F15A
:10CE3000000F14D0C8F8006012E0201D00F064F864
:10CE4000E06A2A6906FA00F111432961144900EBEE
:10CE5000800001EB8000211D00F032F8E2E7EE6176
:10CE600087F31188BCE410B500280BD0044600F00D
:10CE7000B4FB94F85000022807D0002400F0B9FB5E
:10CE8000204610BD04480468F1E7002084F85000F3
:10CE90000124F3E704ED00E044000060D4190060D1
:10CEA0001C18006000F1080141604FF0FF32826001
:10CEB000C16001610021016070470021016170477C
:10CEC00042684A6093688B6093685960916008611A
:10CED0000168491C0160704730B50C68621C02D0C3
:10CEE00000F1080202E0026904E01A4653681D6876
:10CEF000A542FAD953684B6099608A605160086115
:10CF00000168491C016030BD0169D0E901329A60B5
:10CF1000D0E901235A604A68824201D182684A609E
:10CF2000002202610868401E0860704770B5044620
:10CF30000D4600F052FBD4E90F12206801FB0200FD
:10CF400060600020A0632068A060E06B226C216814
:10CF5000401E00FB0210E0604FF0FF3084F84400F8
:10CF600084F8450004F110004DB1FFF79BFF04F178
:10CF70002400FFF797FF00F03CFB012070BD216902
:10CF80000029F8D0FFF7E1FC0028F4D0FF494FF06A
:10CF900080500860BFF34F8FBFF36F8FEBE70346FE
:10CFA0000098002904D00260C36301640121BDE739
:10CFB0000060F9E7F8B506460D461746002D10D07B
:10CFC00006FB05F0483000F048FB04463CB104F194
:10CFD00048023B46294630460094FFF7E0FF2046D2
:10CFE000F8BD0020EEE72DE9F041044600F0F5FA27
:10CFF00094F9455004F1240609E0606A48B13046CE
:10D00000FFF7A3FC08B1FFF71CFD6D1E6DB2002DEC
:10D01000F3DC4FF0FF3684F8456000F0EAFA00F0E8
:10D02000DCFA94F9445004F1100709E0206948B192
:10D030003846FFF78AFC08B1FFF703FD6D1E6DB29D
:10D04000002DF3DC84F84460BDE8F04100F0D1BA73
:10D0500010B5044600F0C1FAA06BE16B884201D123
:10D06000012400E0002400F0C4FA204610BD2DE9A0
:10D07000F041044617460026A56B226C002A10D00A
:10D08000C7B1E06835F064FEE168206C091AE16020
:10D090002268914202D26168081AE060022F16D01D
:10D0A00017E02068A8B96068FFF72DFD064600204C
:10D0B00060600EE0A06835F04BFE216CA06808446B
:10D0C000A0606168884204D32068A06001E005B1D7
:10D0D0006D1E6D1CA5633046BDE8F0812DE9FF474C
:10D0E00082B004468A4699460025A8464FF08056ED
:10D0F000A64F00F072FAA06BE16B884206D3B9F13B
:10D10000020F03D00498F8B115B325E04A46514602
:10D110002046FFF7ACFF616A51B104F12400FFF72C
:10D1200014FC58B13E60BFF34F8FBFF36F8F05E023
:10D1300020B13E60BFF34F8FBFF36F8F00F059FAFD
:10D14000012006B0BDE8F08700F053FA0020F8E7B0
:10D150006846FFF74BFC012500F04BFAFFF7C6F9D4
:10D1600000F03BFA94F94400401C01D184F844805B
:10D1700094F94500401C01D184F8458000F039FA4B
:10D1800004A96846FFF738FC30B12046FFF72BFFB3
:10D19000FFF71BF90020D4E72046FFF759FF88B1BD
:10D1A00004F110000499FFF7B4FB2046FFF71BFFC2
:10D1B000FFF70BF900289CD13E60BFF34F8FBFF300
:10D1C0006F8F96E72046FFF70EFFFFF7FEF890E718
:10D1D000002807D0002141600160C16000231A4689
:10D1E00019467BE7704710B5024600210120FFF782
:10D1F000E1FE04462046FFF7EBFF204610BD10B5C8
:10D200000446FFF732FC616888420BD1E068401E9B
:10D21000E06028B900231A4619462046FFF75EFF52
:10D22000012010BD002010BD10B5044600F0D5F956
:10D23000A06B20B1002400F0DCF9204610BD0124D1
:10D24000F9E730B40B46026C002A0CD0C1681144D7
:10D25000C1604468A14201D30168C160C16830BCAB
:10D26000184635F075BD30BC70472DE9FF4F83B0CF
:10D2700004468B469A460026B1464FF08057DFF8A9
:10D280000C8100F0AAF9A56B95B3E66859462046D3
:10D29000FFF7D7FFBAF1000F13D0E660606A50B114
:10D2A00004F12400FFF751FB28B1C8F80070BFF368
:10D2B0004F8FBFF36F8F00F09CF9012007B0BDE8DE
:10D2C000F08F6D1EA563206810B9FFF759FC6060F0
:10D2D00020690028EFD004F11000FFF736FB00288A
:10D2E000E9D0C8F80070BFF34F8FBFF36F8FE2E74C
:10D2F000FFE7059808B126B107E000F07AF90020B1
:10D30000DCE701A8FFF772FB012600F072F9FFF7D6
:10D31000EDF800F062F994F94400401C01D184F862
:10D32000449094F94500401C01D184F8459000F0E8
:10D3300060F905A901A8FFF75FFB58B12046FFF788
:10D3400052FEFFF742F82046FFF76EFF002898D004
:10D350000020B3E72046FFF767FF00B3206830B92D
:10D3600000F03BF96068FFF78FFB00F042F904F131
:10D3700024000599FFF7CDFA2046FFF734FEFFF7AA
:10D3800024F800287FF47DAF02E0000004ED00E007
:10D39000C8F80070BFF34F8FBFF36F8F71E720465F
:10D3A000FFF721FEFFF711F86BE770B504460D4655
:10D3B000FFF75BFB6368984204D1E068401CE060C3
:10D3C000012070BD00232A4619462046FFF74DFF75
:10D3D0000028F6D0E168491CE16070BD2DE9F041FC
:10D3E000174604461A46BF20EFF3118680F31188D2
:10D3F000BFF34F8FBFF36F8FA06BE36B984205D3E2
:10D40000022A03D0002086F3118865E694F945507E
:10D410002046FFF72CFE681C04D06D1C84F8455094
:10D420000120F0E7606A0028FAD004F12400FFF739
:10D430008CFA0028F4D0002FF2D001203860EFE7FA
:10D4400070B50D46BF21EFF3118481F31188BFF34E
:10D450004F8FBFF36F8F836BC16B994217D990F9D0
:10D4600045205B1C8363511C04D0521C80F845206E
:10D4700001200DE0416A0029FAD02430FFF765FA57
:10D480000028F5D0002DF3D001202860F0E700201F
:10D4900084F3118870BD2DE9F04104469046BF2009
:10D4A000EFF3118780F31188BFF34F8FBFF36F8FB6
:10D4B000A66B002E1DD094F944502046FFF7C1FE04
:10D4C000761EA663681C04D06D1C84F844500120AD
:10D4D00010E020690028FAD004F11000FFF735FAB7
:10D4E0000028F4D0B8F1000FF1D00120C8F80000F6
:10D4F000EDE7002087F31188EEE570B50446BF2004
:10D50000EFF3118580F31188BFF34F8FBFF36F8F57
:10D51000A06B002806D0E6682046FFF792FEE66082
:10D52000012000E0002085F3118870BD10B504468D
:10D5300000F053F8A46B00F05CF8204610BD10B565
:10D54000044600F04AF8D4E90E10441A00F051F8ED
:10D55000204610BD806B704700F0CAB8806B002871
:10D5600001D00020704701207047816BC06B814261
:10D5700001D101207047002070470000BF2080F3D8
:10D580001188BFF34F8FBFF36F8FFEE720384FF046
:10D590008073C36121F0010181612449416140F838
:10D5A000202970474FF0E0202149416107210161A6
:10D5B000704710B51F48016841F47F0101600168A0
:10D5C00041F07F410160FFF7EDFF1B49002008603B
:10D5D000FAF7CEFD002010BD7047BF2080F3118800
:10D5E000BFF34F8FBFF36F8F13480168491C016071
:10D5F000704711490868401E0860002801D180F377
:10D600001188704710B5BF2080F31188BFF34F8F8A
:10D61000BFF36F8FFEF782FE20B106494FF08050B6
:10D620001C390860002080F3118810BD7DD50008EA
:10D630003F19010020ED00E0800000603D4820F02F
:10D6400007003D49086000234B6008314EF6F87230
:10D650004A600B604260016070472DE9F04104466A
:10D660000026FEF743FF344D083D686818B9FFF700
:10D67000E5FF012068603CB10834600704D004F085
:10D680000700C0F108000444601E4EF6F77188429E
:10D6900029D2294A1046016801E00A460146486835
:10D6A000A04202D208680028F7D1234808308142FE
:10D6B00019D016680836086810604868001B1028E2
:10D6C0000DD90B1958604C605C681B4800E010468F
:10D6D00002685768A742FAD302681A600360486874
:10D6E0002968081A2860FEF770FE3046BDE8F08110
:10D6F00010B5002818D008380446FEF7F7FE606819
:10D700000D4900E011460A6853688342FAD308685D
:10D7100020600C60084861680838026811440160A4
:10D72000BDE81040FEF751BE10BD03480838006840
:10D7300070477047181A00608C000060704770B521
:10D740000446C24D40212846FCF727FE0028F9D0A8
:10D75000A1B22846FCF7B4FD204670BD2DE9F0418A
:10D7600086B00746012144F23400FBF734FCB74D84
:10D770002846FCF781FC6815ADF8140003208DF8ED
:10D78000160018208DF81700DFF8C48205A940465E
:10D79000FBF7FDF92E15ADF8146004248DF8174041
:10D7A00005A94046FBF7F3F9ADF8144010248DF8B5
:10D7B000174005A9A748FBF7EAF92001ADF81400C6
:10D7C0008DF8174005A9A448FBF7E1F925208DF84D
:10D7D000000000248DF8014001208DF802008DF832
:10D7E00003006846FAF757FE01979C4BAA1493F87A
:10D7F0005210022925D0012928D0ADF80C40ADF8EF
:10D80000084093F85510012927D0022928D0032970
:10D810002BD0ADF80A40ADF810400C20ADF80E004A
:10D8200001A92846FCF770FC012240F22551284648
:10D83000FCF7F1FC01212846FCF7E1FC06B0BDE84D
:10D84000F081ADF80C60ADF80820DAE74FF4C06065
:10D85000ADF80C00ADF80820D3E7ADF80A20DAE700
:10D860004FF40050ADF80A00D5E74FF44050ADF842
:10D870000A00D0E72DE9F04387B0804601218804F3
:10D88000FBF7B4FB01214820FBF7A5FB744D2846AC
:10D89000FCF7F2FB2E15ADF8186003278DF81A700F
:10D8A00018208DF81B00DFF8BC9106A94846FBF74D
:10D8B0006EF9EC14ADF8184004208DF81B0006A991
:10D8C0004846FBF764F9ADF8184010208DF81B00AE
:10D8D00006A96548FBF75BF927208DF804000024B2
:10D8E0008DF805408DF8067001208DF8070001A81D
:10D8F000FAF7D1FDCDF80880ADF80C405748AA14CE
:10D9000090F85410022925D0012928D0ADF81040F4
:10D91000ADF80C4090F85710012927D0022928D0E3
:10D9200003292BD0ADF80E40ADF814400C20ADF813
:10D93000120002A92846FCF7E7FB012240F225511C
:10D940002846FCF768FC01212846FCF758FC07B084
:10D95000BDE8F083ADF81060ADF80C20DAE74FF4C5
:10D96000C061ADF81010ADF80C20D3E7ADF80E2073
:10D97000DAE74FF40050ADF80E00D5E74FF4405011
:10D98000ADF80E00D0E72DE9F04387B0074601213E
:10D990004804FBF72BFB01210420FBF71CFB334E53
:10D9A0003046FCF769FB0424ADF8184003258DF8D8
:10D9B0001A5018208DF81B00DFF8949006A94846ED
:10D9C000FBF7E5F84FF00808ADF818808DF81B401C
:10D9D00006A94846FBF7DBF8204890F823100129F8
:10D9E00001D0052908D1ADF8188010208DF81B0052
:10D9F00006A91848FBF7CBF826208DF80400002470
:10DA00008DF805408DF8065001208DF8070001A81B
:10DA1000FAF741FD0297ADF80C40ADF80E40ADF8B5
:10DA20001040ADF814400C20ADF8120002A93046A9
:10DA3000FCF76AFB012240F225513046FCF7EBFB74
:10DA400001213046FCF7DBFB81E700000038014094
:10DA5000000801400010014000140140627304609E
:10DA600000480040000C0140001801400044004004
:10DA70004FF0E0210A6922F004020A61234AC0083B
:10DA800010704FF47A73584301235380486108693A
:10DA900040F00100086170472DE9F04100244FF08B
:10DAA000E0277E690546194800784543FFF795FD54
:10DAB000BA69B9699142FCD003D2A2EB01000444D7
:10DAC00003E0A6EB0100104404440A46AC42F0D344
:10DAD000BDE8F041FFF78DBD70B50446FEF7C8FF05
:10DAE00001280CD0094D6888844203D3B4FBF0F0C0
:10DAF000FEF72BFD6888B4FBF0F100FB11444FF4F6
:10DB00007A706043BDE87040C6E70000A000006086
:10DB100010B504466160FAF765FB206010BD01682E
:10DB2000426811440160704710B50446FAF75AFB89
:10DB3000206010BD10B50446FAF754FB2168401A66
:10DB40006168884201D3012010BD002010BD000093
:10DB5000FD490881704730B5C278FB4D0A44303525
:10DB6000D4B2EC70827802EB1122D2B2AA70437860
:10DB70006B7000782870B2EB112F05D25B1CDBB202
:10DB80006B700BB9401C2870C8B284420DD2521C75
:10DB9000D0B2A870002808D16878401CC0B2687064
:10DBA000002802D12878401C287030BD10B58B1891
:10DBB0005B1E0BE04A780C7802EB042292B2104410
:10DBC00080B2904201D2401C80B2891C9942F1D3AC
:10DBD000994207D109780902084480B2884201D2EB
:10DBE000401C80B210BD010241EA102080B2704793
:10DBF00010B50A4601460020FFF7D8FFBDE81040E7
:10DC0000F1E710B51422D1490020FFF7CFFF10B182
:10DC1000BDE81040E7E74FF6FF7010BD10B5CB49E7
:10DC20006FF013030E394A7C097C03EB0121114488
:10DC30008CB2204480B2C54908220C31FFF7B6FFF0
:10DC4000C24922461431FFF7B1FF10B1BDE81040C0
:10DC5000C9E74FF6FF7010BD0620DFE71120DDE7B2
:10DC600070B5B94900224A70B94B487823F81020A2
:10DC7000401CC0B248700A28F7D34A70B54BB42490
:10DC800003F2FE35487800EB800606EB40161E4492
:10DC900072762C54401CC0B248700A28F2D34FF45C
:10DCA000806048814A70AA4B1433487800EB4004E6
:10DCB000C4EB401403EB4404A280401CC0B2487083
:10DCC0000A28F2D370BD70B5002200230021A04CB9
:10DCD0004DF204261434050245EA102085B201EB0A
:10DCE0004100C0EB411004EB40008088B04200D1FD
:10DCF0000122854200D10123491CC9B20A29EED371
:10DD000002B17BB994480068B0F5967F0AD93C21EE
:10DD1000B0FBF1F201FB120020B99049012008701C
:10DD20008F49088000208B4C002504F2FE33B42676
:10DD300000EB800101EB40110A19517E31B1195CF1
:10DD400011B1491E195401E055761E54401CC0B251
:10DD50000A28EDD370BD2DE9F041074688467D4C79
:10DD6000794D4FF4FA4300266889401C80B26881DF
:10DD7000984202D34FF4805068816E70687800EB4F
:10DD8000800101EB40100219507E28B16889FFF72D
:10DD90002AFF91888842E7D06878401CC0B268703A
:10DDA0000A28EBD300226E70687800EB800101EB4B
:10DDB00040110B19597E11B1072902D008E01A460B
:10DDC0000BE022B1997E92F81AC0614500D91A463B
:10DDD000401CC0B268700A28E6D32AB302205076ED
:10DDE00059482C30017811734178517381789173BF
:10DDF000C078D07340F6CA705082908201201082A1
:10DE0000D67690760320107696751020D0756889A6
:10DE1000FFF7E9FE9080A2F80680388810807888A5
:10DE200050801046BDE8F0810020FBE72DE9F0416D
:10DE300005460F46464C0026434B4FF4FA484FF434
:10DE4000805214345889401C80B25881404500D318
:10DE50005A815E705889FFF7C6FE0146587800EB7C
:10DE6000400CCCEB401C04EB4C0CBCF804C06145EE
:10DE7000E8D0401CC0B258700A28EBD300205E7076
:10DE80005A7802EB4201C1EB421104EB410189884F
:10DE900099B1521CD1B259700A29F1D3A8B159894C
:10DEA0000A0242EA11218180C78085B12988018058
:10DEB0006988418040210172B4E7587800EB400145
:10DEC000C1EB401004EB4000E8E70020AAE7066041
:10DED000F0E730B51C4A002555701D4B517833F8DA
:10DEE0001140844203D1507823F8105030BD491CB2
:10DEF000C9B251700A29F1D330BD10B5124A0021C0
:10DF00005170134B517833F811402CB1491CC9B2F0
:10DF100051700A29F6D310BD517823F8110010BDB5
:10DF200010B5094C0146606A0830FFF714FE04F191
:10DF30003001606A0A7802724A7842728A78827284
:10DF4000C978C17210BD0000AC0000601E0A0160FB
:10DF5000841B0160121A0160B80300603C0000607D
:10DF6000A60300602DE9F04F85B0DFF8FC93D9F8E7
:10DF70002440FE4D002605F136014FF6FF7804914E
:10DF800004287AD00499C9F81C10C9F820104FF061
:10DF9000100A032815D0022821D005F12A040528EB
:10DFA0006CD0F34F7888401C78803846A97B008875
:10DFB000401C80B2452963D03880F888401CF88026
:10DFC000ACE0607E00F00F000328F9D1208A002821
:10DFD000F6D1082089F8000002F0BCFDFEE3E2491A
:10DFE0002C31C878401C10F0FF00C8700ED1887822
:10DFF000401C10F0FF00887008D14878401C10F0D9
:10E00000FF00487002D10878401C0870A9F804602D
:10E01000A9F80660607E072812D0052810D00028D5
:10E02000CED0218A59B3A07E411EA176C8D2E07E0F
:10E0300008282DD0617E02290AD0012908D009E0E4
:10E04000A07E401CC0B2A0767828B9D1667665E083
:10E0500005281DD0042800D9042003218140A17681
:10E06000E07E401CE076C248C18C491CC184607EC1
:10E0700000F00F000928A3D203E0E2E125E01AE056
:10E0800038E0DFE800F04BFD0F12FC4BFC4BFC00CE
:10E090006676802089F8000002F05CFD142085F887
:10E0A0002F00EEE385F82F6012E3042089F80000CA
:10E0B00002F050FDF3E300F00F000328C7D1082061
:10E0C00089F8000002F046FD88E3D9F8280080882E
:10E0D0000028BCD0C9F82460C9F81C40C9F8204009
:10E0E000A9F80660A9F80460082089F8000002F089
:10E0F0009BFBA6E1697C2A7C01EB0221B9F8042094
:10E100009142A4D8CB46A9F80410297D890601D1F3
:10E11000697D21B13880B889401CB881C6E1924937
:10E120000E31B1F800E049880391BEF1000F01D132
:10E130000399C9B18D4AEB7DD18B128C112B0CD177
:10E14000414501D142455ED0874B1633B3F800C03C
:10E15000614502D15B889A4255D0714502D103993D
:10E160008A4201D03880A1E1FFF74BFD404506D03F
:10E170003888401C3880F889401CF88196E1E87D99
:10E1800006280AD011283ED0012814D03888401C17
:10E190003880388A401C388288E1B88B401CB883AC
:10E1A000FFF75AFD40456CD0788B401C7883388C43
:10E1B000401C38847AE1B88A401CB88295F8220065
:10E1C000082806D0788A401C7882388B401C388317
:10E1D0006CE185F82260A88C4FF6F771884202D373
:10E1E0000930A88401E00830A884688BE883A88BF4
:10E1F00028845D480E30018869834088A883F88AA6
:10E20000401CF882FDE3BBF804001C38ABF80400A6
:10E21000CBF81C40288DAA4650B1FFF71FFD4045A2
:10E2200006D0B88D401CB885788E401C78863DE1BC
:10E230005048CBF828004E4F33E1818800297DD02B
:10E24000BAF824208A4279D102880AB94388ABB34C
:10E25000424502D14388434530D0BAF81A30934240
:10E2600004D1BAF81C2043889A4227D0BAF81E205D
:10E27000424503D1BAF8203043451FD002E080E385
:10E2800024E217E1DFF8E0C00CF10E0CBCF800301E
:10E290009A4205D1BAF82030BCF802C063450DD0CF
:10E2A000DFF8C4C00CF1160CBCF800309A4245D11E
:10E2B000BAF82020BCF802309A423FD1DBF828207F
:10E2C000D28812B1B1F5884F7AD0BAF82220C28034
:10E2D0000292BAF81A20ADF80420BAF81C30ADF852
:10E2E0000630DBF8123000939DF800709DF8043082
:10E2F000C7F1FF073B438DF804309DF801709DF88E
:10E300000530C7F1FF073B438DF805309DF80270DB
:10E310009DF80630C7F1FF073B438DF806309DF8A6
:10E3200003709DF80730C7F1FF073B438DF80730B6
:10E330000D4FBDF804C016373B8800E0AEE09C45A9
:10E3400005D1BDF806C0B7F802E0F4450BD090F84F
:10E3500004C04FEA0C2C4CEA112189B2A1F5806C63
:10E36000BCF1D20C2DD007E0AC000060100A0160B7
:10E37000DC1D0160981B0160BAF81E10414503D1F5
:10E38000BAF820C0C44507D0994249D1BAF8201044
:10E39000B7F802C0614543D1FE4909884FEA012C14
:10E3A0004CEA1121DDF808C089B261451BD1B0F8F3
:10E3B00004C0614517D19AF83410102906D009E03D
:10E3C00032E0A0F80080A0F802802DE09AF8351025
:10E3D000082904D00280BAF81C10418024E0038090
:10E3E0007988418020E00299A1F5884CBCF5CE7C6B
:10E3F00004D09AF83410102905D008E00280BAF849
:10E400001C10418010E09AF83510082904D00280D1
:10E41000BAF81C10418007E003807988418003E04E
:10E420000280BAF81C104180CBF8246002208BF8DF
:10E430000000CBF81C40CBF82040ABF8066002F09F
:10E44000F3F9B9F80600002830D000F11C01A9F852
:10E4500004100A0A2A7469741121E9750830C0F39E
:10E46000072141EA0020E8842E85D9F82800818818
:10E470006984C188A984C8490A886A834988A983AC
:10E480000188E983408828840498C9F81C00FFF7B4
:10E49000E5FBC04380B2288548B1A0E33A30CBF811
:10E4A0002800DBF82800B842FFF4C7AE7AE3A5F8ED
:10E4B000288094E3B94CB5F822C0B5F81A80A98B2E
:10E4C00004F24D13A88C1DE0627ED2B1A288904266
:10E4D00017D1E288944514D12288904511D16288E1
:10E4E00091420ED1CBF824408BF8006095F82F00B4
:10E4F00041076ED5667620208BF8000002F02AFBDB
:10E5000050E325349C42DFD995F82F1001F03F01EC
:10E51000022918D1ABF80C008BF80160A04A9BF8D7
:10E52000011032F81130834204D100248BF80160CD
:10E530009A4B4FE0491CC9B28BF801100A29EED35F
:10E54000788D401C788595F82F004007AED4B88CA4
:10E55000401CB8841420263568722820ABF80400CB
:10E5600050202872EB78E879E870A978A879A8702B
:10E57000A9716A78687968706A7128788BF80100E7
:10E580002C792C7028715B1C13F0FF03EB71A5F143
:10E5900026050ED1491C11F0FF0185F82C1008D179
:10E5A000521C12F0FF0185F82B1002D1401C85F897
:10E5B0002A00688CABF80C00A98C6984A884688B4D
:10E5C000E883A88B28847448018869834088A883DD
:10E5D000F5E2A4E09BF8011001EB810000EB411093
:10E5E0001844427E12B1072A08D00EE09BF80100C1
:10E5F00000EB800101EB4010C4180CE024B1827ED6
:10E6000094F81AC0624500D90446491CC8B28BF878
:10E6100001000A28DED3B4B3CBF824400320A0764F
:10E620002076A6750420E075E6761A356889A08004
:10E630002889E080288820806888608001216176B0
:10E6400055481E3002782273427862738278A27332
:10E65000C078E0732182E87BE072A87BA072687BBF
:10E660006072287B20720120FFF75AFC287D1A3D3A
:10E6700000F0F001502929D98BF801606FF00401F6
:10E6800001EB10131DE0FFE7388D401C388589E24F
:10E690002A1892F836108BF80210B9B1012902D06D
:10E6A000022904D007E0401C8BF8010009E092F831
:10E6B0003710042920D092F8371039B108448BF86C
:10E6C00001009BF80100B0EB830FE1DB85F82FA080
:10E6D0002E35687840F0020068700220287204200D
:10E6E00068720F20A872CA20E8722C20A9F80400D2
:10E6F000602005F82E0920E29BF8010092F83810FE
:10E70000284490F8390040EA0120ABF80C0040F6AC
:10E71000CA71884200D908466082A082D6E795F87F
:10E720002E10A846090989008BF80110BBF80420B7
:10E73000511A143989B2ABF80410627E02F00F024C
:10E74000022A03D100F03F02122A17D009B981072B
:10E7500014D098F82610227A434691427DD193F83E
:10E760002710627A9142F9D193F82810A27A914247
:10E77000F4D193F82910E27A9142EFD1C00649D53D
:10E78000218A61B304F10C00FFF7E5F9C64698F859
:10E790002A1007E0E2010060BA000060121A01606E
:10E7A000841B0160FA4B1878814233D19EF82B20EC
:10E7B00059788A422ED19EF82CC09A78944529D156
:10E7C0009EF82DC0DB789C4524D120736173A27321
:10E7D000E373E07EC0B9207EA17E01E010E119E084
:10E7E000401AA17DA0EBD10040B20144C9B2A1758D
:10E7F000002801DA404240B2E27DA0EB92001044D2
:10E80000E07500EBD100207601208BF80000207E1F
:10E81000A0762682627E02F00F0009287BD2DFE814
:10E8200000F07A051D8EF4F3F21CF1009BF8000055
:10E83000C00770D00320607640208BF8000026824D
:10E84000BBF8040020B142218BF80010FFF768FBF1
:10E85000ABF8066002F07EF9D2E066E19BF80000BA
:10E86000C00705D098F82F0000F03F00122809D00B
:10E8700020208BF8000002F06DF9DBF824004676CA
:10E8800061E654E198F82E0000F0F001502926D9F5
:10E890008BF801606FF0040101EB10131AE0D8E06F
:10E8A00008EB000292F836108BF80210B9B101297A
:10E8B00002D0022904D007E0401C8BF8010009E0D7
:10E8C00092F83710042927D092F8371039B108444C
:10E8D0008BF801009BF80100B0EB830FE0DB032015
:10E8E000607698F82600207298F82700607298F8F1
:10E8F0002800A07298F82900E0720120FFF710FBB1
:10E9000042208BF800002682ABF80460ABF806606A
:10E9100002F020F974E058E09BF8010092F83810FA
:10E92000404490F8390040EA0120ABF80C0040F672
:10E93000CA71884200D908466082A082CFE798F861
:10E940002F00C10721D0D1061FD4208AE8BBBBF815
:10E950000400401C80B2FFF7E3FA9BF8000040F08F
:10E9600010008BF80000BBF8041019B140F0020051
:10E970008BF8000002F0EEF801202082082060767B
:10E98000E676112085F82F00D1E080060FD598F8A3
:10E99000350098F8341040EA0120DBF81C100144DF
:10E9A000CBF81C10BBF80410081AABF80400BBF835
:10E9B000040048B1D10607D49BF8001041F00201D1
:10E9C0008BF80010FFF7ACFA00E06EE098F8310029
:10E9D00098F8301000EB012080B2ABF80C00A18A4F
:10E9E000814200D308B9ABF80C10BBF80C00608270
:10E9F0009BF80000800758D0ABF8066002F0AAF838
:10EA000004E004E148E0C6E078E04FE099F8000057
:10EA1000810606D5A9F806606676142085F82F00D1
:10EA200085E0C1060AD5A9F80660012020820420ED
:10EA30006076E676112085F82F0078E0B9F80610A8
:10EA400031B1C00700D02682208A90B1A9F8060013
:10EA5000E676D9F82000C9F81C00B9F8060088B19C
:10EA6000208A78B12830A9F80400182085F82F00F2
:10EA700060E0608A884201D2A9F80600B9F8060071
:10EA80002082E5E799F8000080070ED52820A9F834
:10EA9000040085F82FA04DE09BF80000C00704D0CB
:10EAA00066768BF800A002F055F87BE0BBF8040016
:10EAB00008B1FFF735FA98F82F00C00712D09BF87D
:10EAC0000000C00704D007206076A676268201E009
:10EAD000062060760120FFF723FA8BF800A002F0F1
:10EAE00039F822E09BF80000C00703D005206076CB
:10EAF000268257E0BBF80400B8B953E0BBF8040025
:10EB000008B1FFF70DFA98F82F00C0070AD00720C8
:10EB10006076A6760120FFF703FA8BF800A002F0DA
:10EB200019F802E0BBF80400A0B388F82FA0282051
:10EB3000A9F80400502085F82E001835207AA87412
:10EB4000607AE874A07A2875E07A6875207BA873EB
:10EB5000607BE873A07B2874E07B6874062005F86E
:10EB6000010CA0886881E088A881094822380188C2
:10EB700069804088A8802088E88060882881183DC6
:10EB8000607EC00615D585F8316085F8306016E0E6
:10EB9000DC00006006E09BF80000C00702D0072000
:10EBA0006076A676A9F8046089F8006005B0BDE833
:10EBB000F08F0F2085F83000CA2085F83100402002
:10EBC000A875B9F80400010A2974687485F83560DD
:10EBD00085F834606E86FFF73FF8C04368864520AD
:10EBE000A873EE736E752E754020A875B9F80800ED
:10EBF000401CA9F80800010AA974E8742E83FFF7E5
:10EC000000F8C04328830C49C88B401CC8830A49BC
:10EC10008888401C888089F80060C7E7034600297F
:10EC200008DD06488AB2C280006A834202D01946D3
:10EC300034F08EB870470000DC1D0160AC0000604D
:10EC400010B5C04900220A70BF4B087800EB4004A1
:10EC500004EBC0041C442260401CC0B208700828A9
:10EC6000F3D310BDF0B5B74A9078401CC4B294708D
:10EC700000231370B44D117801EB410000EBC1008B
:10EC80002844068847883E4304D0867AA61B782EFF
:10EC900000DB0360491CC8B210700828EBD3F0BD3C
:10ECA0002DE9F041A74F4FF0000C87F800C0A64EA9
:10ECB0003A7802EB420303EBC20333441C8884B16D
:10ECC0005D8875B1B0F80080A0450AD14488AC4297
:10ECD00007D10868586088881881B8789872BDE8AC
:10ECE000F081521CD2B23A70082AE1D387F800C0F2
:10ECF0003B7803EB430202EBC302324414880CB9A5
:10ED0000548824B15B1CDBB23B70082BF0D33B78FA
:10ED1000082B1FD187F803C087F801C087F800C00F
:10ED2000BC783A7802EB420303EBC2033344FD782C
:10ED30009B7AE31AAB4201DDFB707A70521CD2B2AF
:10ED40003A70082AEDD37A783A7002EB420303EB6B
:10ED5000C2023244006810600868506088881081E0
:10ED6000B8789072BBE72DE9F047784D00202988EC
:10ED70002A2902D22880BDE8F0872880744C754F7C
:10ED8000224602F11601B4F81490B2F826C0881D8C
:10ED9000B7F80080128D7B884FF40076B9F5807F3C
:10EDA00008D0B145E7D1C445E5D19A42E3D1BDE8E9
:10EDB000F04775E7C445DED19A42DCD1FFF770FF1A
:10EDC000A682D4F816002062618BA184624B1A6877
:10EDD000C4F816209B886383C4F8062063812060F2
:10EDE000A180A08BE084E08B20853888A083788880
:10EDF000E0834FF4C160A0812A202880BBE72DE981
:10EE0000F05FDFF84CA1544B5046BAF81E104FF695
:10EE1000FF72008C9C881D68914201D1904206D0FF
:10EE20004E4A138899420AD15288904207D14C48E1
:10EE30000168CAF800108088AAF8040040E0454F35
:10EE4000484BB7F800901A88B7F802803D4F01EAA6
:10EE5000020609EA02023F1D964206D15A8800EADC
:10EE6000020308EA0202934205D03F480188398034
:10EE70004088788001E039807880324B4FF0000B79
:10EE800083F800B03E88DFF8C0C07F88197801EBB6
:10EE9000410000EBC10060440288964202D14288E2
:10EEA000974204D0491CC9B219700829EED31978C9
:10EEB000082912D04168CAF800100089AAF8040095
:10EEC000CAF80650AAF80A400820AAF80C001F4801
:10EED00001880E310180BDE8F09FFF2206211C4809
:10EEE00033F048FFCAF820B0AAF824B0CAF8065098
:10EEF000AAF80A40CAF81650AAF81A40AAF82660DA
:10EF0000AAF82870AAF81C90AAF81E804FF4807006
:10EF1000AAF81400AAF80E000820AAF8100006208B
:10EF20008AF8120004208AF813004FF4C160AAF88E
:10EF30000C0007480D493630086004482A2101803A
:10EF4000C9E70000E40000601A1E0160B000006024
:10EF5000100A0160BA000060A4000060C2000060F6
:10EF6000885B0408BE000060E0000060C80000602C
:10EF70002DE9FC4751480546FCF79AFA0646002061
:10EF80004E4C4F49133C2218D27C0A54401CC0B24C
:10EF90000628F8D340F276411420FCF76CFAFEF70D
:10EFA0005FFEA07B40B10621284600F05EFA00F02B
:10EFB00078FA3046BDE8FC87237CE17B43EA0120F8
:10EFC000020242EA1027A27C657C42EA05204FEA51
:10EFD000002C4CEA1020DFF8ECC0ACF80070ACF864
:10EFE0000200A07F677F40EA0720070247EA102758
:10EFF00094F8200094F81FC040EA0C204FEA002C3F
:10F000004CEA1020DFF8C0C0ACF80070ACF8020089
:10F01000A07E94F819C040EA0C274FEA072848EA76
:10F020001729ADF80490277FE47E47EA04284FEAC9
:10F03000082A4AEA1828ADF80680DFF890A0AAF856
:10F040000090AAF80280CCF1FF0C41EA0C018DF887
:10F050000010C0F1FF0003438DF80130C4F1FF0040
:10F0600005438DF80250C7F1FF0002438DF80320DD
:10F0700043EA0120040244EA1020154C208042EAB1
:10F080000520070247EA1020608002EB05201A04E1
:10F0900002EB016108440F4908600120FEF71CFDE6
:10F0A00087E710B50C4940F2EE50FCF702FB80B246
:10F0B00010BD0A4808490088FCF7B2BA75730460AD
:10F0C000A4000060BA000060E0000060BE000060C4
:10F0D000C20000603C010060100A0160B0000060E6
:10F0E00035220270012242708170C01C70473621A7
:10F0F000017004214170F149D1F81910C0F80210D3
:10F10000801D70473221017004214170EB49D1F814
:10F110002110C0F80210801D7047372101700321B3
:10F12000417001228270C17006210171401D70473B
:10F13000FF2100F8011B70472DE9F0410446012032
:10F1400020706070DD4D11352879A0700020E070CE
:10F15000DB4E31686160208180216181D949096875
:10F16000E16020616061A06104F11C006A682968A7
:10F17000074633F0EDFD6868C0F11001384433F004
:10F1800000FE402104F12C0033F0FBFD802104F14E
:10F190006C0033F0F6FD7068C4F8EC00BDE8F08157
:10F1A00070B5C94D2C682046FFF7C6FF012104F158
:10F1B000F000FFF795FFFFF7B0FFFFF7B9FF01463B
:10F1C0002868BDE87040091AFFF728BD70B5BE4D2C
:10F1D0002C682046FFF7B0FF032104F1F000FFF791
:10F1E0007FFFFFF784FFFFF78DFFFFF7A1FF0146C9
:10F1F0002868BDE87040091AFFF710BD10B5441823
:10F200000023AE4A2EE00178332924D006DC012900
:10F210000BD003290ED0062921D110E0352913D0B7
:10F22000362913D0FF291AD120E0D0F80210C2F8F5
:10F23000251014E0D0F80210C2F82D100FE0D0F81D
:10F240000210C2F829100AE0837808E0D0F8021012
:10F25000C2F8191003E0D0F80210C2F81D1041786E
:10F26000801C0844A042CED3184610BD184610BDDD
:10F2700070B595480468207802280FD1042290497F
:10F28000201D33F0C4FD48B98C4D04F11C00D5F8A5
:10F290001520D5F8111033F0BAFD08B1002070BD6B
:10F2A0002069C5F821008948018804F1F000BDE813
:10F2B0007040A3E710B581490020C91C0A689080FE
:10F2C0008348C27B037C02EB0322CA83427C837C9B
:10F2D00002EB03220A84427E837E02EB03224A84ED
:10F2E000C27E037F02EB03228A84427F837F02EB8C
:10F2F0000323CB84C27F90F8204002EB04220A85CE
:10F300004B858A850221817310BD2DE9F0470121CB
:10F310006A4C4FF4BD77002520886E4E4FF4D678A6
:10F32000B8424AD007DC4FF47A7958B1A0F5807022
:10F3300051386FD114E040456DD04FF4D9729042EE
:10F3400068D189E00120A070A4F80F90FFF728FF92
:10F35000B4F80F10E01DFEF7DBFB40F251102080E7
:10F360003078800703D4E01DFEF7E4FBE8B3307883
:10F37000800703D5FFF77CFF022843D0B4F80F00C5
:10F380004EF66021884205D24FF6FF7101EA400037
:10F39000A4F80F00B4F80F00B0F57A5F3FD2A07860
:10F3A0000228D3D1A4F80F903570FFF70FFFB4F8FF
:10F3B0000F10E01DFEF7ACFB27803078800703D4E8
:10F3C000E01DFEF7B7FB00B33078800703D5FFF7E9
:10F3D0004FFF05281BD0B4F80F0042F2107188428D
:10F3E0001AD800F57A7080B200E008E0A4F80F00A7
:10F3F000B0F5FA5F13D2A0780328D6D111E000202F
:10F40000BDE8F0870220A070CCE70020F8E70320D9
:10F41000A07006E026E019E025800020F0E7FFF765
:10F4200049FF264801F0FEFBB4F81F00FEF7DBFBA6
:10F430008146B4F81D00FEF7D6FB09EB00413220EF
:10F440004143E01DFEF764FBA4F80080E01DFEF7D9
:10F4500071FB0028A9D1D3E711B100212280FBE77D
:10F460000320CDE725800220CAE738B5134CC4F845
:10F470001100C4F815100025A5704FF6FF70ADF807
:10F480000000ADF802004FF486416846FEF7CEFC5E
:10F49000C4F8030010B14FF488418180258038BD45
:10F4A00033E708B505488078002806D1ADF800009C
:10F4B000ADF8020003490880488008BD721E016053
:10F4C0008E5B0408BA000060C8000060B0000060F5
:10F4D00062730460AC0000600B0A0370417000218D
:10F4E0008170C170110A017142717047F14A03784D
:10F4F00013704378537000239370D37013710323F8
:10F50000537183799371C07940F08000D07111728A
:10F51000E949092088807047E84800681C30D0F825
:10F520000510002903DDD0F80100FFF777BB704715
:10F53000E24800680021C0F821107047DF480068E9
:10F54000DD498A7842F080028A7000210177C0F894
:10F5500021107047D848817821F080018170704770
:10F56000D548817821F0800181707047D248817838
:10F5700021F08001817070472DE9FF5F0024CF48A2
:10F5800006681C36DFF838B39BF80000800601D50A
:10F59000FFF7ECFF9BF80000000601D5FFF7E0FF46
:10F5A0009BF80000C00601D5FFF7D4FF9BF80000D0
:10F5B000400601D5FFF7C2FF9BF80000C00701D04D
:10F5C000FFF7B6FF9BF80000BB4F800732D5BE485F
:10F5D000BC4D01682A88BD4833F0BAFBDFF8EC82E5
:10F5E0004FF0010A98F80000EE2815D198F80100B4
:10F5F000102811D198F8020070B998F8030058B992
:10F6000098F8040040B998F8050028B998F8060061
:10F6100010B998F8070050B1AD4C98F806104FF0AB
:10F620000009207981420AD0FF2904D00FE001248B
:10F6300087F803A024E198F80700192807D00124CF
:10F64000A7F80490A149012018F07AFA18E10029DE
:10F650007ED098F80700032813D0062811D0102870
:10F660000FD019280DD001280BD0022809D004286A
:10F6700007D0052805D00F2803D0182801D0FF286F
:10F6800066D1102805D198F80C002A88101A0D2888
:10F690005ED1387828B106218C48FFF727FF012476
:10F6A000EEE08C480278002A52D0D8F80000009092
:10F6B000D8F804000190884B78781B5C521E904269
:10F6C00002DA401C787001E087F8019084F8243059
:10F6D0000020DFF810C2814A4FF0020E804B9CF8E8
:10F6E00000C017E012F80080414502D184F824E000
:10F6F0000EE0DFF8F48118F80080414502D184F86B
:10F70000249005E013F80080414501D184F824A03D
:10F71000401CC0B26045E5D394F823000A2801D10B
:10F7200084F824907148007808B1022803D1704809
:10F730000068FCF7B5FF6F4880F800A06E4880F8BD
:10F7400000906E480068FCF7ABFF6D48006800E071
:10F75000AEE0FCF7A5FF6B480068FCF7A1FF6A4824
:10F760000068FCF79DFF5A4890F82300012807D055
:10F77000052805D0022803D0062801D0032803D18C
:10F7800062480068FCF78CFF614880F84B900124C8
:10F79000A7F80490DFF83481032198F807000228C5
:10F7A0002BD0012829D003282DD004282BD00622C5
:10F7B0009DF801009DF8001040EA012102A8FFF722
:10F7C0008BFE2888801F85B24FF48070854200D957
:10F7D00005462A4608F106014E4833F0B9FA87F883
:10F7E00000A0DFF8EC8002AB294698F824204948B5
:10F7F00016F0D5FBB88858B114E098F80B00C01D7E
:10F8000001EBD002D4E798F80B0001EB4002CFE700
:10F810001420FEF761F998F8242002AB29463D48F0
:10F8200016F0BDFB87F80090B88818B90B21684620
:10F83000FFF75CFE2D4880F800A0374880F8009064
:10F840002E480068FCF77EFF2D480068FCF77AFF21
:10F850002C480068FCF776FF2B480068FCF772FF25
:10F8600098F82300012807D0052805D0022803D0E6
:10F87000062801D0032803D124480068FCF762FF62
:10F880009BF8000000F0040100F00202114305D1D2
:10F89000C10703D1410601D4000709D5012C07D1C6
:10F8A000044846F8010FB8887060BDE8FF5F33E692
:10F8B000BDE8FF9FCF200160EC000060D000006039
:10F8C000AC000060B0000060C8000060A31F0160D1
:10F8D00062730460090300602403006092460460C0
:10F8E0002E460460F0020060CA450460EF03006029
:10F8F0002803006044020060450200608C04006040
:10F900002C04006038040060280400607404006067
:10F910004C7D0460A31E0160F003006038B54DF219
:10F9200004242046FEF7E9FA4FF0FF32042168462E
:10F9300033F020FA21466846FEF778FA002800D016
:10F94000848038BD70B505464321FD4833F019FA6F
:10F95000FB4C15B1012D03D004E06520208001E0AF
:10F96000672020801D206080F64D2878A080687870
:10F97000E080A8782081E878608195F8230008B9B4
:10F980003221A181411F032944D90C2842D02320D0
:10F99000A0812879E081E87B2082287C6082687CD5
:10F9A000A082A87CE082B5F921002FF094FA208390
:10F9B00040F2B1202FF08FFA6083E8792FF08BFAB4
:10F9C000A083E1480068C0F3072141EA0021618477
:10F9D000DE49097884F82410010C090241EA10601C
:10F9E000A4F83900002084F83B00B5F84910A1873D
:10F9F000D749097884F83E1084F83F000A2184F83A
:10FA0000401084F8410084F84200D24901220A7073
:10FA1000487070BD4A20A081BBE738B5CD4C0025A9
:10FA2000206A002800D08580A068C0F3072141EA41
:10FA30000022C3B2120241EA032142EA1121ADF8C9
:10FA40000010C0F30741090241EA1060010241EAD7
:10FA50001020ADF80200A089C0F3072141EA002080
:10FA600081B26846FEF7E2F92062002806D0BA4962
:10FA700009880A0242EA11218180257138BD2DE9E9
:10FA8000F04F89B000250024B44890F800A0BAF1E6
:10FA9000430F05D8B24852460168B24833F058F9CE
:10FAA000B04F0126DFF89C8238784FF000096428B7
:10FAB00003D0062266287CD07BE2A64B012018707A
:10FAC000787800B9B87898F8101098F8112098F85C
:10FAD000126098F80FC014E007EB850090F801B0B1
:10FAE000E3450CD190F802B08B4508D190F803B0F3
:10FAF000934504D10079B04201D183F800906D1C88
:10FB0000EDB2B5EB9A0FE7D3187800287ED000202D
:10FB1000FFF718FF8A4D0020A877E87785F82000C6
:10FB200085F8210005F1250014228F49089033F053
:10FB30000FF9204600EB400101EB8010641C05F139
:10FB40004307E4B238444322294633F001F9002642
:10FB50006FE0DFF818C2C6EBC60101EB0C02937927
:10FB6000DC2B0FD21CF80100DFF8049200F0070A2A
:10FB700009EBD009012099F8009000FA0AF019EA7F
:10FB8000000F54D0232B52D098F802A098F800C050
:10FB900098F8019098F803E04FEA0A4B0CEB092023
:10FBA0000BEB0E6B8344D2F8010083453FD0A88055
:10FBB00000E04DE1C0F3072BA5F806B0C0F3074BFA
:10FBC000A5F808B0000E6881AB816848405CE88108
:10FBD00000206884A5F83900012085F83F0085F8E9
:10FBE0001EC085F81F9085F820A085F821E0507987
:10FBF00000F00F01491E85F84110000985F8420008
:10FC00005C48142200EB0611089800E0F0E033F0A5
:10FC10009FF81D2C0BD2204600EB400101EB801019
:10FC2000641CE4B238444322454933F091F8761C11
:10FC3000F6B25148007886428BD30026DFF83CA10B
:10FC4000DFF83CB149E006EB860000EBC60101EBB2
:10FC50000A09D9F80100A880020AEA80020C2A8168
:10FC6000000E688199F80A00A8811AF80100E8815D
:10FC700098F80000A87798F80100E87798F8020053
:10FC800085F8200098F8030085F821001D2C0BD280
:10FC9000204600EB400101EB8010641CE4B23844C4
:10FCA0004322274933F054F8D9F80500A880010A07
:10FCB000E980010C2981000E68811D2C0BD22046A1
:10FCC00000EB400101EB8010641CE4B23844432295
:10FCD0001B4933F03DF8761CF6B29BF800008642D3
:10FCE000B1D398F84E00012803D0264800780128A7
:10FCF0007ED10026DFF890A0DFF890B098E02B20AE
:10FD000006FB00A1887CD0B9D1F80500B8B1A88065
:10FD1000020AEA80020C2A81000E6881887A18B9EA
:10FD20001B4B9A88521C9A8025F80C0F4A7A6A80DD
:10FD300098F80000A87498F80100E8742AE075E0CB
:10FD4000C322016062730460840200605B02006091
:10FD5000E2030060F4000060A2030060B0000060F5
:10FD6000C8000060E02A016008B10360A861046077
:10FD70006C6504603C590460F00200607A6A0460BB
:10FD80001A030060FC0300602CCE03606202006076
:10FD90005082046098F80200287598F8030068758E
:10FDA0000868C0F3072141EA0021E9822A76010CA4
:10FDB000090241EA1060A5F82D00142103A832F0D1
:10FDC000E0FF4D208DF80C0053208DF80D005420DD
:10FDD0008DF80E0050208DF80F003A208DF810009D
:10FDE0004FF000098DF81F90142203A9089800E035
:10FDF000D6E032F0ADFF0C2085F833001BF06BFC31
:10FE000085F835000C3DC8B102281CD085F8429019
:10FE10001D2C0BD2204600EB400101EB8010641C2E
:10FE2000E4B238444322DD4932F092FF761CF6B248
:10FE30009BF800008642FFF462AFF6E0D8480078F5
:10FE400085F84200E4E7D748007885F84200DFE70C
:10FE50007B7898F80F108B427DD1B97898F81030E4
:10FE6000994278D1F97898F81130994273D139795B
:10FE700098F8123099426ED1787C98F80010884238
:10FE80000ED1B97C98F80120914209D1F97C98F8FB
:10FE90000220914204D1397D98F8032091420AD082
:10FEA00000287DD1B87C00287AD1F87C002877D151
:10FEB000387D002874D10120FFF744FD4321B74865
:10FEC000FEF7ACFE88F80E90797988F80F10B879B3
:10FED00088F81000F87988F81100387A88F812004C
:10FEE00098F82A20012A07D0092A05D098F8282056
:10FEF000012A01D0092A01D1AB4A16707A7A88F812
:10FF00001920BA7A88F81A20FA7A88F81B203A7BE6
:10FF100088F81C207A7B88F81D20BA7B88F81E2080
:10FF2000FA7B88F81F203A7C88F82020C1B3B8B348
:10FF30002F2024F0BCFC98F81010302024F0B7FCDF
:10FF400098F81110312024F0B2FC98F812103220E9
:10FF500024F0ADFC00E02CE098F81910332024F0D8
:10FF6000A6FC98F81A10342024F0A1FC98F81B1075
:10FF7000352024F09CFC98F81C10362024F097FCC7
:10FF800098F81D10372024F092FC98F81E103820A5
:10FF900024F08DFC98F81F10392024F088FC00E034
:10FFA00043E098F81C103A2024F081FC7F488670CA
:10FFB0003BE069284BD06C2837D0652853D17C4D65
:10FFC000A88990B3B5F83900010241EA1021688C84
:10FFD000030243EA102761F31F47A98F8DF8111020
:10FFE000080A8DF81200287C8DF80D00A87C8DF889
:10FFF0000E00287D8DF80F00A87D8DF810008DF87B
:020000040801F1
:100000000C20ADF814908DF8169003AA4FF4F071FF
:10001000384627F0AEFDCDE90096029695F82420EB
:10002000002303A938460EF0C7FE002C1BD05F4901
:10003000CC706048006802688A60C088020242EAA8
:10004000102080B2C86009B0BDE8F04FE5E40020A0
:1000500059493A1852780A54401CC0B20A28F8D3B9
:1000600056480670E1E709B0BDE8F08F54480178C2
:10007000080708D553484D4A006810615369C31AF0
:10008000642B00D35061880700D5F8E470472DE950
:10009000F047002446488C21463032F072FE484832
:1000A000007800071DD5474E404D3068A861E969CA
:1000B000401A642815D32879A8B1E978491C8842E8
:1000C0000DD2401E00EB400101EB8010334943315B
:1000D00008444321FEF7A2FD2879401C28713068AE
:1000E000E861BDE8F087DFF8C8C02F200CF1460CAE
:1000F0008CF80000344807788CF801703348017898
:100100008CF8021041788CF8031081788CF8041078
:10011000C0788CF805002E4B4FF00108DFF8B49042
:1001200013E0C4EBC400185C09EBD00100F0070237
:10013000097808FA02F2114201D0012200E00022FF
:100140000CEB44014A758875641CBC42E9DB002154
:100150000020224ADFF880A04FEA470914780EE019
:100160002B2202FB00A2937C3BB909EB41036344C1
:1001700083F81580527A9A75491C401CC0B2A0427F
:10018000EED378188CF8010009488C214630FEF730
:1001900045FD2879401C2871A1E70000C3220160B9
:1001A0006D0300606F030060E0070060F400006012
:1001B000E02A0160D400006010180060F9030060BC
:1001C000AC00006030000060F00200606273046008
:1001D000A86104606C6504602CCE0360620200605C
:1001E00010B50020FD4BFE49052200EB800404EB16
:1001F00040141C44647E1CB10C5C052C00D20A54D3
:10020000401CC0B20A28F0D310BD0021F54A32F8D4
:100210001130834201D101207047491CC9B20A291B
:10022000F5D300207047F0B5FF21FF240020EB4DEF
:10023000EB4E00274FF0B40C00EB800202EB4012B3
:100240002A44527E02F00F02072A24D0052A22D027
:10025000401CC0B20A28EFD3002000EB800202EB62
:1002600040122A44527E02F00F0222B1335CA342B4
:1002700001D81C460146401CC0B20A28EDD30A2909
:1002800013D201EB810000EB41102844477606F8B9
:1002900001C00120F0BD00EB800101EB40112944B9
:1002A0004F7606F800C00120F0BD0020F0BD2DE91A
:1002B000F05F0024DFF830B3CC4FDFF83493BBF8A5
:1002C0002100DFF830A30026CB4D4FF001080028B5
:1002D00007D0010241EA102080B2FFF796FF70B10B
:1002E0002E700020BD4A00EB800101EB401111444B
:1002F000497E01F00F01F9B107291DD01EE02878D1
:10030000401CC0B2287001280AD00228E9D389F81D
:100310000080AAF800802E70F88C401CF884E0E77A
:10032000BBF82100010241EA102080B2FDF7E5FD93
:10033000F88E401CF886D4E7641CE4B2401CC0B2BE
:100340000A28D0D38CB1AE703920FBF77EF8AB49C8
:1003500004282DD3EA7890421DD30A682B699A426B
:1003600019D16A78521C6A7016E0A878401CC0B295
:10037000A8700228E8D3FFF756FF18B1B88E401CCA
:10038000B88606E089F80080AAF80080B88E401C84
:10039000B886AE70D8E76E706A78022A09D389F8F9
:1003A0000080AAF800806E703A8F521C3A8700E0F5
:1003B0006E70E87008682861BDE8F09F38B50024C9
:1003C000FAF7E8FC04E0641CE4B23220FDF784FB99
:1003D000FEF7CEFD08B1642CF5D3834CA07B08B1A9
:1003E000022834D1022801D10120A073B4F82100E1
:1003F000010241EA102080B2FDF77FFD04F01CFCF1
:10040000FFF78CFA607FA17F00EB0120ADF80000C0
:10041000E07F94F8201000EB0120ADF8020002F01C
:100420003FF8684602F02FF894F84800012801D9F7
:1004300000F034FD94F84700022808D170A001F0C4
:10044000CCFF73A001F0C9FF75A001F0C6FF78488A
:1004500069490068C86038BD2DE9F05F664C012627
:10046000207900280CD126714FF4FA7104F12C0088
:10047000FDF74EFB42F2107104F13400FDF748FB2A
:10048000FEF70FFE6B4D2880DFF86481DFF864A172
:10049000694F4FF41679C8B300206081574801684E
:1004A000491C0160654806704FF40060FDF79BFB36
:1004B000634CA189884217D10120FDF753FD28889C
:1004C000002810D0FEF79BFCFEF7F3FD01280AD1AF
:1004D0005C490868401C08603E7098F800000028DD
:1004E00001D1AAF8009067E740F60600FDF77BFB14
:1004F000A1898842F7D1FEF736FC28880028F2D07F
:10050000FEF7D7FD0128EED13E7055E7FFE73A48E8
:100510002C30FDF70FFB0028E5D037482C30FDF7D5
:10052000FEFA0024DFF8B4B004EB840000EB4410C2
:1005300000EB0B01444801600220FDF713FD288801
:1005400058B1FEF75CFCFEF7B4FD012805D13E7002
:1005500098F8000008B9AAF80090641CE4B20A2CCC
:10056000E2D30024DFF8E480DFF8E49004EB4400F9
:10057000C0EB441008EB4000C9F800000520FDF76F
:10058000F1FC288830B1FEF73AFCFEF792FD012815
:1005900000D13E70641CE4B20A2CE7D31648343014
:1005A000FDF7C8FA00289ED013483430FDF7B7FA9B
:1005B000BDE8F05FFEF756BB00240025DFF894A0ED
:1005C00001208AF83C00FFF7F9FEDFF88C90002646
:1005D00089F800601DF015FE40E00000121A01606D
:1005E000101E0160841B016062730460508204600D
:1005F0003C000060A6030060180100604004006039
:100600007777772E333332322E6F72670000000017
:100610007777772E64796E646E732E636F6D00004A
:100620007777772E6E6F2D69702E636F6D000000E7
:10063000B8030060B00000605E0400605F0400600A
:10064000100A016044040060D0000060981B016043
:10065000D40000604C7D0460F6000060DFF8F4B365
:10066000DFF8F483FD4F8BF80060FFF7F5FE387874
:10067000012803D0FA480078012828D101200FF082
:100680000FF80FF068FA48B188F8006088F8016048
:1006900088F802600FF0FCFF0FF05DFA40F30001F4
:1006A000491C88F8001040F34001491C88F80110EB
:1006B00040F38000401C88F802000FF043FD6D1CE1
:1006C000EDB20A2D03D100253E7016F04CF999F8D1
:1006D000000040B1641CE4B2642C04D9002489F801
:1006E000006016F04DF9F8F73EFB0520FDF7F4F930
:1006F000BAF80000401CAAF80000B4E770B586B054
:10070000D84DD94C28686061A169401A642810D37B
:10071000D64E307858B1D648B0F85812FEF77EFA67
:1007200000203070D349087808B1401E087028684E
:10073000A061D148007880071AD5D149CF48086018
:10074000D04CD1492288096832F002FBCF49208879
:10075000088001234FF41672C84901A804F02FFC49
:100760000246002A04D00123C44901A82BF0E9FB6A
:1007700006B070BD38B5BC4C0025A06A002800D07A
:100780008580C3480068C0F3072141EA0022C3B254
:10079000120241EA032142EA1121ADF80010C0F330
:1007A0000741090241EA1060010241EA1020ADF858
:1007B0000200B8480088C0F3072141EA002081B256
:1007C0006846FDF733FBA062002807D0B249B1F8B4
:1007D00049100A0242EA11218180A57138BD70B525
:1007E000A548007800071ED59E4D9F4C2868E06103
:1007F000216A401A322816D3A079617988420DD235
:1008000040F22D114843A54901EB4000B0F85812C1
:10081000FEF704FAA079401CA07102E09D49002077
:1008200008602868206270BD70B59B489C4CB0F889
:100830004900010241EA1020216882B28888824280
:100840000DD160B1CB8893490988C1F3072545EAEA
:10085000012189B28B4202D18349C97971B18242A7
:1008600001D104F013FA20688088A0F58A409C38F2
:100870000AD0A0F50C40683808D102E0BDE870400D
:10088000ADE7FFF7F3FB01E0FFF738FF2068C08812
:10089000B0F5864F10D008DCA0F54050753813D065
:1008A000A0F580608B380FD109E0B0F5A04F0BD0D8
:1008B000B0F5F64F08D105E0FEF7F2FD04E001F0D7
:1008C00078FD01E000F0B4FC76480088010241EABE
:1008D000102081B220688088814205D1002803D091
:1008E000BDE87040FFF7D3BB70BD002809D06E494A
:1008F000401A252190FBF1F00A2802D26B4AB4215C
:10090000115470472DE9F04F89B0044625685A4EBE
:100910003078000715D50021654801EB810210F8F9
:100920002220B2EB156F08D101EB810100EB8100B1
:100930004D49097AFEF772F903E0491CC9B20A2948
:10094000EBD330784FF00007810600D567760106BB
:1009500000D56776C10600D56776400607D5032027
:100960006076E188204615F082F8524908703078A8
:1009700080076DD5DFF80CB14348DFF83CA1BBF828
:100980000020DFF838814FF001090B2A31D00D2A01
:100990002FD00A2A2DD00C2A01D0112A58D1016853
:1009A00004A832F0D5F98AF800909DF811000BF0F8
:1009B00037FA00EBC00101EB410202EB0804B4F886
:1009C0001510090A401C43D09DF81000B0EB156FBC
:1009D0003ED1E1B39DF81C009DF819309DF81B50E5
:1009E00000EB03609DF81A301B0403EB0523184449
:1009F000A1E0016804A832F0ABF99DF811000BF0FA
:100A00000FFA411C24D000EBC00000EB400303EBC5
:100A10000804B4F81510080A9DF81020B2EB156F01
:100A200016D1BBF800200D2A04D101F07F05042D5A
:100A300000D1012068B19DF81C209DF819509DF847
:100A40001B6002EB05629DF81A502D0438E06CE043
:100A500068E039E0F803006030E7036003040060F9
:100A6000EF000060300000601801006010030060BB
:100A7000B22B016011030060AC0000609ECD0160EC
:100A8000FC010060B0000060C8000060E40100608C
:100A90007C02006080020060627304600C2E0160C2
:100AA000D4000060A2030060121A0160101E0160F1
:100AB000A0A3016002030060160300601CB1036084
:100AC00005EB062556190DE00B2A02D00A2A07D09D
:100AD00008E09DF81A209DF8195002EB052601E068
:100AE0009DF819609DF81650227D95421AD1002A72
:100AF00018D09DF8172001F07F018A4212D1CDE96C
:100B00000067029018F80300E178401CC3B26078D7
:100B1000401EC2B2A07808F0E7FF8AF80090A776DE
:100B200084F80B9009B0BDE8F08F9DF81B009DF88C
:100B30001A3000EB0320CDE90171009018F8020093
:100B4000E178401CC3B26078401EC2B2A07808F0C1
:100B5000CBFFE7E738B5C748C74CB0F82100010222
:100B600041EA102081B220688288914204D1FEF7C8
:100B700003FD2068FFF7B9FE2068C04DC088B0F5BE
:100B8000A04F1FD1BE480068010EC0F3074242EAE1
:100B900001210A0242EA1121ADF80010C0F3072139
:100BA000024661F31F22120261F31F2042EA102065
:100BB000ADF8020000F03BFE2878800702D52068DF
:100BC000FFF793FE2068C088B0F5C85F1AD1AD4822
:100BD000D0F80200C0F30741020E41EA02210A02E6
:100BE00042EA1121ADF80010C0F30721024661F37B
:100BF0001F22120261F31F2042EA1020ADF802000A
:100C000001F029FA20684FF20162C188914208D1AF
:100C1000FFF778FE2878800703D52068BDE83840C4
:100C200063E638BD2DE9F0410446974F34F8210FB3
:100C3000388060887880954EA0883080E088708009
:100C4000934DA0892880E089213C688001F028FC30
:100C500004F1290001F017FC864CB4F821000102D0
:100C600041EA102080B2FDF748F994F848000128C5
:100C700001D900F013F994F8470002280BD1AFF224
:100C8000806001F0AAFBAFF2786001F0A6FBAFF242
:100C9000706001F0A2FB774804227B490F3032F0EC
:100CA000B6F8B8B33888FCF79EFF000A10D1388830
:100CB000FCF799FF10F0FF0F0AD17888FCF793FF3B
:100CC000000A05D17888FCF78EFF10F0FF0F21D0C5
:100CD0003888FCF788FF000AE0733888FCF783FF48
:100CE00020747888FCF77FFF000A60747888FCF72E
:100CF0007AFFA074E17B2F2023F0D9FD217C3020E6
:100D000023F0D5FD617C312023F0D1FDA17C322080
:100D100023F0CDFD574804225C49193032F077F8B2
:100D2000B8B33088FCF75FFF000A10D13088FCF7B9
:100D30005AFF10F0FF0F0AD17088FCF754FF000A29
:100D400005D17088FCF74FFF10F0FF0F21D03088DD
:100D5000FCF749FF000A60763088FCF744FFA07674
:100D60007088FCF740FF000AE0767088FCF73BFFD4
:100D70002077617E332023F09AFDA17E342023F07A
:100D800096FDE17E352023F092FD217F362023F071
:100D90008EFD384804223E491D3032F038F8C8B381
:100DA0002888FCF720FF000A10D12888FCF71BFFD9
:100DB00010F0FF0F0AD16888FCF715FF000A05D173
:100DC0006888FCF710FF10F0FF0F23D02888FCF78D
:100DD0000AFF000A60772888FCF705FFA07768887B
:100DE000FCF701FF000AE0776888FCF7FCFE84F856
:100DF0002000617F372023F05AFDA17F382023F0A7
:100E000056FDE17F392023F052FD94F820103A205E
:100E100023F04DFDE07B217C627CA37C657EC5F1E7
:100E2000FF052843A57EC5F1FF052943E57EC5F1F1
:100E3000FF052A43247FC4F1FF04234341EA002431
:100E4000250245EA1424134D2C8043EA022426028D
:100E500046EA14246C80090401EB00600E4903EBA0
:100E600002221044486203F0E7FEBDE8F041FEF7BD
:100E700055BD000062730460D0000060AC000060EB
:100E8000880100608CC10160BA000060BE00006093
:100E9000E0000060C20000601801006010B5F14978
:100EA00001200870F0A001F098FAF4A001F095FA82
:100EB000BDE81040F5A001F090BA2DE9F0470C46CE
:100EC0001646984600256060F4496423B1F9002075
:100ED00092FBF3F149B292FBF3F703FB172252B2F4
:100EE00000290DDA4942CBB25142C9B24FF46162D6
:100EF0005343C1EB011103EB8101401A60600AE02A
:100F0000CBB2D1B24FF461625343C1EB011103EB99
:100F1000810108446060DFF888A39AF8000070B18E
:100F2000E048E149B0F807000988884207D3DF4963
:100F30000988884203D8606800F561606060606875
:100F4000DB4AB0FBF2F102FB1101A160B0FBF2F74A
:100F5000E7604FF46162B1FBF2F0E075B1FBF2F0D3
:100F600002FB1011A4F819103C22B1FBF2F020761C
:100F7000B1FBF2F002FB101984F81B90384632F0F6
:100F800064FACC4ACC4B32F0D2F932F098FA80B203
:100F90002082B8F1000F19D000F2B27189B240F28C
:100FA000B552B7FBF2F28A0714D06FF4B67202FBA7
:100FB0000072A2EB900212B2A4F81520491E890714
:100FC00002D0521CA4F81520BC4A2DE000F26C712E
:100FD00089B2E4E76FF4B67101FB0071A1EB9001F7
:100FE000491C09B2A4F81510B8F1000F02D1491C30
:100FF000A4F81510B14A0C3208E01334638823803A
:10100000535DC91A6180133C6D1CEDB2B4F9151023
:101010000029F2DC0CE0133463882380535DC91A85
:101020006180133C6D1CEDB2B4F915100029F2DC9F
:10103000A574B8F1000F15D000F2B270208286F8C6
:101040000090207E7070E07DB070E07CF070A07C3D
:101050007071207CA0F5FA60B0719AF8000070728F
:10106000BDE8F08700F26C702082E8E72DE9F041DE
:101070008D4D002028808D4C2080924B904A93F813
:101080006310491E05E0165C2F883E442E80401CEC
:10109000C0B28142F7DC002093F86510491E05E0DC
:1010A000165C27883E442680401CC0B28142F7DC93
:1010B00013F8640F29880844288098782188084408
:1010C00020807848807900F5FA60FAF790FB0028D4
:1010D00005D02888401C28802088401C2080BDE83E
:1010E000F081FEB504460F4615461E460DF001FD83
:1010F000E11B01EBC10100EB81006A4C6A4AB4F8C4
:101100000710128891420AD3684A1288914206D881
:10111000A91BC1EB4112C2EB012100EB011001231D
:10112000604A6949FFF7C9FE002220786178CDE95D
:1011300001020091A378E2786179A079FAF7FAFBCD
:10114000FEBD10B56049086046490C398860002A28
:101150000DD1006A10F05CF80023524A5A49FFF79B
:10116000ACFE5A49012008703E490420087010BDA9
:1011700000B58DB03021DB208DF8040000228DF801
:10118000052004208DF80600FA208DF807008DF860
:10119000082001208DF809008DF80A208DF80B2019
:1011A0008DF80C208DF80D000A2001AB02E01A54D6
:1011B000401CC0B28842FAD301A8FDF72FFD0DB044
:1011C00000BD38B5274C0C3C6068002801D00022D7
:1011D0008280080EC1F3074242EA0020020242EA7E
:1011E0001020ADF80000C1F307200A4660F31F226B
:1011F000120260F31F2142EA1120ADF802004FF401
:10120000F6416846FCF712FE60600120207038BD90
:1012100070472F4890F8F010012902D0114800784B
:10122000704790F8EF0008B1002070470420704725
:1012300070B5284C2078000708D50A4D0C3D287859
:1012400020B10020FFF794FF00202870207880074D
:1012500007D521480022018820480068BDE8704079
:101260006FE770BD6401006074696D652E77696E0B
:10127000646F77732E636F6D0000000074696D6595
:101280002E6E6973742E676F760000006E74702E78
:10129000736A74752E6564752E636E009E0300601C
:1012A0006B03006010180060680200606A02006052
:1012B000805101007B14AE47E1D37640965B040871
:1012C0007C5B040862730460ECBB0160F90300609E
:1012D000AED80260AC000060B0000060C8000060E2
:1012E00010B56C4C94F82300411F032901D90C2838
:1012F00017D194F84D00012802D1022002F080FE9F
:1013000094F82800092807D0012805D094F82A006D
:10131000092801D0012804D1BDE81040002002F0C6
:101320006FBE10BD10B501468A1E042A1DD20229C7
:1013300006D0032909D004290CD005290FD011E0CB
:10134000AFF2B80001F07AF80CE0AFF2D00001F093
:1013500075F807E0AFF2F00001F070F802E04E48D7
:1013600001F06CF84D490068086010BD2DE9FE4F92
:10137000484ADFF82C9192F84800022803D299F8E5
:10138000F000012810D1474E3068401C3060464FB5
:10139000DFF818810025397841B14549884203D9E1
:1013A0003D7088F800503560BDE8FE8FFFF731FFD3
:1013B0004FF0010A04280FD098F8000003285ED2ED
:1013C00030681421B0FBF1F301FB13000028EBD1CE
:1013D00099F8F000C0B34CE089F8F1A099F8F0005A
:1013E00078B9344801784278CDE9011500928378C4
:1013F000C27841798079FAF79DFAFAF792FAFFF705
:101400006FFF0DF076FB2C4C2060010EAE2023F018
:101410004EFA2068C0F30741AD2023F048FA208837
:10142000C0F30721AC2023F042FA2178AB2023F04F
:101430003EFA20682DF04EFDC9F8CA0088F8005029
:1014400087F800A03560AFE7FFE792F84800FFF7A4
:1014500069FF1248C178027841EA026142788078D7
:10146000120442EA002001431448B0F90000FFF7DB
:10147000A8FE98F80000401C88F8000094E799F84E
:10148000F00010B9032004F018F988F8005087F82C
:1014900000A089E76273046008BC0160B4030060C7
:1014A000AED802601C040060FE030060FF03006011
:1014B0000046050010180060880200609E0300606E
:1014C0000021EB4801700122427081700171704768
:1014D000E74801218170002101707047E449887854
:1014E000012801D101224A7070472DE9F041002105
:1014F0000020E04A02F5B07605E0535C3354401C0E
:1015000080B2491C89B2302802D2535C002BF4D13E
:101510002F2802D90020BDE8F0813A213154401C27
:1015200080B20021D34A203205E0535C3354401C82
:1015300080B2491C89B2302802D2535C002BF4D10E
:1015400030280AD04FF0000C06F800C0002000221E
:1015500000210023C84DC94F28E00020DBE700022E
:1015600020445B1C9BB2521CD2B2032A1ED1002223
:10157000840C15F804804C1CA4B207F80180C0F359
:10158000053115F80180611C89B207F80480C0F3A9
:10159000851415F804804C1CA4B207F8018000F0F3
:1015A0003F00611C285C89B238550020402B02D2D4
:1015B000F456002CD3D13D23022A02D0012A16D0A2
:1015C00027E00002820CAC5C4A1C92B27C54C0F34F
:1015D00005316C5C511C89B2BC54C0F385102A5C87
:1015E000481C80B27A54411C89B23B5411E0020479
:1015F000900C2C5C481C80B27C54C2F305316A5CB0
:10160000411C89B23A54481C80B27B54411C89B2B7
:101610003B5407F801C001207DE7F0B587B0984939
:101620000888ADF818004988ADF81A10904CC7B278
:101630000A342770020A6270CBB2A370090AE17003
:101640008B4D8C4EE8786036002804D0012821D0DC
:1016500002283DD053E0FFF748FFC0B1E178A278FF
:101660006078CDE90121834A009040322378854992
:1016700002F1200032F088FE80B2E88030447F4AD8
:10168000814932F081FEE9880844E88037E0002093
:1016900007B0F0BDFFF729FFC0B1E178A27860780C
:1016A000CDE90121734A009040322378774902F155
:1016B000200032F069FE80B2E88030446F4A7449FD
:1016C00032F062FEE9880844E88018E00020DFE795
:1016D000CDE90172CDE903316648664A4030009099
:1016E000A0F120036B49203032F04EFE80B2E8803A
:1016F0003044694932F048FEE9880844E880E078DF
:10170000A178CDE900105D486378227863A140306C
:1017100032F03AFE28810120BAE738B5544C624DC8
:101720002078296801280ED04FF4FA72022826D0BA
:1017300003282BD0042821D16069081A90421DD9B2
:10174000BDE83840C4E659480068020EC0F30743BC
:1017500043EA0222130243EA1222ADF80020C0F34A
:101760000722034662F31F231B0262F31F2043EA92
:101770001020ADF8020002202070616138BD606960
:10178000081A9042FAD9BDE83840A1E6FFF745FFB4
:10179000012128B10420207028686061217138BDC2
:1017A000A17038BDF0B4049F314E7478012C39D14A
:1017B0000024DFF8C0C00CF1400C155D2DB10CF811
:1017C0000450641CA4B2202CF7D30125202C23D074
:1017D0000022DFF8A0C09C5C2CB10CF80240521C27
:1017E00092B2202AF7D3202A18D00022214C20348C
:1017F000BB5C23B1A354521C92B2202AF8D3202AF6
:101800000ED03161F070357000217170B170032815
:1018100008D9B570F0BC7047B570FBE7B570F9E753
:10182000B570F7E7F0BC78E711480078704770B5FD
:101830001F4D0F4C287800070BD52078042808D1BD
:10184000207930B1002020710A48E1886030FDF72E
:10185000E5F92878410601D503212170800704D5D8
:101860002078042801D10520207070BD7047704792
:101870006C01006026BC0160AE5B0408B6BD01606F
:10188000BA000060286C0408FC6A0408B46B040801
:10189000586B04089C6C0408B86A040825752E254A
:1018A000752E25752E2575003000006088010060BA
:1018B000AC00006010B52021394831F062FA384898
:1018C0002021203031F05DFA35482021403031F0C0
:1018D00058FABDE81040FFF7F3BD08B501460020F7
:1018E000002906D0012908D002290AD003290CD0EA
:1018F0000EE02CA000F0A2FD0AE02EA000F09EFD5C
:1019000006E030A000F09AFD02E032A000F096FD63
:10191000002811D0006800909DF803009DF8001089
:101920009DF8022000EB01609DF80110090401EB15
:10193000022108442B49486008BD10B5FFF7C0FDDF
:10194000284C2078FFF7C9FF0120607010BD38B522
:10195000244C2078032821D0617801291ED120B1A0
:10196000012805D0022806D007E01F49616004E085
:101970001E49616001E01E4961600949084B403120
:1019800000911C492033064A085C6168FFF70AFF92
:10199000FFF7A4FD012801D10020607038BD704719
:1019A00006BE01607777772E333332322E6F72673F
:1019B000000000007777772E64796E646E732E6373
:1019C0006F6D00007777772E6E6F2D69702E636FC5
:1019D0006D0000006E65776669726D776172652EC5
:1019E000636F6D00840100600FB0B87675F80DCCA0
:1019F0006EE01708EF5B04082249002008702249B6
:101A00000860704778B50078C1B21E4890F90000B0
:101A1000C0F10202D20091401B4E34680C43346086
:101A200002282DD10020194A6D4600EB40014900E3
:101A300024FA01F3C3F3050111542954192902DCD6
:101A40004131115417E0A1F11A03192B02D8473183
:101A5000115410E0A1F13403092B02D8091F1154CD
:101A600009E03E2902D03F2903D004E02B21115484
:101A700001E02F211154401C0428D6D300203060EF
:101A800078BD000094010060900100609C0100603E
:101A9000FE4800210170C0F8021070472DE9F047A0
:101AA0000546FB4CFFF7A8FF642104F5FD7031F0FB
:101AB00068F9284631F08CF90246294604F5FD7094
:101AC00031F046F9002504F5FD7031F081F9C7B217
:101AD0000326B7FBF6F006FB107048B104F5FD7065
:101AE00031F076F9C01CB0FBF6F000EB4000C7B255
:101AF00000264FF00D084FF00A09DFF898A326E002
:101B0000E24864383044FFF77DFF9AF80000401C3B
:101B100040B28AF80000032817D1642D04D104F8DC
:101B2000018B04F8019B00250020DA490831C0F13F
:101B300003028A5C04F8012B401CC0B20428F6D3CF
:101B40002D1DEDB200208AF80000761CF6B2BE42D0
:101B5000D6D3CF48284410F8011C412907D110F8EA
:101B6000021C412903D13D21801E4170017084F87F
:101B7000008084F80190AD1CE8B2BDE8F0872DE943
:101B8000F05F03461A789C78303A02EBC20505EB09
:101B9000021204EB82045A786FF02F03303A02EB02
:101BA000820203EB4202224492B2002954D0B74988
:101BB0004C230D2409780A26B54D4FF0480C4FF000
:101BC0004F0A4FF0200B4FF05409022921D0AF4F9C
:101BD0004FF0410E032941D0DFF8BCC24FF4A77883
:101BE0000E2959D00F2969D00D297ED00B1F032B48
:101BF00076D23B4603F16A0C03F19C0293F86A80AB
:101C000093F89C3004296CD005296BD006296AD042
:101C1000C2E0DC2A68D14520287085F801C003277E
:101C2000AB7085F803A0052185F804B09B4A681DB8
:101C300004E000F8013B521C491C89B21378002BC8
:101C4000F7D1481C80B26C54411C89B22E54904884
:101C5000FCF7E4FF8D480770BDE8F09FFA2AD9D160
:101C600085F800E05520687085F8029085F803C07B
:101C700085F804B06B7185F806A04720E87149200B
:101C800028724E206872AC720C21EE728048FCF70C
:101C9000C5FF0E203870DFE74245DDD1BCF81600E5
:101CA000401CACF816007D486630FFF7F7FE014691
:101CB0007748FCF7B3FF0F203870CDE74245CBD112
:101CC000BCF81800401CACF818007448A230FFF7AC
:101CD000E5FE01466E48FCF7A1FF3C70BCE704E05E
:101CE00083E031E046E052E085E0FA2AB4D04D20AE
:101CF000287085F801E04921A970EB7085F804B0DF
:101D0000462169715221A97185F807A028723A20ED
:101D100068723C20A8720B22B91D5D480B3004E0AC
:101D200000F8013B491C521C92B20B78002BF7D1F2
:101D30003E21017044708670D21C91B25448FCF769
:101D40006DFF0420387087E797F83800202804D00A
:101D50004E483830052139701EE0B8F1200F03D00D
:101D600060460621397017E0202B44D01046072129
:101D7000397011E0B8F1200F03D0604606213970A8
:101D80000AE0202B4DD010460721397004E0202BAB
:101D900047D01046072139705221297043216970BC
:101DA0005021A97085F8039085F804B085F8059056
:101DB00085F806A03A21E9713C21297209223449AB
:101DC000093104E001F8013B401C521C92B2037837
:101DD000002BF7D13E2008704C708E70D21C91B24F
:101DE000BDE8F05F2A48FCF719BF072919D0082978
:101DF00028D00B29A7D12948244F401F80F834113F
:101E000051202870552068704920A87085F80390EB
:101E10002C716E7106211E48FCF700FF0C203870F3
:101E20001AE74420287085F801E085F8029085F8CB
:101E300003E02C716E7106211548FCF7EFFE0820B7
:101E4000387009E7B2F5B17FD5D10920387003E7C2
:101E50002DE9F35F00200E4C462121707221617044
:101E60006F22A2706D21E1704FF03A0B84F804B03C
:101E70004FF0200884F805804FF0220C84F806C04B
:101E80000721024EB31DE41D0FE000008CC101606C
:101E90002EBF01609401006050820460510803600D
:101EA00004F8015B5B1C491C89B21D78002DF7D139
:101EB00004F801CB04F8018B4FF03C0904F8019BB6
:101EC000C91C89B2B31D04E004F8015B5B1C491C0A
:101ED00089B21D78002DF7D14FF03E0A84F800A09A
:101EE0000D2767704FF00A0E84F802E05423E37068
:101EF0002271641D04F801BB04F8018BC91D8BB26B
:101F0000002252B1012A10D096F89C1020293ED010
:101F1000AC490D46012810D014E096F8381020295D
:101F200035D0A84964390D46F4E796F86A1020299F
:101F30002DD0A44932390D46ECE72C2004F8010BD2
:101F40005B1C9BB284F800C0601C5B1C9BB204E06D
:101F500000F8014B491C5B1C9BB20C78002CF7D19C
:101F600000F801CB00F8018B00F8019BDB1C99B253
:101F700004E000F8013B6D1C491C89B22B78002B52
:101F8000F7D100F801AB0446491C8BB20120521C6A
:101F9000D2B2032AB5D32770754684F801E09B1CA2
:101FA0005320A0707520E070622020716A2060715B
:101FB0006520A0716320E07174202072093404F858
:101FC00001BB04F8018B09331FFA83F914227EA1A7
:101FD000804830F0BDFE7F484FF0090808E05A29DC
:101FE00019D004F8011B401C09F101091FFA89F9F5
:101FF00001780029F3D127706570A41C09F102094A
:102000001FFA89F9734864223230009930F0A0FE3B
:10201000704832300CE004F8018B401CE4E75A2988
:1020200015D004F8011B401C09F101091FFA89F9B8
:1020300001780029F3D12770657009F102091FFAB0
:1020400089F16548FCF7EAFD3570BDE8FC9F04F8AE
:10205000018B401CE8E770B5604D5E4C287804F1B8
:102060009604000707D52078092804D1C821A4F2D6
:102070002630FFF7EDFE2878800711D55548C82196
:10208000C83830F07EFE5748554E016851483288B6
:10209000C83830F05DFE4F483188C838FFF76FFD13
:1020A0002878C00710D020780A280DD14A480D2280
:1020B00002700A2141702E238370C27001710521C4
:1020C000FCF7ACFD0B2020702878400601D50220DB
:1020D000207070BD1CB5444C6068002802D0407E62
:1020E000002819D1C0208DF80000A8208DF801002B
:1020F00000208DF8020040208DF803004AF6C00051
:10210000ADF804004FF48040ADF8060045F6043108
:1021100001A8FBF720FE60601CBD38B5334C601D84
:1021200030F056FE20284BD2601D00F056F9601D9D
:1021300030F04EFE02462EA1601D30F068FE0025F4
:1021400030B1601D00F07AF90068C4F8010006E0C3
:10215000C0206070A820A070E57007202071224880
:10216000417801292CD145702049164832222F315F
:10217000963830F0EDFD1D4912483222BC316438EA
:1021800030F0E6FD19490F483222F831323830F08C
:10219000DFFDA078617840EA0120010241EA1020C9
:1021A000ADF800002079E17840EA0120010241EA1F
:1021B0001020ADF802004FF4C8516846FBF7CBFD84
:1021C00038BD000028C20160414C41524D20212100
:1021D000210D0A00F6C001602EBF0160AC00006056
:1021E000B0000060C8000060940100604C0803600B
:1021F0006C6F63616C686F737400000010F8011BF2
:1022000002E0401C491EC9B20029FAD10178002918
:10221000F4D1401C704770472DE9F047A94D0026C6
:102220002E70A94A4FF00108287800EBC00101EB9D
:10223000401084182078012801D0022837D10228C4
:1022400020D00220207084F80180A6709F4FD7F81C
:102250000090C9F80060C9F80460C9F808602878DF
:10226000FBF7C1FCA9F8000089F802804FF48070E8
:10227000A9F8040039680C31241D641C0A46491C65
:102280006E7022E06078401E10F0FF0060700ED18A
:10229000A078401CC0B2A0700A2802D0A07860705C
:1022A000D4E7042020700021601DFFF7B4FF2878D8
:1022B000401CC0B228700528B6D3BDE8F08701F8ED
:1022C000010B6878401C6870641C20782E2801D0AF
:1022D0000028F4D16878107020780028CDD12869C2
:1022E0000860287D08713868BDE8F047091A491D63
:1022F000C9B2FCF793BC2DE9F041744F3C682088CB
:10230000FBF771FC6F4EC0B2307100EBC0016E4A3A
:1023100001EB40118D1805283DD2287802283AD1CA
:1023200003202870E07800F00F00287130B10420FD
:1023300028700021681DBDE8F0416CE7A088FBF71C
:1023400052FCB070E088FBF74EFCF07038680C303F
:10235000FFF754FF001D4FF4807719E001788909D9
:1023600001D0841C02E0FFF749FF04462088B842F0
:1023700006D16088B84203D12089B0F5806F0CD0B7
:102380002089FBF730FC20440A30F178491EF170B7
:10239000F1780029E2D1BDE8F0816089A5F8250037
:1023A000A089A5F8270005F12501681DBDE8F041C9
:1023B00031E710B546480068C088B0F5545F0BD1CE
:1023C000444C2078000701D5FFF726FF20788007CE
:1023D00002D5BDE810408EE710BD70B50146394DFD
:1023E0000020E871A8716871374B687900EBC00272
:1023F00002EB4012D418227862B1E278AE7AB21AB7
:10240000AE79B24201DDAA71E871401CC0B26871B8
:102410000528EAD36879052806D1E879687100EBC8
:10242000C00202EB4010C418601D30F0FDFC01201A
:102430002070A87AE070401CA87270BD2DE9F041B0
:102440000746204D002028721F4E287A00EBC0015D
:1024500001EB401084192078032804D1611D38460F
:1024600030F0BDFC38B1287A401CC0B22872052873
:10247000EBD300208FE704F125008CE71148C068FA
:102480000028FFD1704710B50E4CE168002901D03B
:1024900000228A804FF45451FBF7C8FCE06010BD65
:1024A00010B5084900234B72074A487A00EBC00474
:1024B00004EB40141355401CC0B248720528F4D3F5
:1024C00010BD0000A00100605AC20160C800006099
:1024D000D4000060AC00006010B5044619F0FBF8B1
:1024E000F14902280ED091F82300032820D00428B7
:1024F0001ED007281CD00C281AD0082818D0EB486A
:10250000046010BD91F82300E94903280AD004288B
:1025100008D0072806D00C2804D00A2805D0C1F816
:10252000AC4110BDC1F8AC4110BDE248046010BD23
:10253000E148046010BD38B502460846062A15D0A9
:10254000052A1DD0DD4C42B3092A36D0DC4C012AC5
:1025500043D0032A52D0DB4C022A60D0042A71D027
:102560000A2A7FD00B2A6CD0002038BD042801D362
:10257000002038BDD44900EB40100844153038BD68
:10258000082801D3002038BDC0EBC000CF4900EBC4
:10259000400001EB4000153038BD694610F00AF9E3
:1025A0009DF80000802801D3002038BDC0EBC00199
:1025B00001EB40102044153038BD694610F008F991
:1025C0009DF80000802801D3002038BDC0EBC00179
:1025D00001EB40102044153038BD694610F006F973
:1025E0009DF80000402801D3002038BDC0EBC00199
:1025F00001EB001004EB4000153038BD694610F0C7
:1026000003F99DF80000402801D3002038BDC0EB3D
:10261000C00101EB001004EB4000153038BD6946E5
:1026200010F000F99DF80000402801D3002038BDCB
:10263000C0EB001000EB40002044153038BD01E035
:1026400010E024E0694610F0FBF89DF800004028F7
:1026500001D30020F2E7C0EB001000EB4000204463
:102660001530EBE748B1012809D0022809D003282A
:1026700009D0042809D096A0E0E798A0DEE79BA047
:10268000DCE79FA0DAE7A2A0D8E7A5A0D6E708B1CB
:102690008FA0D3E7A5A0D1E738B502460846052AA2
:1026A00015D0062A1FD0854C32B3092A33D0844C6A
:1026B000012A3FD0032A4DD0824C022A5AD0042A44
:1026C00067D00B2A76D00A2A79D00020B6E70828EE
:1026D00001D30020B2E7C0EBC0007C4900EB400012
:1026E00001EB4000AAE7042801D30020A6E77649C1
:1026F00000EB40100844A1E7694610F05BF89DF834
:102700000000802801D3002098E7C0EBC00101EB56
:102710004010204492E7694610F05AF89DF80000F6
:10272000802801D3002089E7C0EBC00101EB4010F5
:10273000204483E7694610F059F89DF800004028CE
:1027400001D300207AE7C0EBC00101EB001004EBDD
:10275000400073E7694610F057F89DF800004028E4
:1027600001D300206AE7C0EBC00101EB001004EBCD
:10277000400063E7694610F055F89DF800004028D6
:1027800001D300205AE7C0EB001000EB40002044CA
:1027900054E7694610F054F89DF80000402801D332
:1027A00000204BE7C0EB001000EB4000204445E761
:1027B00000E004E008B146A040E75FA03EE748B172
:1027C000012809D0022809D0032809D0042809D0FB
:1027D0003FA033E741A031E744A02FE748A02DE711
:1027E0004BA02BE74EA029E708B50A46002809D0E0
:1027F000012855D0022854D0042853D0032852D0A1
:10280000002008BD694610460FF0D4FF9DF8000077
:10281000802801D3002008BDC0EBC00101EB4011AE
:102820002648014491F8260040B391F8231039B3AB
:10283000012827D0022827D00B2827D00C2827D002
:102840000D2827D00E2827D0102827D011287BD07C
:1028500012287AD0132879D0042878D0052877D088
:10286000082876D0092875D0072874D0172873D087
:10287000182872D0162871D05F2008BD5F2008BDCF
:102880005F2008BD3E2008BD402008BD052008BDD2
:10289000062008BD032008BD022008BD492008BD50
:1028A00073E0BAE0DCE0E1E0627304608801224298
:1028B0000000234280012142A0812242F2E802600E
:1028C00008350560C84005606C5603605C4E0360C7
:1028D00072657365727665640000000070616E65F4
:1028E0006C206E756D626572000000007278206F5A
:1028F00066206D61696E2072733438350000000007
:102900007278206F662073756220727334383500D8
:102910007278206F662065746865726E6574000059
:102920007278206F662077696669000046414E2004
:102930004D4F44450000000046414E204D4F444558
:10294000205459504500000009E00AE00BE00CE07B
:102950000DE00EE00FE010E011E012E013E048207F
:1029600008BD472008BD462008BD352008BD3620DB
:1029700008BD2F2008BD302008BD242008BD1D2023
:1029800008BD602008BD622008BD694610460FF0F2
:102990002DFF9DF80000402801D3002008BDC0EBAA
:1029A000C00101EB0011FE4800EB410090F8281037
:1029B00009B390F82D0003281FD007281DD009283F
:1029C0001BD004281BD0082819D00A2817D00D289E
:1029D00017D0132817D00B2815D0102815D0112880
:1029E00013D0122811D01A2811D01B2811D01C285E
:1029F00011D05F2008BD5F2008BD3E2008BD4020EB
:102A000008BD022008BD052008BD622008BD1B20AE
:102A100008BD1D2008BD602008BD694610460FF0A6
:102A200001FF9DF80000C0EB001000EB4001DD4805
:102A3000084490F9280058B101280BD002280BD087
:102A4000052809D0042807D0062807D05F2008BD34
:102A50005F2008BD052008BD622008BD022008BD1A
:102A6000402A01D3002008BD5F2008BD402A01D3C1
:102A7000002008BD5F2008BD38B502460846C94C95
:102A8000022A10D0042A1BD0052A26D0062A32D0CA
:102A9000C54C7AB3092A49D0C14C012A57D0032A20
:102AA00070D00020CAE569460FF0BCFE9DF800001A
:102AB000C0EB001000EB4000204490F82600BDE57C
:102AC00069460FF0BDFE9DF80000C0EB001000EB62
:102AD0004000204490F82600B0E5082801D30020EB
:102AE000ACE5C0EBC000B14900EB400001EB400099
:102AF000C07FA3E509E0042801D300209EE5AC498E
:102B000000EB40100844C07F98E569460FF052FE84
:102B10009DF80000802801D300208FE5C0EBC001A4
:102B200001EB4010204490F8220087E569460FF041
:102B30004FFE9DF80000802801D300207EE5C0EB09
:102B4000C00101EB4010204490F8220076E5694670
:102B50000FF04CFE9DF80000802801D301206DE5A8
:102B6000C0EBC00101EB001004EB400090F827100F
:102B7000012904D090F8230000F00F005EE5012049
:102B80005CE5FFE769460FF03FFE9DF800008028F6
:102B900001D3002052E5C0EBC00101EB001004EBB3
:102BA000400090F82710012904D090F8230000F08D
:102BB0000F0043E5012041E52DE9F84F0C4615468D
:102BC0007C4FDFF8E4B1DFF8D8A1DFF8EC91DFF853
:102BD000EC81744E0B287DD2DFE800F0066474555A
:102BE000FAF9F87C7C23E100694628460FF0E2FD03
:102BF0009DF80000C0EBC00101EB4010584490F874
:102C00002310012902D00020BDE8F88FD0F81E0063
:102C10002CF060F930F0FAFBBDE8F84F684930F06D
:102C2000CABA694628460FF0D3FD9DF80000C0EBF4
:102C3000C00101EB4010584490F8231009B1002066
:102C4000E2E790F82610A1F10C020A2A0FD91739F1
:102C5000072906D801EBC10202EB0111795C0129B9
:102C600005D090F8240001280AD00020CCE790F885
:102C70002400012802D04FF07E50C5E70020C3E7B2
:102C80004FF07E50C0E7694628460FF0BDFD9DF825
:102C90000000C0EBC00101EB00100AEB400090F80F
:102CA000281011B3694628460FF0A0FD9DF80000DA
:102CB000C0EBC00101EB00100AEB400090F82810B7
:102CC000012934D0694628460FF0ACFD3D48017813
:102CD0003D4800E037E1007808449DF80010884244
:102CE00040D80F2C2ED048468EE790F82D10A1F139
:102CF0000C020A2A0FD91739072906D801EBC1029D
:102D000002EB0111795C012905D090F82600012819
:102D10000AD0002078E790F82600012802D04FF072
:102D20007E5071E700206FE74FF07E506CE7D0F8DF
:102D30001E002CF0CFF830F069FBBDE8F84F2049B9
:102D400030F039BAC1EB011000EB40003044D0F84C
:102D50001E002CF0BFF830F059FBBDE8F84F1849C1
:102D600030F029BA08EB811050F8242048468242FE
:102D700085D0C1EB011000EB4000304490F82310E7
:102D800039B30CF039FC9DF80050A84227D808EB65
:102D900085100B4950F8240030F0DBF91AE0BAE056
:102DA00008350560C8400560F2E802605C4E0360CB
:102DB0006C5603605AE4026000007F43587F036052
:102DC00000007A44A7020060A802006096E085E057
:102DD0002EE009E030F05FFBF74921F8150008EB21
:102DE000851050F824000FE712F0FF4F01D00121A9
:102DF00000E0002190F92800A0F10C020A2A0DD968
:102E00001738072806D800EBC00202EB0010385C28
:102E1000012803D0012908D00020F5E6012902D0BD
:102E20004FF07E50F0E60020EEE64FF07E50EBE6ED
:102E3000694628460FF004FDE0480178E048007834
:102E400001449DF80000814212D80F2C01D0484661
:102E5000DAE6C0EB001000EB40003044D0F81E0072
:102E600008B1012000E00020BDE8F84F30F0D7BAEB
:102E700008EB801151F82410494501D14846C3E6BA
:102E8000C0EB001000EB4000304490F823200AB162
:102E90000846B9E611F0FF4F01D0012100E0002102
:102EA00090F92800A0F10C020A2A0DD9173807283A
:102EB00006D800EBC00202EB0010385C012803D0FA
:102EC000012908D000209FE6012902D04FF07E5052
:102ED0009AE6002098E64FF07E5095E6C5EBC500D7
:102EE000B84900EB400001EB4000807F08B10120B1
:102EF00000E00020BDE8F84F30F091BAB24905EB90
:102F000045100844807F08B1012000E00020BDE8A2
:102F1000F84F30F084BAAD48052D0FD2DFE805F048
:102F20000306080A0C00AA48007808E0006806E0DA
:102F3000406804E0806802E0C06800E00020BDE86E
:102F4000F84F30F06CBA00205EE6A2487047A24B02
:102F500000EBC00003EBC00000EBC100805C7047D9
:102F600030B5ADF5197D01EBC1049C4901EB0411AD
:102F700001EB021101EB43056D788DF8005011F85B
:102F800013108DF8011000218DF802108DF8031038
:102F9000914901EBC40101EBC201C95CCDF80710F6
:102FA00009218DF8061040F2622269462FF0D0FE0A
:102FB0000DF5197D30BD10B5034600200022864C6A
:102FC00003EBC30304EBC30303EBC1018B5CFF2BD7
:102FD00001D0401CC0B2521CD2B2082AF6D310BD98
:102FE0002DE9F0437E4B01241C707E4B1C741C7633
:102FF0000023DFF8E4C100EBC006784F0CEBC600FD
:1030000000EBC10007EB0616FF2506EB01114AB9DC
:1030100001EB4306767816B911F8136036B124EA4D
:103020000306C654C65CFF2E02D00BE0C554F9E778
:1030300001EB4306767816B911F81360BEB124EAA5
:103040000306C6545B1CDBB2082BE0D30023C25C32
:10305000FF2A46D001EB430811F8134098F80120ED
:10306000C2EB021204EB82045A1CD2B237E00BB15D
:10307000C554E7E7CE780EB98E780EB10470E1E75B
:103080000570DFE710F802C0BCF1FF0F25D001EB9F
:10309000420711F812607D78C5EB051506EB850631
:1030A000B4421AD9254634463C26B4FBF6F988F8D2
:1030B0000190B4FBF6F906FB194901F81390B5FB32
:1030C000F6F987F80190B5FBF6F706FB175501F8FE
:1030D0001250C55C00F803C08554521CD2B2082AB5
:1030E000D0D35B1CDBB2082BB1D3BDE8F08330B585
:1030F00000250024012221462846FFF771FF641CA9
:10310000E4B2092CF6D36D1CEDB2082DF1D330BD1D
:1031100000207047F0B500220021C0EBC00303EB94
:103120000010314B012703EB40060020755C07FAC5
:1031300000F4254201D0521C92B2401C80B20828F3
:10314000F5D3491C89B22E29EFD3D0B2F0BDC0EB24
:10315000C00101EB0010244901EB40002E212FF0AB
:1031600010BE70B5421C93B2204E214DB279920729
:1031700008D01C226A700022AC5C9C4205D21B1B4A
:103180009BB206E01D226A70F5E7521C8A70CB7074
:103190000C22521C92B20C2AEED3B6F80720072359
:1031A000824227D9101A90FBF3F203FB1200327906
:1031B000101AC01D80B225E0AED10260A7020060E7
:1031C000A80200605C4E03606C56036020800460BF
:1031D0005B02006008B103602C540360AC4F0360D5
:1031E000EE03006030E70360F056036010180060E3
:1031F00022D40260801A90FBF3F203FB12003279B2
:10320000104480B2B0FBF3F203FB1200401C0871C3
:10321000B07900F5FA60088070BD2DE9FC47824660
:10322000914600260025C1EBC10000EB0110FE49CC
:103230004FF0010801EB40070024785D08FA04F123
:1032400008420AD0B14506D104EBC500401E80B249
:103250006946FFF786FF761CB6B2641CA4B2082C40
:10326000EBD36D1CADB22E2DE6D30098CAF800004A
:103270009DF804008AF80400BDE8FC872DE9F843B6
:103280001C46EA4901250D70E94F002601281ED091
:10329000DFF8A08302287DD0042816D169461046A5
:1032A0000FF0CEFA9DF8001040290ED23D70C1EB10
:1032B000011000EB4000404480F823605F2C70D088
:1032C00080F8285001220FF0C9FABDE8F88369465A
:1032D00010460FF08BFA9DF800004028F5D2D64931
:1032E0005F2C07D1C0EBC00202EB001201EB4202DF
:1032F00082F82D603E2C08D1C0EBC00303EB001315
:1033000001EB4303032283F82D20402C08D1C0EBAE
:10331000C00303EB001301EB4303042283F82D20C9
:10332000032C0ED1C0EBC00202EB00120D2301EB07
:10333000420223329372137803F00F0343F0100319
:103340001370052C10D1C0EBC00202EB001201EB90
:10335000420202F123024FF013039372137803F039
:103360000F0343F0300313700ED0032C0CD0C0EBCE
:10337000C00202EB001201EB420212F8233F03F0FD
:103380000F0343F0400313707D70C0EBC00202EBEB
:10339000001001E008E004E001EB40000FF009FB41
:1033A00093E780F828608DE7694610460FF03AFAF7
:1033B0009DF80010402988D23D70C1EB011000EB50
:1033C0004000404480F823505F2C05D080F82850FE
:1033D00001220FF043FA78E780F82860F8E72DE93A
:1033E000F843014610461C46904A01251570904E40
:1033F000914FDFF84092DFF844820A291CD2DFE8BF
:1034000001F061054A1C3387971B1B7469460FF056
:10341000EDF99DF8000040280ED27570C0EBC00198
:1034200001EB001007EB40002168C0F8151061683F
:10343000C0F819100FF0BDFA47E769460FF0E4F93C
:103440009DF800004028F7D27570C0EBC00101EB79
:10345000001007EB40002168C0F815106168C0F843
:1034600019100FF0A6FA30E769460FF0E9F99DF858
:1034700000104029E0D23570C1EB011000EB400094
:1034800048442268C0F815206268C0F8192001225B
:103490000FF0E4F919E769460FF0C4F99DF8001040
:1034A0004029C9D23570C1EB011000EB40004844FF
:1034B0002268C0F815206268C0F8192001220FF0B8
:1034C000CDF902E769460FF075F99DF800008028F4
:1034D000B2D2B570C0EBC00101EB4010404421688E
:1034E00040F8151F61684160EFE669460FF070F91A
:1034F0009DF8000080289FD2B570C0EBC00101EBA1
:1035000040104044216840F8151F61684160DCE6C6
:10351000082891D23571C0EBC000494900EB40004A
:1035200001EB4000216840F8151F61684160CCE65E
:10353000042898D27571434900EB40100844216873
:1035400040F8151F61684160BFE62DE9F84F0E464F
:1035500015461C46354901270F70DFF8D490DFF877
:10356000E8A0DFF8E8B0DFF8E8800A2841D2DFE819
:1035700000F005A6FED8FDFCFB4040413549C88B54
:10358000401CC883694628460FF014F99DF80000D6
:1035900080282ED2C0EBC001284D01EB40102844FA
:1035A00090F82300012811D12B4920462FF0D1FD9E
:1035B0002FF058FF2BF08EFC01469DF80000C0EB69
:1035C000C00202EB40102844C0F81E1089F80270B7
:1035D000214920462FF0BDFD2FF044FF2BF07AFC4F
:1035E0009DF80010C1EBC10202EB41112944C1F862
:1035F0001E0012E4694628460FF0EAF89DF8000024
:103600008028F6D2C0EBC0010C4D01EB40102844DD
:1036100090F82300F0BB104920462FF09AFD2FF0C0
:1036200021FF2BF057FC19E0F0560360EE03006019
:1036300030E70360C840056008350560F2E80260C5
:103640005C4E03606C560360A7020060A802006035
:10365000587F03605082046000007A4402469DF85F
:103660000000C0EBC00101EB40104119C1F81E2061
:1036700091F82600A0F10C020A2A11D91738072860
:1036800007D800EBC00202EB0012FE48805C012864
:1036900006D000E010E014F0FF4F0AD0012009E04E
:1036A00014F0FF4F03D0002081F8240004E0012033
:1036B000FAE7002081F8240089F8027003E46946E3
:1036C00028460FF093F89DF800004028F6D289F8BC
:1036D0000170C0EBC001EC4D01EB001005EB4000A8
:1036E00090F82800012811D1E84920462FF031FD3B
:1036F0002FF0B8FE2BF0EEFB9DF80010C1EBC102DD
:1037000002EB011105EB4101C1F81E009DF800001C
:10371000C0EBC00101EB001005EB40000FF049F9D0
:1037200012E4694628460FF06FF89DF80000402823
:10373000F6D289F80170C0EBC001D34D01EB001047
:1037400005EB400090F8280008B3D04920462FF040
:1037500000FD2FF087FE2BF0BDFB9DF80010C1EBA4
:10376000C10202EB011103E0AFE19AE145E016E18D
:1037700005EB4101C1F81E009DF80000C0EBC0013F
:1037800001EB001005EB40000FF013F931E7BF49E2
:1037900020462FF0DEFC2FF065FE2BF09BFB02464F
:1037A0009DF80000C0EBC00101EB001005EB4001EB
:1037B000C1F81E2091F82D00A0F10C020A2A0FD9A1
:1037C0001738072807D800EBC00202EB0012AD48FB
:1037D000805C012804D014F0FF4F0AD0012009E0DA
:1037E00014F0FF4F03D0002081F82600C4E7012029
:1037F000FAE7002081F82600BEE7694628460FF068
:103800001FF89DF80050402DC0D2012089F800001B
:103810009F4FBC4204D108EB851040F8267095E01C
:10382000C5EB0510DFF86C9200EB400000EB0901DE
:1038300091F92800A0F10C020A2A16D91738072896
:1038400007D800EBC00202EB00128E48805C012812
:103850000BD09AF800009BF800201044A8425CD9D5
:1038600014F0FF4F41D0012040E09AF800009BF88F
:1038700000201044A8421CD914F0FF4F15D000209E
:103880002FF0CDFD08EB851141F82600284625F0E4
:1038900052F960B100209DF80010C1EB011101EB5D
:1038A0004101494481F8250050E00120E8E701206A
:1038B000F1E704F0FF40002807D04FF0000081F846
:1038C000250005D14FF0010004E04FF00100F6E7BC
:1038D0004FF000002FF0A3FD014608EB8510C163F7
:1038E0000F2E33D040F8267030E000202FF097FDE7
:1038F00008EB851141F82600284625F01CF908B18F
:10390000012000E000209DF80010C1EB011101EB47
:103910004101494481F8250018E014F0FF4F01D01F
:10392000012000E0002081F825000F2E03D008EBD5
:10393000851040F8267014F0FF4F01D0012000E000
:1039400000202FF06CFD08EB8511C8639DF8000086
:10395000504CC0EB001101EB41012144002281F8E1
:10396000232002F0B1FE02F04AFA9AF800009BF818
:10397000001008449DF80010884207D8C1EB0110E0
:1039800000EB40002044012280F82220C1EB01100E
:1039900000EB4000204400220EF060FF29E669465B
:1039A00028460EF03FFF9DF800004028F6D289F827
:1039B0000070C0EB0011374D01EB4101294481F843
:1039C00023709BF800109AF80020114481421BD903
:1039D00008EB801141F8264023F049FB2B492FF0DA
:1039E000B8FB2FF03FFD2BF075FA9DF80090C9EB66
:1039F000091101EB41012944C1F81E002FF006FD19
:103A00000146484602F0FFF99AF800009BF80010C2
:103A100001449DF80000814228D8C0EB001101EB61
:103A20004101294481F8227008EB8010C4630F2EF5
:103A300002D0174940F82610144920462FF089FB80
:103A40002FF010FD04462BF045FA9DF80010C1EB55
:103A5000011101EB41012944C1F81E0020462BF061
:103A600039FA0D499DF8002021F8120002F0C7F93B
:103A70009DF800100022C1EB011000EB400028442B
:103A80000CE000005AE402600835056000007A444A
:103A900000007F43C8400560AED102600EF0DEFE3C
:103AA000A7E589F80470F74920462FF052FB2FF064
:103AB000D9FC2BF00FFA0146C5EBC500F24A00EB2A
:103AC000400002EB4000817793E589F80570ED49ED
:103AD00020462FF03EFB2FF0C5FC2BF0FBF9EB4A04
:103AE00005EB45111144887783E52DE9F84F04462D
:103AF0008A461646E64801250570DFF89893DFF8F8
:103B0000988377B2042C11D188F80050694650464A
:103B10000EF096FE9DF80010C1EB011000EB400086
:103B2000484480F8227001220EF098FE022C11D138
:103B300088F80050694650460EF074FE9DF800105B
:103B4000C1EB011000EB4000484480F822700122D4
:103B50000EF084FED14F092C0ED188F80250694630
:103B600050460EF035FE9DF80000C0EBC00101EBA1
:103B70004010384480F82260002C0ED188F80250A2
:103B8000694650460EF016FE9DF80000C0EBC001DD
:103B900001EB4010384480F822602AE52DE9F84313
:103BA000014610461E46BA4A01241470BA4DBC4F55
:103BB000DFF8E092DFF8E4820A2922D2DFE801F0A0
:103BC00077055B223F9BAA21218969460EF00EFEF4
:103BD0009DF80000802814D26C70C0EBC00101EB8E
:103BE000001007EB4000152231462FF0B1F89DF888
:103BF0000000C0EBC00101EB001007EB40000EF02D
:103C0000D8FE19E469460EF0FFFD9DF800008028FB
:103C1000F7D26C70C0EBC00101EB001007EB400065
:103C2000152231462FF094F89DF80000C0EBC0013A
:103C300001EB001007EB40000EF0BBFE13E46946F9
:103C40000EF0FEFD9DF800004028F7D22C70C0EB6E
:103C5000001000EB40004844132231462FF078F862
:103C60009DF800100122C1EB011000EB4000484418
:103C70000EF0F4FD0EE469460EF0D4FD9DF8000050
:103C80004028F7D22C70C0EB001000EB40004844F5
:103C9000132231462FF05CF89DF800100122C1EB91
:103CA000011000EB400048440EF0D8FD09E46946DD
:103CB0000EF080FD9DF800008028F7D2AC70C0EBBC
:103CC000C00101EB40104044152231462FF040F86E
:103CD0000AE469460EF07CFD9DF800008028F7D2CA
:103CE000AC70C0EBC00101EB4010404415223146DE
:103CF0002FF02EF80BE40828FCD22C71C0EBC0008A
:103D0000614900EB400001EB4000152231462FF0E5
:103D10001FF80CE40428FCD26C715C4900EB4010E5
:103D20000844152231462FF013F80DE4584B0122B8
:103D30001A70594B1A76014614225A482FF008B8C7
:103D400070B50022594D00EBC000574E05EBC00581
:103D5000002306EB0010FF2405EBC10500EB01106A
:103D600000EB42014B7000F81230AC54521CD2B23E
:103D7000082AF5D370BDF0B5DDE90556444F01249E
:103D80003C70454F3C74484C00EBC00004EB001401
:103D900004EB011404EB42077B7004F81250434B10
:103DA00003EBC00000EBC1008654F0BD77B5384985
:103DB00001250D7038494D743D49BDF804308979AD
:103DC00001F5FA62934229D13A4B890709D01C21A7
:103DD000597000229DF80640641E0B2C0BD8002160
:103DE00007E01D215970F4E75E5C324492B2491C31
:103DF000C9B28C42F8DC9DF80710114489B2C0EBBF
:103E0000C00202EB00122C4800EB420000EBD10094
:103E100001F0070102788D402A4302707EBD10B583
:103E2000264840F2E53400880146FF286ED00CDCBD
:103E3000022851D004DC002868D0012811D112E0FA
:103E4000032856D094280CD160E0A0F54070E538E6
:103E500042D00A2807D0D1284BD0A0F57C401A3890
:103E600054D0084610BD1548142215A1801C2EF010
:103E70006FFF1248142216A116302EF069FF40F28F
:103E8000EF3010BD00007A445C4E03606C56036056
:103E9000EE030060C840056030E70360F2E80260AE
:103EA0000835056008B10360AC4F03602C54036013
:103EB0001018006022D40260F0560360B601006062
:103EC0004E4554495820436F6E74726F6C730000F6
:103ED0004E434342000000001422FAA1FC482EF099
:103EE00037FFFB481422FBA114302EF031FF20468F
:103EF00010BD1422FAA1F6482EF02AFFF44814222D
:103F0000FCA114302EF024FF204610BD1422FCA189
:103F1000EF482EF01DFFEE481422FDA114302EF0C4
:103F200017FF942010BDEA487047E94814307047E5
:103F300010B5FB4B01225A7601461422E4482EF0BC
:103F400007FFBDE810400CF0FDB810B5F44B01229E
:103F50005A760146DE48142214302EF0F9FEBDE8F0
:103F600010400CF0EFB810B50446E1B2AF20F6F700
:103F7000C0FC210AE120F6F7BCFC002C0CD0FF2C81
:103F80000AD0A4F57F40FF3806D0012C04D0022CC3
:103F900002D0CF48801E048010BDE24948727047AD
:103FA000E048407A002800D001207047DE490268CE
:103FB0000A6002790A71DB4AC378D370837853713F
:103FC0000379137100783C38C0B2907100F5FA6043
:103FD0000880D649012008707047D54902680A60F8
:103FE000D04902788A7042784A7080780870CF4948
:103FF000012008707047CF48B0F900007047704743
:104000000EB5C9490A68019209798DF80810C849A6
:104010000968009102280DD1C74A01211170C74AD1
:1040200000211170C64A052111700246694601A897
:1040300029F032FB0EBD70B503460C461046C14A4E
:1040400001211170B64A5176BF49C04E042B097840
:104050000FD0022B66D10C4446F824002FF01BFA37
:10406000BB4921F81400E0B2BDE87040002101F026
:104070001CBF8C4256D246F82400C4EB041101EB5D
:104080004102B449551895F82310A1BB95F92810A1
:10409000A1F10C020A2A0FD91739072907D801EB19
:1040A000C10202EB0111AC4A515C012904D010F0AD
:1040B000FF4F15D0012014E010F0FF4F0CD000206E
:1040C0002FF0ADF946F82400204624F034FD28B145
:1040D000002085F8250012E00120F1E70120F8E733
:1040E00000202FF09CF946F82400204624F023FD00
:1040F00010B1012001E00FE0002085F8250095F8BF
:10410000250028B14FF47A7120460BF083F903E0C3
:10411000002120460BF07EF92046BDE870400021CA
:1041200001F0C3BE70BD884A884B0428127803D0C2
:10413000881853F8200070479142FCD253F82100B0
:104140007047F0B5002100220020854B834C03F519
:10415000007503F1400603F51077C0EBC00C0CEBC3
:10416000001C04EB4C0C9CF828C0BCF1010F0CD0D7
:10417000B0543A54521CD2B2401CC0B24028ECD3C6
:104180007848017078480270F0BD58542954491C91
:10419000C9B2F1E7F0B5002100220020704C6D4D4E
:1041A000803404F5007604F1400704F5107CC0EB80
:1041B000001303EB43032B4493F82330012B0DD062
:1041C000B8540CF80020521CD2B2401CC0B2402897
:1041D000EDD36648017066480270F0BD60543154FA
:1041E000491CC9B2F1E730B5002100220020614C22
:1041F000C0EBC00303EB4013234493F82330012B9F
:1042000006D15D4D685405F500752954491CC9B2A5
:104210003BB9594B8033985403F500731A54521C20
:10422000D2B2401CC0B28028E2D354480170544836
:10423000027030BD70B502460020484C454D4D4BD4
:10424000062A17D2DFE802F0039EB1172AC4002223
:10425000C2EBC20303EB021304EB430393F82830D1
:10426000012B03D18A422BD0401CC0B2521CD2B2C7
:10427000402AEDD3BDE00022C2EBC20303EB0213E0
:1042800004EB430393F828301BB98A4218D0401C32
:10429000C0B2521CD2B2402AEED3AAE00022C2EB36
:1042A000021303EB43032B4493F823301BB98A42D8
:1042B00006D0401CC0B2521CD2B2402AEFD398E0C4
:1042C00099E000004A6574436F6E74726F6C7300FE
:1042D000B80100604A65742050726F6475637400A1
:1042E0004E6577726F6E20536F6C7574696F6E7365
:1042F000000000004E6577726F4E6F64650000002D
:1043000054656D636F436F6E74726F6C7300000061
:1043100054656D636F2050726F64756374000000A4
:1043200030E70360101800609E020060F90300602F
:10433000A30200609E03006010030060170300608A
:1043400011030060EE030060A7020060588F036055
:10435000AED10260C84005605AE4026008350560CD
:1043600028C30160D404006011050060D50400601A
:1043700013050060F2E8026028C40160D604006002
:10438000120500600022C2EB021303EB43032B442F
:1043900093F82330012B03D18A422CD0401CC0B2A9
:1043A000521CD2B2402AEED323E00022C2EBC20458
:1043B00004EB42141C4494F82340012C03D18A429C
:1043C00019D0401CC0B2521CD2B2802AEED310E0E9
:1043D0000022C2EBC20404EB42141C4494F82340B4
:1043E0001CB98A4207D0401CC0B2521CD2B2802AEB
:1043F000EFD34FF0FF3070BD70B50022F64DF74C93
:10440000F74B062874D2DFE800F0033C4F172A620E
:104410000020C0EBC00303EB001305EB430393F84C
:104420002830012B03D18A4264D0521CD2B2401CE6
:10443000C0B24028EDD35BE00020C0EBC00303EB2B
:10444000001305EB430393F828301BB98A4251D07F
:10445000521CD2B2401CC0B24028EED348E000202B
:10446000C0EB001303EB4303234493F823301BB941
:104470008A423FD0521CD2B2401CC0B24028EFD377
:1044800036E00020C0EB001303EB4303234493F812
:104490002330012B03D18A422CD0521CD2B2401CB3
:1044A000C0B24028EED323E00020C0EBC00404EBF0
:1044B00040141C4494F82340012C03D18A4219D0A3
:1044C000521CD2B2401CC0B28028EED310E00020B3
:1044D000C0EBC00404EB40141C4494F823401CB906
:1044E0008A4207D0521CD2B2401CC0B28028EFD3FF
:1044F0004FF0FF3070BDBB49085C40280FD2C0EBC5
:10450000C00101EB0010B44901EB400090F82D0010
:10451000401E0A2801D80020704701207047002063
:10452000704710B5002240281DD2401EAA4BC0EB98
:10453000C00404EB001003EB400049B190F82D10CB
:104540004B1E0A2B0FD80B3180F82D10012010BD07
:1045500090F82D10A1F10C030A2B04D80B3980F828
:104560002D10012010BD104610BD9E498031085C01
:1045700040280ED2C0EB0010984900EB40000844E0
:1045800090F92800401E0A2801D800207047012019
:10459000704700207047002240281CD2401E8F4BDD
:1045A000C0EB001000EB4000184449B190F928100E
:1045B0004B1E0A2B0FD80B3180F8281001207047B2
:1045C00090F92810A1F10C030A2B04D80B3980F8BC
:1045D000281001207047104670478349085C8028E6
:1045E0000ED2C0EBC00101EB40107D49084490F8A9
:1045F0002600401E0A2801D800207047012070477D
:104600000020704710B5002280281CD2401E744B39
:10461000C0EBC00404EB4010184449B190F82610D8
:104620004B1E0A2B0FD80B3180F82610012010BD2D
:1046300090F82610A1F10C030A2B04D80B3980F84E
:104640002610012010BD104610BD2DE9F0410025B7
:104650000024C0EBC00101EB0010644901EBC0076E
:10466000C4EBC40000EB041038440646401C2EF096
:10467000AFFB38B1701C2EF0ABFB142802D86D1CB8
:10468000EDB200E00824641CE4B2082CE8D35448DE
:10469000C0F82A532846BDE8F08110B5C0EBC0022F
:1046A00002EB0012514800EBC200C1EBC10202EB69
:1046B00001114418601C2EF08BFB002805D0601CF3
:1046C0002EF086FB142800D8601C10BD70474649A8
:1046D0008031085CC0EBC00101EB00123E4901EBE8
:1046E0004201434AD1F81E1052F82030994203D0BB
:1046F00042F8201001207047002070473A49C0312D
:10470000085CC0EBC00101EB0012334901EB420130
:10471000374A91F9261052F82030994203D042F8D6
:104720002010012070470020704710B5014600207E
:10473000304A515CC1EBC10202EB4113284A1A44D2
:104740002D4BD2F81E2053F82140A24202D043F84C
:104750002120012010BD10B501460020244A803AD6
:10476000515CC1EBC10202EB41131D4A1A44224BBA
:1047700092F8242053F82140A24202D043F821208D
:10478000012010BD1B498039085CC0EB001101EB12
:10479000410212491144194AD1F81E1052F8203032
:1047A000994203D042F82010012070470020704742
:1047B00010494039085CC0EB001101EB4102074988
:1047C00011440E4A91F9251052F82030994217D021
:1047D00042F820100120704708350560C840056088
:1047E000F2E8026068C30160A8C40160F8DE0360FB
:1047F00028C7016028C6016028C8016028CA016076
:104800000020E8E710B50446A1B2A32020F04FF83D
:10481000C4F30721A42020F04AF8C4F30741A520DF
:1048200020F045F8210EBDE81040A62020F03FB84A
:1048300070B5E54C0225E54E94F82800092806D10C
:1048400084F8285086F82650002011F08FFF94F845
:104850002A00092808D184F82A5086F82850BDE893
:104860007040022011F082BF70BDD9480078012845
:10487000B1D1D8483C210088B0FBF1F000F07F00B6
:104880008030C1B2E920F6F734B8A4E770B5002053
:1048900020F06DF8CC491D2028311FF0F9FFCA4DDA
:1048A000CA4C2835263428782070022020F05FF882
:1048B000A91C1F201FF0ECFFA878A07070BD10B5D8
:1048C000C34A1078002804D0C249088810B1401E9D
:1048D000088010BD0020107008800021E9201FF022
:1048E000E6FFBDE81040D1E701469D201FF0DFBF85
:1048F00000B585B0042802D0B7A005B000BD1421D2
:1049000068462EF03EFAB148FE304278007869469B
:10491000012A03D0022A0BD0B1A0EEE7B2A212887E
:10492000ADF800200A22891C21F02EF96846E4E740
:10493000AEA21288ADF8002052228DF802200A2281
:10494000C91C21F021F96846D7E72DE9F047042872
:1049500002D00020BDE8F0879C4E08789A4BDFF823
:1049600090C2B6F8014196F8035101276FF02F0865
:10497000492804D191F80190B9F14E0F02D0562880
:1049800025D04FE086F8FF708878303809280CD899
:10499000C978A1F13009B9F1090F06D800EB800000
:1049A00008EB40000844C2B202E0092800D8C2B2B5
:1049B0000AB186F8FE208548D0F8FD0043F85C0F68
:1049C0009C809D718CF819700BF0BCFB2AE0487834
:1049D000412827D18878522824D1022086F8FF0068
:1049E000C878303809280CD80979A1F13009B9F113
:1049F000090F06D800EB800008EB40000844C2B263
:104A000002E0092800D8C2B20AB186F8FE206F4839
:104A1000D0F8FD0043F85C0F9C809D718CF81970F4
:104A20000BF090FB012095E7F0B5ADF25C6D05460B
:104A30000E460024CDF84C46CDF85046CDF85446ED
:104A4000CDF858464FF41871FBA82EF09AF94FF4A0
:104A5000F07183A82EF095F94FF48270ADF84C06F2
:104A60000127CDF84E7637208DF804008DF80540EB
:104A700073208DF806008DF807508DF808603020FF
:104A80008DF809008DF80A405A4907200870701BFC
:104A9000401C00EB40004FF6FF7101EA001256483F
:104AA000028056490DF10B002EF052F9FBAA01A924
:104AB000062024F0E3FDFBA983A824F0A5FA83A92E
:104AC000CDF85216CDF856064D4807704D48047083
:104AD0004D4905200870801F00F032F97EA800F0D3
:104AE0004EFB02220DF24C617EA827F075FD0DF2FF
:104AF0005C6DF0BD30B5ADF25C6D05460024CDF8BF
:104B00004C46CDF85046CDF85446CDF858464FF4B3
:104B10001871FBA82EF035F94FF4F07183A82EF030
:104B200030F900944FF48270ADF84C060120CDF8B6
:104B30004E0607208DF804008DF805405E218DF8A3
:104B400006108DF807408DF808400A218DF80910ED
:104B50008DF80A402749087027480480FBAA01A95C
:104B6000062024F08BFDFBA983A824F04DFA83A92D
:104B7000CDF85216CDF856062448007818B1601EBC
:104B80000DF25C6D30BD22490220087021490320DE
:104B900008702B20454320482844204D417A297035
:104BA00000687EAA694622F0A4FF1D4C50B1287807
:104BB000401EFE2806D200220DF24C617EA827F08E
:104BC0000BFD20702078DBE762730460AED80260D2
:104BD000FA030060480400606572726F72000000A2
:104BE0006E756C6C00000000494E0000564152008A
:104BF00030E70360480200604E02006022E5026078
:104C00001003006017030060110300604D02006094
:104C10004C020060E20700602CCE0360BF0700601A
:104C200060030060F74948807047F6491431086016
:104C30007047F4498860704738B50020FFF7F9FFE6
:104C40000020FFF7F2FFF04C2088FFF7EBFF2088F1
:104C5000010241EA102080B2F9F74FF94FF0FF321C
:104C6000042168462EF086F834F84909010241EA29
:104C7000102081B26846F9F7D9F8002805D0B4F8B9
:104C800049100A0242EA1121818038BDF0B587B08F
:104C9000DE4EDC4D3078000721D5DD4F3868E86006
:104CA0002969401A64281AD3DA4CDB4920780A783B
:104CB00090420FD20A280DD240F22D114843D74915
:104CC00001EB4000B0F85812F9F7A8FF2078401C1B
:104CD000207002E000202070087038682861307869
:104CE00080071AD5CE48E861CE4CCF4922880968A2
:104CF0002EF02EF82088A8800120009000234FF489
:104D00001672C74902A825F09FFD0246002A04D06A
:104D10000123C34902A827F014F907B0F0BDB94830
:104D200080687047B7488068401C00D001207047F9
:104D3000B448143000687047B249183108607047B1
:104D4000BA49020E0A70020C4A70020A8A70C870D0
:104D5000AC484088020A0A7148717047A948183067
:104D600000687047A748408870470023002805D096
:104D700050F8013F0B60808810800623184670476A
:104D80002DE9F047ADF5247D0446AC9E91461D46C5
:104D90004FF0000ACDF878A24FF41E7841466846DD
:104DA0002DF0EFFFA24F9749387848B9012E07D16F
:104DB0008868002804DA00200DF5247DBDE8F0871E
:104DC00081208DF800000220ADF880022089A0F536
:104DD0007F42FF3A09D008B1A07A30B1207820B1E3
:104DE00006280CD04FF0FF30E6E786481830006800
:104DF0009F9048889E900B208DF8010007E09EAAA6
:104E00009FA92046FFF7B1FF0A208DF801009F9867
:104E1000A190BDF87802ADF88202CDF888A2CDF855
:104E20008CA2281D81B2EA460DF1020025F094FB08
:104E3000841C0AEB04002A4649462DF089FF2C44C5
:104E4000012E08D1387860B12246694679482DF0A4
:104E50007FFF79480480414668462DF092FF204646
:104E6000AAE721466846F9F7D9FEF4E738B50D46BA
:104E70001346724801240470714A00201070714A70
:104E800005201070801FFFF75BFF00212A460846AF
:104E90000094FFF775FF38BD2DE9F047ADF5267D8D
:104EA000044691461D464FF00008CDF880824FF42D
:104EB0001E77394602A82DF064FF81208DF8080086
:104EC0000220ADF8880220894E4EA0F57F41FF39BF
:104ED0000BD008B1A07A40B1207830B106280ED0AE
:104EE0004FF0FF300DF5267D68E746481830006822
:104EF000A1907088A0900B208DF8090007E0A0AA6F
:104F0000A1A92046FFF731FF0A208DF80900A198DA
:104F1000A390BDF88002ADF88A02CDF89082CDF85A
:104F20009482281D81B20DF1080A0DF10A0025F0C6
:104F300013FB841C0AEB04002A4649462DF008FFA7
:104F40002C443E48007878B3306A08B1A0F8048059
:104F50003C4905200870354948780A7840EA022023
:104F6000020242EA1020ADF80400C878897840EACD
:104F70000120010241EA1020ADF80600708801020C
:104F800041EA102081B201A8F8F750FF306210B159
:104F900044F29C518180224602A92B482DF0D8FE74
:104FA0002948A0F8584204E0FFE721462748F9F7CE
:104FB00035FE394602A82DF0E4FE204692E72DE9A1
:104FC000F0478EB080460D46174600260D9609968E
:104FD0000A960B960C9605960696079608960196E5
:104FE0000296039604960024DFF84490054A99F847
:104FF000000000282CD1012B2AD19168002927DA42
:105000000EB0DBE6E0010060AB730460AC00006052
:1050100030000060550100605401006068A4016028
:105020009ECD0160B0000060C800006042030060D7
:10503000BE04006066F50460C604006010030060F2
:105040001703006011030060B22B016028CB0160E0
:105050009188D561012B04D118B9002901DC002009
:10506000CEE72978812900D080B195F801A00DA95B
:10507000A81C25F076FA0A96ADF82660ADF8166001
:10508000ADF8066099F8000010B108E00020B7E71D
:1050900046480068C188ADF8261000680A90BDF83F
:1050A0003400001F0D90BAF10A0F03D0BAF10B0FB4
:1050B00037D122E0FFF73CFE0A99884207D1FFF77B
:1050C00051FEBDF82610884201D10D9629E009A9AC
:1050D000404625F068FBBDF83400B84205D30AE02D
:1050E000281900792855641CA4B2BDF83400001DAD
:1050F0008442F5D315E00D9613E009A9404625F04A
:1051000052FBBDF83400B84205D309E028190079F4
:105110002855641CA4B2BDF834008442F6D300E0E4
:105120000D96BDF834006BE72148B0F84200704797
:1051300070B500281ED0062505701E4B5969C0F8B1
:1051400001105988A0F805101949B1F842200281D0
:10515000B1F842200024A2F57F46FF3E0BD052B1A9
:105160001A78012A09D0857251F8132F40F80B2FB5
:105170008988818070BD847270BD8472F4E70021DB
:10518000002812D0062202700A4A9369C0F8013042
:105190005288A0F805204FF6FF7202810022827229
:1051A0004318DA72491C0729FADB7047D400006003
:1051B00062730460E00100602DE9FF5FDDE90EA687
:1051C000DDE91075894693469846002D53DB05EBC3
:1051D0000510FF4900EB400001EB4004662120462A
:1051E0002DF0CFFD022084F863000120E07184F8E7
:1051F000655084F858B009F07CFC29F06BFEC4F8C7
:105200000E003A20A07484F85790F2480188A4F860
:105210005510491C018084F80B8000982DF0D8FDB2
:10522000A07404F1130000992DF0FEFDBAF1000FF7
:1052300002D0FF2084F8590066B104F15901002022
:1052400004E03A5C01F8012B401C00B2B04201DAE4
:105250000528F6DB002084F86300DF490878401C4D
:10526000C0B20870102801D910200870DB490888E6
:10527000401C088001E04FF0FF356D1C04B028B2DF
:10528000BDE8F09F2DE9F0470646DDF8209017466F
:105290009846CF4C0025E079012807D0A07A70B35A
:1052A0000020A0726D1C28B2BDE8F08794F8580069
:1052B000B8421AD1B8F1000F08D0B4F85500B6F9C9
:1052C0000010884211D16D1C28B2EDE7207A60B938
:1052D00030462DF07DFD94F91210884205D13146FB
:1052E00004F113002DF07BFD30B166346D1C2DB23E
:1052F000102DD0DB0020D7E76D1C28B2D4E7FFE7E4
:10530000A9F800500020CFE72DE9F04F85B00EAD91
:105310008046E0CD894692469B464FF0FF34049488
:1053200004A800900023524649464046FFF7AAFFD2
:10533000002803DD204605B0BDE8F08FBDF9104020
:10534000002C15DB8DE8E0005B465246494640469E
:105350000394FFF731FFA248017841F00101017089
:10536000A04901200870C82241469F482DF0F0FC5A
:10537000BDF81000401C00B2DDE72DE9F04FB7B0DA
:10538000002400250026A1460020984A4FF001087D
:10539000C0EBC00101EB001102EB410191F92310B8
:1053A000CB0707D009F1010909F0FF0908FA00F15C
:1053B0000D4306E0890704D5761CF6B208FA00F121
:1053C0000C43401CC0B22028E2D3C82105A82DF010
:1053D000D8FC2C274FF0200BB9F1000F7ED04F20C6
:1053E0008DF8140070208DF8150065208DF81600DA
:1053F0006E228DF817208DF818B063208DF81900F3
:1054000069208DF81A0072218DF81B1063218DF828
:105410001C1075214FF00A0A8DF81D108DF81E0022
:1054200074208DF81F008DF820B06F208DF82100BA
:105430008DF822208DF823B049208DF824004E20CD
:105440004FF0120C8DF82500002008FA00F12942D7
:105450002DD0092810D2411CB1FBFAF20AFB12121E
:1054600005AB30320CF10101C9B203F80C204A1C23
:1054700002F0FF0C5F541AE0431CB3FBFAF905AAD3
:1054800009F130090CF10101C9B202F80C90B3FB2B
:10549000FAFC0AFB1C33303301F1010C0CF0FF095C
:1054A000535409F1010101F0FF0C02F80970401C8E
:1054B000C0B22028C9D3BCF13A0F01D94FF03A0C41
:1054C00005A9002001F80C004A4A4B4B484992F9C3
:1054D000002093F90030CDE9003200E00DE0CDE985
:1054E000021046480023FF21027805A8FFF70CFFB1
:1054F000C0B210B1424880F80080C82105A82DF044
:1055000040FC002E7ED053208DF8140068208DF8CA
:1055100015006F218DF8161072208DF81700742079
:105520008DF818008DF819B063228DF81A206922C1
:105530008DF81B2072238DF81C3063230A258DF80B
:105540001D3075238DF81E308DF81F208DF820003A
:105550008DF821B08DF822106E208DF823008DF883
:1055600024B049208DF825004E2113208DF82610F7
:10557000002108FA01F2224225D009290DD24A1C45
:10558000B2FBF5F305FB1323303305AE421CD2B258
:105590003354501CC0B2B75415E04A1CB2FBF5FCA2
:1055A000134605AE0CF1300C421CD2B206F800C016
:1055B000B3FBF5F005FB10303030531CDBB2B054B8
:1055C000581CC0B2F754491CC9B22029D1D31AE0E3
:1055D0001ADC02606C020060580200607402006015
:1055E000AA0200609501006066BE01600835056092
:1055F000D3020060D2020060D1020060AB02006002
:10560000D00200601DE03A2800D93A2005AA002106
:105610001154DC4ADC4BDA4892F9002093F900304F
:10562000CDE90032CDE90201D8480023FF210278FC
:1056300005A8FFF769FEC0B2002802D0D44880F860
:10564000008037B078E6F0B5B7B004460E46154690
:105650001F46C82105A82DF094FB3CB33B463246BB
:10566000CCA105A800952EF08FFE05A82DF0B0FB6B
:1056700000213A2801D98DF84E10C24AC24BC048C9
:1056800092F9002093F90030CDE90032CDE9020112
:10569000BE480023FF21027805A8FFF735FE002849
:1056A00002DDBB490120087037B0F0BD3B463246F1
:1056B000C1A105A82EF068FED7E710B5B6B0044624
:1056C000C82104A82DF05DFB012C2ED0022C31D076
:1056D000032C34D0042C37D0052C3AD0072C22D1FF
:1056E000C1A104A82EF050FE04A82DF071FB0021EA
:1056F0003A2801D98DF84A10A24AA34BA04892F942
:10570000002093F90030CDE90032CDE902019F4835
:105710000023FF21027804A8FFF7F6FD002802DD30
:105720009B490120087036B010BDB5A104A82EF029
:105730002BFED9E7BBA104A82EF026FED4E7BFA11B
:1057400004A82EF021FECFE7C2A104A82EF01CFE73
:10575000CAE7C74903200870C64981F8C200C6A13C
:1057600004A82EF011FEBFE730B589B004460D46FF
:10577000142104A82DF005FB24B1012C08D0022C23
:105780000CD010E02A46C1A104A82EF0FDFD0AE0CD
:105790002A46C5A104A82EF0F7FD04E02A46C9A1B7
:1057A00004A82EF0F1FD04A82DF012FB0021754A8B
:1057B000754B734892F9002093F90030CDE900321F
:1057C000CDE9020171480023FF21027804A8FFF708
:1057D0009BFD002802DD6E490120087009B030BD34
:1057E0002DE9F04180460E461746BE4C0025E07973
:1057F000B0B194F85800B84212D194F85700B042B2
:105800000ED1207A60B940462DF0E2FA94F91210D8
:10581000884205D1414604F113002DF0E0FA30B181
:1058200066346D1C2DB2102DE1DBBDE8F081012046
:10583000433404F83B0C0020E07620776077A077B3
:10584000E07714F83A1C29B9A74B19784A1E1A7048
:1058500000D21870A548017841F002010170E4E718
:1058600070472DE9F84F00259E4A00920026474ACE
:10587000DFF874824FF0010992F800C00027009A07
:10588000D379002B65D092F86330EBBB022382F80A
:105890006330034600240DE093F807A0BAF1000F2F
:1058A00005D092F865A093F865B0DA4504D0641C81
:1058B00024B266338C42EFDB8C4202DB82F86370E9
:1058C00047E09C7A24B3137A4BB9537A3BB998F8E2
:1058D00000305C1E88F8004001D288F80070D77153
:1058E00082F863701772577282F80A9082F86470B7
:1058F00092F85830634506D102F85E7F5770977072
:10590000D77017715E3A00E023E045F0020520E011
:105910005B7AE3B1537AD3B9137A3BB998F8003084
:105920005C1E88F8004001D288F8007082F8099067
:1059300082F8647092F85830634506D102F85E7FB1
:1059400057709770D77017715E3A45F0010582F86D
:105950006370761C36B266320092102E8FDB002DFB
:105960000AD0624991F9000040F001000870AA07CE
:1059700002D540F002000870BDE8F88F70470000C3
:10598000D3020060D2020060D1020060AB0200606E
:10599000D00200604944203A257520534E3A202514
:1059A0006C752068617320636F6E6C696674205338
:1059B0004E3A20256C7500004944203A2575205345
:1059C0004E3A20256C752068617320636F6E6C6998
:1059D0006674207769746820543320636F6E747224
:1059E0006F6C6C657200000043414E204E4F542096
:1059F000434F4E4E45435420534E54500000000038
:105A00004C6F737420636F6D6D756E696361746F35
:105A10006E207769746820746F7020626F617264A1
:105A2000000000005245414420414F204665656416
:105A30006261636B204641494C000000557064610F
:105A400074652074696D6520736572766572206671
:105A500061696C004C6F736520636F6D6D756E6965
:105A6000636174696F6E2077697468207069630080
:105A7000A0040060AED80260534420434152442049
:105A800049532041424E4F524D414C005052472005
:105A90002564206572726F72203A2064656164200B
:105AA0006379636C6531000050524720256420659E
:105AB00072726F72203A2064656164206379636C4E
:105AC00065320000505247202564206572726F7263
:105AD000203A2074616B6573206C6F6E6720746967
:105AE0006D6500001ADC026058020060AA020060C6
:105AF0002DE9F047FF49C0EBC00301EB83040A2204
:105B0000A275E17C01296ED0FB4900EB400001EB5E
:105B10008005E11C204604F0F5FD04F10E01C81ECD
:105B200004F0F0FD0026B046E07D4FF6FF7101EA7B
:105B30000020217E084487B2D4F8030029F0CAF976
:105B4000DFF8B893C9F80C00D4F80E0029F0C2F9B8
:105B5000C9F81000D9F80C10A1EB000C002127B1F6
:105B600064200CFB00F090FBF7F1DFF894934945BB
:105B700000DD4946207D00B94942286800EB0C024F
:105B8000A07D4008424368680244002804DBB2F567
:105B9000000F06DBDB4A04E012F5000F01DCD94AF6
:105BA00052426A60637E83B1207D10B103FB02F62E
:105BB00001E003FB1266607D18B13C2096FBF0F615
:105BC00003E04FF4616096FBF0F6E27EA2B1286834
:105BD0004FF0640800FB08F090FBF7F04042277D8F
:105BE00017B1424302E021E052424243A07DC0EBA4
:105BF0000010800092FBF0F8642098FBF0F008445D
:105C0000A17E0844484500DD4846002800DA00200F
:105C100033B13044484500DD4846002800DA002012
:105C2000C5F800C029F056F9C4F80700BDE8F087B0
:105C30002DE9F843B44C0026DFF8D082DFF8D0928B
:105C4000002798F80400401E45B2002D00DA062512
:105C5000E07FE8BB94F8280090B1694604F1270082
:105C600004F050FD0098002802D04FF0010001E040
:105C70004FF0000084F8210004D04FF0080501E047
:105C800084F8217094F8250090B1694604F124004D
:105C900004F038FD0098002802D04FF0010001E028
:105CA0004FF0000084F8200004D04FF0070501E019
:105CB00084F82070974806EBC60200EB021000EB58
:105CC000051000F10E004FF0070198F8023000E0D7
:105CD00018E098F801C009EBC20202EBC502555C5E
:105CE000FF2D06D04578AB4208D802D10578AC45E7
:105CF00004D2801E491E49B20029F0DA505CFF2808
:105D000007D0A0772A34761C76B2082E99DBBDE83E
:105D1000F883A777F6E730B57F480021C27FCAB97C
:105D200001237A4AB2F80720521E42F3C70402F058
:105D3000070293405AB2C1EBC103784D03EB011344
:105D400005EB43031B5D134202D00122827701E081
:105D500000228277491C49B221300429DEDB30BDA4
:105D600010B500206E4B0021C0EBC00202EB001208
:105D700003EB420282F82910401CC0B21028F3D372
:105D8000684890F8090102281ED00020664CC0EB3C
:105D9000C00101EB810114F81120002A14D0012A5E
:105DA0000ED104EB41014979102909D2C1EBC1029E
:105DB00002EB011103EB410111F8292F521C0A706B
:105DC000401CC0B2F028E2D310BD10B54B4AD188B8
:105DD000642911D30023D38011794C1C1471B1FBB9
:105DE000F0F400FB1410002808D1137103F0FDF843
:105DF000BDE8104003F0ACBA491CD18010BD3F494A
:105E000000208860704770B504460846C4EB041152
:105E1000464A01EB41011144454D91F928100929E9
:105E200038D2DFE801F03705101B10101B102600D8
:105E300040492DF0C0F92DF02EFB81B22046BDE87F
:105E4000704009F0E7BA3C492DF0B5F92DF023FB7D
:105E500081B22046BDE8704009F0DCBA37492DF028
:105E6000AAF92DF018FB81B22046BDE8704009F078
:105E7000D1BA03212DF0DDF929462DF09CF93049E6
:105E80002DF00FF92DF007FB81B22046BDE87040E0
:105E900009F0C0BA29462DF08EF92DF0FCFA81B236
:105EA0002046BDE8704009F0B5BA2DE9F047054637
:105EB0000A46244B24491878097844182448234971
:105EC00000EB8516AC4201D8F161AFE6C5EB0510D9
:105ED00000EB400415481F4F0444DFF87C9094F811
:105EE0002200DFF84CA04FF47A7810B1FFF787FF5B
:105EF00034E03AE072FC0260F6CF01600402006018
:105F0000A0860100FFFF7F005C4E03601018006058
:105F10002C540360AC4F03606C560360F056036072
:105F2000DC090360AED80260BC0C0360C8400560A9
:105F300000007A44000020410000C8420000A04157
:105F400000004843A7020060A802006000007F43F1
:105F5000587F03605AE40260AED1026094F82300D7
:105F6000002862D0002A75D0C1E0F16194F82300C6
:105F7000C0B109F041FBA84250D9284621F077F87A
:105F800051462DF0E6F82DF06DFA28F0A3FFC4F885
:105F90001E0028F09FFF2DF039FA01462846BDE883
:105FA000F04730E7284622F0C6FD4FF47A714843A7
:105FB00028F090FFC4F81E0094F92800A0F10C010D
:105FC0000A290FD91738072806D800EBC00101EBC2
:105FD0000010385C012805D0284622F0ACFD58B1ED
:105FE00001200AE0284622F0A6FD18B1002084F81E
:105FF000250004E00120FAE7002084F8250094F849
:10600000250028B141462846BDE8F04709F002BA0C
:106010002846BDE8F047002109F0FCB9D4F81E007D
:1060200028F058FF29F8150000E62AB994F8250051
:10603000012810D00020F061187885420FD2284640
:1060400022F079FD4FF47A71484328F043FFC4F8F9
:106050001E0010E041E04FF07E50F061ECE7284672
:1060600021F005F851462DF074F82DF0FBF928F0D9
:1060700031FFC4F81E0094F92800A0F10C010A2990
:106080000FD91738072806D800EBC00101EB001024
:10609000385C012805D0284622F04DFD58B101207A
:1060A0000AE0284622F047FD18B1002084F82500B8
:1060B00004E00120FAE7002084F8250094F8250088
:1060C00028B141462846BDE8F04709F0A3B9284663
:1060D000BDE8F047002109F09DB9D4F81E0028F072
:1060E000F9FE2DF093F951462DF065F8F06109F0B5
:1060F00083FAA84214D9284620F0B9FF51462DF062
:1061000028F82DF0AFF928F0E5FEC4F81E0028F0BD
:10611000E1FE2DF07BF901462846BDE8F04772E626
:10612000D4F81E0028F0D6FE29F815007EE508B543
:10613000F6F7E0FB0090DFF8EC93012689F8456064
:10614000F9480025457005708570C570F74890F8CE
:106150000901022801D0FFF703FE0024E0B200216C
:10616000FFF7A3FEFFF74BFE641CA4B2402CF5D34F
:10617000EF49C6201EF08CFBED4F3878401CC1B2B1
:106180003970C6201EF093FB3878DFF8A883052805
:106190000FD9002000EB800101EB4011414481F850
:1061A0002050401C80B21028F4D30021C6201EF0DD
:1061B0007EFBE1480670E14905200870FCF797FF77
:1061C0004FF4FA716846F6F796F929F05FF8DC4863
:1061D00090F82300082802D10220FFF7F6FDD949E4
:1061E00009200870CF48418A491C418209F008FB08
:1061F000D54800683C2806D9387820B13D70002188
:10620000C6201EF054FB05F05DFB01282CD10024B4
:1062100004EB840000EB441000EB0809B9F81E0001
:10622000E0B199F82000012802D089F8225017E047
:10623000DFF818B39BF800A004EB4400C449C0EB9E
:10624000C41001EB001120B201F07BFD9BF80000AF
:10625000A0EB0A00401C89F8220001E089F82250D6
:10626000641CA4B2102CD3D329F082FA0022B948BE
:1062700090F8009039E0B84802EB420100EB810150
:10628000B64B887803EBD00300F007041B7806FABE
:1062900004F0034201D0002300E00123002091F824
:1062A00007A05CB2DFF8B8C20AE0CB780344C3EBC6
:1062B000031303EB4303634483F82740401C80B27D
:1062C0008245F2D8002091F808A00AE00B79034437
:1062D000C3EB031303EB4303634483F82740401CE1
:1062E00080B28245F2D8521C92B24A45C3D3DFF83D
:1062F000389299F80000401CC0B289F800001428B8
:1063000016D30024DFF85CA2C4EBC4000AEB8000C3
:10631000807810B120B2FFF7EBFB641CA4B2102C04
:10632000F2D389F80050002009F0BAF909F0F7F922
:1063300099F80200052803D2401C89F8020005E004
:1063400089F80250FFF774FCFFF7E5FC86480178F6
:1063500001B105708548864A01681160056085496C
:106360004FF080500860BFF34F8FBFF36F8F27E768
:106370002DE9F0470646C6EB061000EB40017848D1
:1063800000220C187D4994F924007B4BDFF8F09132
:106390007C4F4FF07E5A01EB86154FF47A78002837
:1063A0000AD002287DD001287CD17748A8613046E8
:1063B000BDE8F047012178E5FFF721FD94F82300BF
:1063C000F8B1AA6184F82520387886426BD230462D
:1063D00022F0B1FB4FF47A71484328F07BFDC4F8FA
:1063E0001E00304622F0A7FB00EB4001C1EBC010BD
:1063F0004FF6FF7101EAC0013046BDE8F04709F0F1
:1064000009B894F92800A0F10C010A2913D917380A
:10641000072806D800EBC00101EB0010185C01282A
:1064200009D0AA613878864224D2304622F083FB14
:10643000E0B101201BE0C5F818A03878864209D2E7
:10644000304622F078FB18B1002084F825001CE0CB
:106450000120FAE7304620F00AFE10F0FF4F03D08B
:10646000002084F8250010E00120FAE7002084F8DD
:1064700025000AE0304620F0FAFD10F0FF4F01D071
:10648000012000E0002084F82500387886420ED2F2
:10649000304622F050FB4FF47A71484328F01AFD41
:1064A00002E034E00FE11DE0C4F81E000BE03046CE
:1064B00020F0DDFD49462CF04CFE2CF0D3FF28F0F7
:1064C00009FDC4F81E0094F8250028B14146304665
:1064D000BDE8F04708F09EBF3046BDE8F047002118
:1064E00008F098BF304620F0C2FD49462CF031FE3E
:1064F0002CF0B8FF28F0EEFCC4F81E0028F0EAFCEF
:106500002CF084FF01463046BDE8F0477BE4FFF7FE
:1065100076FC94F8230020B194F9280009286FD262
:1065200034E03AE04C7D046004020060AED80260C2
:10653000E9030060A2E602604A0200604B020060CC
:1065400062730460F8030060B8030060300000600C
:106550003E480260F0020060F64604606C6504602C
:10656000C840056072FC02601C02006028020060E6
:106570002402006004ED00E05AE40260587F0360EA
:1065800000007A44A702006000007F43DFE800F0CB
:106590007C73767976767976760094F92800A0F186
:1065A0000C010A2914D91738072806D800EBC001B6
:1065B00001EB0010185C01280AD0C5F818A0387843
:1065C000864224D2304622F0B6FAE0B101201BE028
:1065D000AA613878864209D2304622F0ACFA18B166
:1065E000002084F825001DE00120FAE7304620F065
:1065F0003EFD10F0FF4F04D0002084F8250011E08C
:1066000042E00120F9E7002084F825000AE0304646
:1066100020F02DFD10F0FF4F01D0012000E0002000
:1066200084F82500387886420AD2304622F083FA70
:106630004FF47A71484328F04DFCC4F81E000BE07B
:10664000304620F014FD49462CF083FD2CF00AFF63
:1066500028F040FCC4F81E0094F8250028B14146FB
:106660003046BDE8F04708F0D5BE3046BDE8F047FB
:10667000002108F0CFBE7148A8610EE07048A86103
:106680000BE07048A86108E0D4F81E0028F022FC56
:1066900090FBF8F02CF0BAFEA861304620F0E7FC41
:1066A00049462CF056FD2CF0DDFE28F013FCC4F812
:1066B0001E0028F00FFC2CF0A9FE01463046BDE874
:1066C000F047FFF7A0BBAFE470B504465E485F49F2
:1066D000007809780144A14205D85E495C4801EB85
:1066E0008411C8616BE0C4EB041101EB41025A490B
:1066F0005A4E551895F82310D1B184423FD2204606
:1067000022F019FA4FF47A71484328F0E3FBC5F8F8
:106710001E00204622F00FFA00EB4001C1EBC01032
:106720004FF6FF7101EAC001204608F073FE46E013
:1067300084420AD2204622F0FEF94FF47A7148438F
:1067400028F0C8FBC5F81E000BE0204620F08FFCA7
:1067500031462CF0FEFC2CF085FE28F0BBFBC5F882
:106760001E0095F8250028B14FF47A71204608F0F4
:1067700051FE24E00021204608F04CFE1FE008F006
:106780003BFFA04214D9204620F071FC31462CF08A
:10679000E0FC2CF067FE28F09DFBC5F81E0028F0F9
:1067A00099FB2CF033FE01462046FFF72CFB06E058
:1067B000D5F81E0028F08EFB294921F81400BDE809
:1067C00070400AF0C9B830B50020264B214C204D4E
:1067D00004EB80114A6AAA4205D01A5C12B1521E1B
:1067E0001A5400E04D62401CC0B24028F0D330BDC6
:1067F00070B51D4890F85A1000291ED01B4AC1EBF5
:1068000001119068431C9360B0EB810F15D90020F3
:10681000906000240E4D0F4E002106EB841040F8CE
:106820002150491CC9B21029F9D300212046FFF795
:106830003CFB641CE4B2402CEED370BD0000204150
:106840000000C8420000A041A7020060A80200604A
:1068500000007F43587F0360C840056000007A4411
:10686000AED10260B6D001606273046004020060C1
:1068700010B50146F7A02CF0A1FAF749002210B19B
:106880004A80012010BD4888401C80B24880B0F585
:10689000FA6F02D94A80012010BD002010BD3CB51E
:1068A000002301930090C3B28DF80730C0F3072492
:1068B0008DF80640C0F307458DF80550000E8DF8A1
:1068C0000400012A0AD0022A0DD0032A10D0042A7B
:1068D00003D1C8708D704C700B703CBD08704D704A
:1068E0008C70CB703CBD8870CD700C704B703CBD13
:1068F00048700D70CC708B703CBD38B50023009390
:10690000CBB2C1F30724C1F30745090E042A06D010
:10691000032A0DD0022A14D0012A1BD022E08DF8C0
:1069200000308DF801408DF802508DF8031019E009
:106930008DF800508DF801108DF802308DF803406D
:1069400010E08DF800408DF801308DF802108DF8C0
:10695000035007E08DF800108DF801508DF80240CB
:106960008DF803309DF800104FF6FF7202EA012106
:106970009DF8012011439DF8022042EA01219DF873
:10698000032042EA0121016038BD4178007841EAE4
:10699000002070470178427841EA02218278C0786D
:1069A000120442EA006008437047AC49AC4A0868E8
:1069B000904201D800207047001F086000687047AF
:1069C00070B50546A74A106810F8024B10600846DB
:1069D00000F092F84FF47A7190FBF1F004EB44016F
:1069E000A14A01EBC4011144B1F80910814207DD4D
:1069F000002805DB9D4951F8241051F8200028603B
:106A000070BD0246B2F901301278832A0AD0842A76
:106A100008D0852A08D0862A03D1C8564FF47A7147
:106A200048437047C8587047C85E4FF47A7148436E
:106A300070472DE9F04103468D4E00273760894DA0
:106A40002A681478A4F18200042808D8D21C2A608D
:106A500003B11F602868BDE8F041C01ED1E781483E
:106A60000068401C9C2C06D09E2C15D09D2C32D04A
:106A70000020BDE8F08192780C2A08D07C4928607B
:106A800003F040FE2868801C28603068F1E7286029
:106A90007748FFF795FFF8E792780C2A0AD028602C
:106AA00000231A46724904F0F1FD2868401D286051
:106AB0003068DEE70446601D2860084600F01CF8D8
:106AC0004FF47A7190FBF1F000231A466849204692
:106AD00004F0DCFDECE7521D2A6003B11F6028685A
:106AE00050F8040CC5E75D4A5D4B1168503399427C
:106AF00001D201C1116070472DE9F14FA0B0DFF85C
:106B000064A1DAF80000007882381C2805D800203B
:106B10002099FFF78EFFFFF7E6FF564C564E4FF0D9
:106B20000108534FDFF854914FF47A75B0E2DAF868
:106B3000000010F8011BCAF8000056297ED047DC7F
:106B40003B297CD027DC31297AD016DC072978D084
:106B50000ADCA1F1020105290ED2DFE811F06E076F
:106B600075077C078F07960708296BD010296AD014
:106B70002929DBD02C29D9D0F8E332390929FBD2D5
:106B8000DFE811F0CF023704220717075E03BF05C5
:106B9000E505480391063C391829EDD2DFE811F0EC
:106BA000AF03CA0379037802A606A606F4072605F2
:106BB000E603EA07F007E703E603E603E6033B071D
:106BC0002A07CF02E502E60378021208FE061F0735
:106BD0007A297DD028DCA1F157012329CCD2DFE826
:106BE00011F00C063706C503C503C503C503C5036D
:106BF000C503C50328025802C503C503C503A30086
:106C00004E01D600F5009700C50368007F004002E2
:106C10001002C503C503700288027201AB018E0128
:106C20000002C503C503E401C7296ED031DCC229C7
:106C30006CD025DC7B296AD0A42905E0F8E3F8E3D1
:106C4000F8E3F8E3F8E3F8E37ED0A5297DD0C12985
:106C500092D1F3E301FFFE001C020060B00200606D
:106C600040E40360AC02006058900360D8E1036028
:106C7000C0020060C4020060C8020060101800601A
:106C8000C3297CD0C4297BD0C5297AD0C629DFD1BD
:106C9000FEE3C8390B29A1D2DFE811F02E07350732
:106CA0003C0743074A0768030E04660468037D0235
:106CB0009702FFF77AFE2060FFF777FE30602068CA
:106CC00028F008F92060306828F004F9306000E00E
:106CD0004FE12168084428F0FDF8FFF704FF25E79D
:106CE000FFF763FE2060FFF760FE3060206828F049
:106CF000F1F82060306828F0EDF830602168401A23
:106D000028F0E8F8FFF7EFFE10E7FDE3FDE397E07A
:106D1000FFF74BFE206028F0DDF82060404228F0AD
:106D2000D9F8FFF7E0FE01E7FFF73FFE3060FFF71D
:106D30003CFE206028F0CEF82060306828F0CAF8C9
:106D4000306090FBF5F001E085E293E203B2206849
:106D50000246012B12DD00215B1E0DE090FBF5FCCD
:106D600005FB1C0C0CFB02FC9CFBF5FC90FBF5F0FE
:106D700000FB02C0491C09B29942EFDB02E0F0E3DC
:106D8000F0E3F0E328F0A6F8FFF7ADFECEE6FFF75C
:106D90000CFE3060FFF709FE206028F09BF82060B1
:106DA000306828F097F801463060206890FBF5F2D3
:106DB00005FB12024A4392FBF5F290FBF5F000FB53
:106DC000012028F087F8FFF78EFEAFE6FFF7EDFD14
:106DD0003060FFF7EAFD206028F07CF82060306822
:106DE00028F078F88246306020B350462CF00EFB35
:106DF000834620681F9090FBFAF10AFB11002CF0EB
:106E000005FB59462CF0D7F9FD492CF0A2F9834631
:106E10001F984FF47A7190FBFAF048432CF0F6FA81
:106E200059462CF03EF92CF01DFB28F053F8FFF7E3
:106E30005AFE7BE6284628F04DF8FFF754FE75E62B
:106E4000FFF7B3FD3060FFF7B0FD206028F042F897
:106E50002060306828F03EF8306050B1216891FB26
:106E6000F0F028F037F84FF47A714843FFF73BFE13
:106E70005CE6284628F02EF8FFF735FE56E6FFF7C9
:106E800094FD3060FFF791FD206028F023F820602A
:106E9000306828F01FF8306078B1216891FBF0F27B
:106EA00000FB121090FBF5F020604FF47A7148431C
:106EB00028F010F8FFF717FE38E6284628F00AF801
:106EC000FFF711FE32E6FFF770FD3060FFF76DFD52
:106ED000206027F0FFFF2060306827F0FBFF90FB69
:106EE000F5F03060216891FBF5F1216048404FF4E6
:106EF0007A71484327F0EEFFFFF7F5FD16E6FFF73E
:106F000054FD2060FFF751FD3060206827F0E2FF5C
:106F10002060306827F0DEFF30602168014305D033
:106F2000284627F0D7FFFFF7DEFDFFE5002027F01A
:106F3000D1FFFFF7D8FDF9E5FFF737FD2060FFF738
:106F400034FD3060206827F0C5FF2060306827F0EE
:106F5000C1FF3060216831B128B1284627F0BAFF5F
:106F6000FFF7C1FDE2E5002027F0B4FFFFF7BBFD0E
:106F7000DCE5FFF71AFD2060FFF717FD30602068A1
:106F800027F0A8FF90FBF5F02060306827F0A2FF03
:106F900090FBF5F03060216801434FF47A7048436C
:106FA00027F098FFFFF79FFDC0E5FFF7FEFC20608C
:106FB000FFF7FBFC3060206827F08CFF90FBF5F0BA
:106FC0002060306827F086FF90FBF5F03060216884
:106FD00001404FF47A70484327F07CFFFFF783FDB0
:106FE000A4E5FFF7E2FC206027F074FF206030B1D9
:106FF0000020206027F06EFFFFF775FD96E5012069
:10700000F7E7FFF7D2FC3060FFF7CFFC206027F0F6
:1070100061FF2060306827F05DFF306021688142A9
:1070200001DD012000E0002027F054FFFFF75BFDA9
:107030007CE5FFF7BAFC3060FFF7B7FC206027F073
:1070400049FF2060306827F045FF306021688142A9
:1070500001DB012000E0002027F03CFFFFF743FDAB
:1070600064E5FFF7A2FC3060FFF79FFC206027F08B
:1070700031FF2060306827F02DFF306021688142A9
:1070800001DA012000E0002027F024FFFFF72BFDAC
:1070900011E2FFF78AFC3060FFF787FC206027F0E1
:1070A00019FF2060306827F015FF306021688142A9
:1070B00001DC012000E0002027F00CFFFFF713FDAA
:1070C000F9E1FFF772FC3060FFF76FFC206027F0FA
:1070D00001FF2060306827F0FDFE306021688142AA
:1070E00001D1012000E0002027F0F4FEFFF7FBFCB7
:1070F000E1E1FFF75AFC3060FFF757FC206027F012
:10710000E9FE2060306827F0E5FE306021688142AA
:1071100001D0012000E0002027F0DCFEFFF7E3FCB7
:10712000C9E1FFF742FC206027F0D4FE2060002870
:1071300000DA404227F0CEFEFFF7D5FCBBE1FFF7B7
:1071400034FC20602CF070F900222E4B2CF0EFF86C
:107150002EF0A6FA2CF0DFF929492BF0FAFF2CF0DB
:1071600081F92060FFF7BFFCA5E1FFF71EFC20605E
:107170002CF05AF90022234B2CF0D9F82EF026F9E6
:107180002CF0C9F91E492BF0E4FF2CF06BF92060BC
:10719000FFF7A9FC8FE1FFF708FC20602CF044F911
:1071A000194A1A4B2CF051F80022194B2CF0BFF859
:1071B0002EF05AFC2CF0AFF911492BF0CAFF2CF03D
:1071C00051F92060FFF78FFC75E1FFF7EEFB2060BF
:1071D0002CF02AF90C4A0D4B2CF037F800220C4BFE
:1071E0002CF0A5F82EF0A4F82CF095F904492BF01A
:1071F000B0FF2CF037F92060FFF775FC5BE1000071
:1072000000007A4400408F406E861BF0F92109404F
:1072100000F90541FFF7C9FB20602CF005F90022B9
:10722000FE4B2CF084F82EF06FFC2CF074F9FC4926
:107230002BF08FFF2CF016F92060FFF754FC3AE199
:10724000FFF7B3FB90FBF5F04FF47A7148432060F1
:10725000FFF749FC2FE110F8030C402807D2C0EBE0
:10726000C00101EB0011EF4800EB41001E90FFF759
:107270009CFB20E110F8030C402807D2C0EBC001B2
:1072800001EB0011E74800EB41001E90FFF78DFB7A
:1072900011E1E54A117841B1FFF787FB27F01AFEAB
:1072A00083460020FFF71FFC21E001689068A1EBF6
:1072B000000BBBF1000F05DDFFF777FB0020FFF7A8
:1072C00012FC14E0D9495844884208D1FFF76DFBFD
:1072D00027F000FE83460020FFF705FC07E0FFF7DC
:1072E00064FB27F0F7FD83460120FFF7FCFBDAF88B
:1072F0000000C0F800B0001DCAF80000DBE0B0F9E3
:10730000000027F0E8FDCA4909680844C949086037
:1073100010F8011C29B1006827F0DCFDFFF7E3FB42
:1073200002E00020FFF7DFFBDAF80000801CCAF85B
:107330000000C0E0B0F9000027F0CDFD0146BC48D8
:1073400000680844BB49086010F8011C19B100200E
:10735000FFF7C9FB04E0006827F0BCFDFFF7C3FBA3
:10736000DAF80000801CCAF80000A4E0FEE3FFF792
:107370001CFB90FBF5F000B2AF490978884203D1BD
:107380000120FFF7B0FB96E0C11700EB5171AB4B4A
:10739000CA1021F007019A5C431A08FA03F10A4265
:1073A00003D00120FFF79FFB85E04FF0000ADFF8D4
:1073B00094B2A34B9BF8002011E02B2101FB0A3172
:1073C00091F804C0844502D0497A814203D101205A
:1073D000FFF789FB05E00AF1010A0FFA8AFA9245E4
:1073E000EBDB9BF80000824588D10020FFF77BFB98
:1073F00061E010F801BBCAF8000000203860824646
:107400000CE0FFF7D2FA206027F064FD20603968B5
:10741000084438600AF1010A0FFA8AFADA45F0DB0B
:10742000386890FBFBF027F055FDFFF75CFBF3E3BA
:10743000B3E184E3D6E3F4E2F9E200E02CE310F8F0
:1074400001BBCAF8000000203860824623E0FFF745
:10745000ACFA206027F03EFD2060396801443960B5
:10746000BAF1000F03D190FBF5F1774A1171BAF12F
:10747000010F03D190FBF5F1734A9170BAF1020F3D
:1074800003D190FBF5F0704908800AF1010A00E091
:1074900024E30FFA8AFADA45D9DBDFF8ACA1ABF1C5
:1074A000020B8AF803B014F0D4FFDAF80E0027F0CC
:1074B00011FDFFF718FBAFE3514610F801AB086070
:1074C000AAF10302172A93D200230DF13C0B0BE023
:1074D000FFF76BFA90FBF5F02060AAEB0301491E61
:1074E0002BF811005B1C1BB25345F1DB57480078A9
:1074F0008DF87200BDF83C008DF87300BDF83E00B9
:107500008DF87000010A01E0EFE2CBE2032202EB0A
:1075100041118DF87110802101EBD0208DF874009D
:10752000AAF1020A0AF0FF0C002002AA0AE0811C5C
:107530003BF811100B0A02F8103002EB40035970AF
:10754000401C00B25045F2DB4FEA4C02012302A975
:107550001CA8CDF8008003F09FFC2846FFF7C3FA73
:107560005AE3A6E2ACE2B2E210F801BBCAF80000AE
:10757000ABF1030017289ED200230DF13C0A0BE06B
:10758000FFF713FA90FBF5F02060ABEB0301491E07
:107590002AF811005B1C1BB25B45F1DB2B4800781D
:1075A0008DF87200BDF83C008DF87300BDF83E0008
:1075B0008DF87000010A182202EB41118DF871104C
:1075C000802101EBD0208DF87400ABF1020B0BF0A1
:1075D000FF00420001230AF104011CA8CDF800803D
:1075E00003F05AFC2846FFF77EFA15E310F801BBBA
:1075F000CAF80000FFF7D9F990FBF5F083B2FFF766
:10760000D4F990FBF5F000F0FF0AFFF7CEF990FBFC
:10761000F5F0BBF1030F1ED0002019E000408F40B1
:1076200000007A44083505601C020060EB32A4F8C3
:10763000B4020060CC020060AB0200606C650460C4
:107640002CCE036062020060507304605B02006035
:10765000FFF749FAE0E2FF2820D80BB15B1E237048
:10766000BAF1010F14D0BAF1020F14D003226270E4
:10767000A070E0700021217100230122F949204609
:1076800004F004F8284627F025FCFFF72CFAC3E2A3
:1076900002226270ECE784F80180E9E72370AAF126
:1076A000040ABAF1060F16D2DFE80AF00306090C45
:1076B0000F121D22627010E0152262700DE01E2272
:1076C00062700AE01F22627007E01C22627004E010
:1076D0001622627001E01C226270E070020AA27041
:1076E000C0F306408030207100230122DD4920468E
:1076F00003F0CCFF4FF4FA6027F0ECFBFFF7F3F94F
:107700008AE210F801BBCAF80000FFF74EF927F033
:10771000E1FB38604FF0000AABF1010B0FE0FFF71F
:1077200044F9206027F0D6FB2060CF490860396813
:10773000884200DD38600AF1010A0FFA8AFADA4558
:10774000EDDB386827F0C6FBFFF7CDF964E210F8EF
:1077500001BBCAF80000FFF728F927F0BBFB38602F
:107760004FF0000AABF1010B0FE0FFF71EF92060AC
:1077700027F0B0FB2060BC4908603968884200DA15
:1077800038600AF1010A0FFA8AFADA45EDDB386847
:1077900027F0A0FBFFF7A7F93EE2FFF706F927F075
:1077A00099FB90FBF5F00FFA80FAFFF7FEF827F04F
:1077B00091FB90FBF5F001B24FF47A60824500DD59
:1077C0008246BAF1000F01DA4FF0000A5046491E16
:1077D000C1EBC102A54901EB8201CA7C2AB9087636
:1077E000C21700EB1262120ACA754FF47A7148434D
:1077F00027F070FBFFF777F90EE2FFF7D6F827F0D6
:1078000069FB0A2190FBF1F03860FFF7CEF827F012
:1078100061FB90FBF5F001B23868002801DA002026
:1078200038603868C82801DDC82038603868491ECB
:10783000C1EBC1028D4901EB8201CA7C02B9C87655
:1078400000EB8000400027F045FBFFF74CF9E3E137
:10785000FFF7ABF827F03EFB90FBF5F00FFA80FA4C
:10786000FFF7A3F827F036FB90FBF5F001B2BAF171
:10787000FF0F01DD4FF0FF0ABAF1000F01DA4FF000
:10788000000A5046491EC1EBC102784901EB820152
:10789000CA7C02B948764FF47A71484327F01AFB44
:1078A000FFF721F9B8E1FFF780F890FBF5F02060D1
:1078B000FFF77BF890FBF5F030602168012901DAD1
:1078C000C4F800802168052901DD052121602178A7
:1078D0001331CAB201B2104627F01CFC64492BF0E8
:1078E00038FC2BF0BFFDFFF7FEF895E1FFF75DF8E0
:1078F000206027F0EFFA2060FFF757F8306027F09C
:10790000E9FA02463060206890FBF5F0401E01B2B3
:1079100099F80400401E002800DA0620DAF800304A
:1079200013F8013C402B0CD008EB410109B2AA42EC
:1079300003DB092901D2002806DC0020FFF7D3F879
:107940006AE1490009B2F2E792FBF5F392FBF5F226
:107950005B1EDFF820C103EBC3030CEB0313521EC5
:1079600003EB001302EBC2020CEB021203EB410328
:1079700002EB00105B7810F811004FF4616A03FB12
:107980000AF3C0EB001003EB800038604FF47A710B
:10799000484327F09FFAFFF7A6F83DE199F8030066
:1079A0004FF47A714843386027F094FAFFF79BF858
:1079B00032E199F804004FF47A714843386027F0B7
:1079C00089FAFFF790F827E1B9F807004FF47A71C8
:1079D0004843386027F07EFAFFF785F81CE199F8F4
:1079E00005004FF47A714843386027F073FAFFF7C7
:1079F0007AF811E12048417829B1002027F06AFA8D
:107A0000FFF771F808E180F80180012027F062FAA1
:107A1000FFF769F800E1012027F05CFAFFF763F84F
:107A2000FAE0002027F056FAFFF75DF8F4E0284668
:107A300027F050FAFFF757F8EEE04FF4FA6027F01E
:107A400049FAFFF750F8E7E040F6B83027F042FA7D
:107A5000FFF749F8E0E04FF47A6027F03BFAFFF7D0
:107A600042F8D9E0C0020060BC02006072FC026013
:107A700000401C46AC4F03601C02006041F288309D
:107A800027F028FAFFF72FF8C6E041F2707027F0D0
:107A900021FAFFF728F8BFE0284627F01BFAFFF786
:107AA00022F8B9E04FF4FA6027F014FAFFF71BF858
:107AB000B2E040F6B83027F00DFAFFF714F8ABE06B
:107AC0004FF47A6027F006FAFFF70DF8A4E041F2D0
:107AD000883027F0FFF9FFF706F89DE041F270705B
:107AE00027F0F8F9FEF7FFFF96E041F6583027F04F
:107AF000F1F9FEF7F8FF8FE04FF4FA5027F0EAF9BA
:107B0000FEF7F1FF88E042F2283027F0E3F9FEF7B4
:107B1000EAFF81E042F2107027F0DCF9FEF7E3FFA4
:107B20007AE042F6F82027F0D5F9FEF7DCFF73E0A3
:107B300042F6E06027F0CEF9FEF7D5FF6CE099F849
:107B40000200FE4940F25372484399F80110514334
:107B500000EB411199F8000000EB4002C2EBC010AD
:107B600001EBC000386027F0B5F900E04BE0FEF70C
:107B7000BAFF51E0012027F0ADF9FEF7B4FF4BE06A
:107B80000020FEF7B0FF47E00020ED4A00EB0011B7
:107B900001EB410102EB4101CB79012B01D1497A83
:107BA00039B1401CC0B21028F0D30020FEF79BFF73
:107BB00032E0012027F08EF9FEF795FF21B0012079
:107BC000BDE8F08FFEF7F1FE90FBF5F0FEF7EDFE5D
:107BD00090FBF5F0FEF7E9FE90FBF5F0D948FEF7D3
:107BE00082FF19E0017882390A2906D8B0F901002C
:107BF0004FF47A714843FEF776FFDAF80000C01CB4
:107C0000CAF8000008E0401ECAF8000000202099D1
:107C1000FEF70FFFFEF767FFDFF82CA3DAF800008E
:107C200090F90000FEF724FE00283EF480AF514694
:107C300008680278FF2A01D1401C0860FEF7B5FEF3
:107C400021B0BDE8F04F27F045B910B5B0F90130CB
:107C5000B3F5FA7F0DD8007883280BD0842809D09B
:107C60004FF47A74852807D0862802D191FBF4F06E
:107C7000D05410BDD15010BD91FBF4F0D05210BDC6
:107C8000B24BB34A1968914202D20A1D1A600860C9
:107C90007047AE49AE4A0868503A904201D8002079
:107CA0007047001F086000687047F0B5059DB0F987
:107CB0000170EE1936F904CCBCF1000F0BD0002A8C
:107CC00007DD944505DB002B03DD36F902CC9C452E
:107CD00009DA0120F0BD002B03DD36F902CC9C450A
:107CE00001DA0120F0BD0078882806D0892804D068
:107CF0008A2804D08B2805D103E0042402E0022462
:107D000000E0012436F8026C521E5643F218521E4F
:107D100062433A4412B2882808D0892806D04FF42A
:107D20007A738A2804D08B2809D105E0A95006E08F
:107D300091FBF3F0A85202E091FBF3F0A85400206D
:107D4000F0BD2DE9F04F97B083460F4681480026DD
:107D5000354606707C4C384627607D497B4A503951
:107D6000116000880E90BDF9380027F0B4F80E902D
:107D70001FFA80F9B8B321680844401D20600088CC
:107D80000E90BDF9380027F0A6F80E901FFA80F883
:107D900021688A1C05920144891C2160642801DD48
:107DA00005200E9008880E90BDF9380027F093F852
:107DB0000E902168891C21600A180892664A116099
:107DC00009EB080108440BEB8B01644A01EB4B11F2
:107DD0001144C883DFF88881A8F80460DFF884A123
:107DE0004FF001093AE0FFE7002017B0E8E60598F8
:107DF000FEF782FE02465C48026020682346014688
:107E0000401CCAF800009AB109780246186049B1CE
:107E100098F8001001B106600168D8F808201144F4
:107E2000016018E002F8019CDAF80000066012E038
:107E300009780246186029B102F8016CDAF80000EE
:107E4000066008E098F8001001B106600168D8F8F3
:107E50000820114401601868001D18602168089806
:107E6000814207D2B8F80400411CA8F80410B0F50C
:107E7000FA6FBCD3B8F804100BF101001690B1F5FD
:107E8000FA6F06D31698C1B20020FDF76DFC0020F2
:107E9000ABE73846A2462760044600880E90BDF93D
:107EA000380027F018F801460E901590A41CDAF857
:107EB0000000801CCAF8000042185178927801EB4B
:107EC000022CBCF5FA6F01D900208EE700EB0220EE
:107ED0000844CAF800000020A8F8040023480068FD
:107EE00004900BF1010B0FFA8BF651E01F4A126858
:107EF000049BD21AB2F5FA7F01D9002075E74FF042
:107F0000000BCDF82CB015B1012840D007E00128B6
:107F100002D04FF0FF3068E7C91CCAF80010DAF849
:107F2000000010F8011BCAF800002329DDD030DC66
:107F3000A1F108011A29D8D21AE0000080EE36001B
:107F40001ADC026018FCFFFFAC020060B0020060A7
:107F500090E40360D0020060B4020060A2E6026018
:107F60001C020060CC020060B802006030000060BB
:107F7000DFE801F032320EEF0EEEED0EECEBEAE947
:107F8000E8E70EFF0E0EF90E3232E50E0EE4002584
:107F9000E9E340296FD00ADCA1F125010A29A4D226
:107FA000DFE801F01A1ACBCB1AD1FC1A1A1A84296D
:107FB00008D008DC41297DD043297CD0592994D0B0
:107FC000832992D1CFE0852905D0862903D087293E
:107FD00001D08A2989D1C6E010F8011C4FF00008B1
:107FE00009290FD008290DD001220A920278A2F1A6
:107FF00082030A2B09D84FF001080746C01CCAF8B3
:1080000000001BE000220A92F0E79C2A02D09E2A80
:1080100009D013E04FF09C08B0F80120C01C129268
:10802000CAF800000AE0401C4FF09E080268109257
:1080300002798DF84420401DCAF800001C2903D0A5
:108040002D2901D0252902D14FF47A7007901D29DE
:1080500003D02E2901D0262901D1CDF81CB0092941
:108060000AD0292915D02C292CD0082944D0B8F1C0
:10807000010F50D054E083E00598FEF73DFD0790D6
:10808000B8F1010F4CD101463846059AFFF7DDFDE6
:1080900046E0012006900598FEF72EFD82460598E1
:1080A000FEF72AFD07904FF47A719AFBF1F30599D8
:1080B000009101E0CAE0ACE101463846069AFFF7BC
:1080C000F4FD2DE00598FEF717FD06900598FEF7E4
:1080D00013FD82460598FEF70FFD07904FF47A7165
:1080E000069A9AFBF1F392FBF1F205990091014691
:1080F0003846FFF7DAFD13E00598FEF7FDFC014670
:108100004FF47A7091FBF0F040B20A900598FEF7B8
:10811000F3FC079004E03846059A0799FFF795FDB0
:10812000B8F19C0F03D0B8F19E0F06D112E00023E6
:1081300007A912A80A9A02F021FC14E345E1F0E233
:1081400017E018E04EE075E0AAE260E2DDE240E20E
:1081500001E2D6E1CDF800B0002307A910A80A9AE1
:1081600002F09AFEFFE210F8011B0844CAF8000072
:10817000F9E2012039E6FFF78CFDCAF80000F2E2CF
:108180000598FEF7B9FC0FFA80F8B8F1010F09DB8A
:10819000DAF800004178414504DB09E033E0401C97
:1081A000CAF80000DAF8000001780129C5D0F6E726
:1081B0000278142A04D100EB4100801CFFF760FD17
:1081C000DAF80000A8F1010800EB480040880D90A3
:1081D000BDF9340026F07FFE0D902044801ECAF8C1
:1081E0000000C0E200F1020800880D90BDF93400E3
:1081F00026F071FE0D902044801ECAF80000404613
:10820000FFF73EFDAFE2DFF8348498F8001069B163
:1082100000880D90BDF9340026F05DFE0D902044DD
:10822000801ECAF8000088F800B09CE2801CCAF8E2
:10823000000098E200880D90BDF9340026F04BFE56
:108240000D902044801ECAF800008CE21E226D2191
:108250002AF0D3FD071E02D06D200D9009E0F848EA
:108260001E226E2100682AF0C8FD071E01D06E2074
:108270000D90FF2038700598FEF73EFC804605986B
:10828000FEF73AFC82460598FEF736FC0790EC486C
:10829000016811F8010B0C90E9480160E9480C9A5B
:1082A0002AF056FDE7490C9801F800B0E44801684F
:1082B0000C980844E24910F8012B0860F2B3BDF9AC
:1082C000341014916D291AD107995144414502DAAD
:1082D00000F801BC13E000F8019CDC48DA490023F7
:1082E00090F90020DA4890F90000CDE90002CDE9CC
:1082F000021BD84831460278D248FDF705F8149899
:108300006E285ED10798AAEB0000404504DDCC48FA
:10831000006800F801BC54E0C948006800F8019CFE
:10832000CA48C949002390F90020C94890F90000C3
:10833000CDE90002CDE9021BC64800E005E0027865
:108340003146C048FCF7E0FF3BE0BDF93410139123
:108350006D2918D1D04516DA00F8019CB74880F88D
:108360000090BA48B849002390F90020B84890F925
:108370000000CDE90002CDE9021BB6483146027883
:10838000B048FCF7C1FF13986E281AD1D04518DD0C
:10839000AB48006800F8019CA84880F80090AB4802
:1083A000A949002390F90020A94890F90000CDE9DF
:1083B0000002CDE9021BA74831460278A148FCF72C
:1083C000A3FFBDF834003870CDE10178FF2902D059
:1083D0009D4B9E4A12E09E4940220A70401CCAF8FA
:1083E0000000C0E192F9001010F801CB01F1010882
:1083F00082F8008003F801C0CAF80000DAF8000033
:1084000001780029EED1DAF80000401CCAF800001B
:10841000A9E18A4880F800B00598FEF76DFB8E4907
:108420000860DAF800000068079026F053FD079016
:10843000DAF80010091D11F8018BCAF800108648FF
:108440000068A0B342467F482AF082FC7D4800F8CD
:1084500008B0DAF800004044CAF800007F490A7802
:108460000AB1079A02600068002806DD8968401A90
:1084700026F030FDDAF80010086000283BDC734974
:108480007148002391F90020714991F90010CDE95C
:10849000020BCDE900126F48314602786948FCF7BB
:1084A00033FFC0B238B3654880F8009023E0FFE79F
:1084B00001EB08000068002811DC424661482AF000
:1084C00047FC604800F808B06248314602785D48D1
:1084D000FDF786F96248017841F001010170DAF890
:1084E00000004044CAF80000079826F0F3FC07900B
:1084F000DAF800100860DAF80000001DCAF8000081
:1085000031E10746C01CCAF800000598FEF7F4FAEE
:1085100083460598FEF7F0FA80460598FEF7ECFAD8
:10852000D8450ADB59463846059AFFF78EFBDAF83C
:108530000000801CCAF8000015E1DAF8000000888D
:108540000B90BDF92C0026F0C6FC0B902044801E39
:10855000CAF8000007E100880B90BDF92C0026F056
:10856000BAFC0B902718BF1CF81CCAF8000005982D
:10857000FEF7C2FA0598FEF7BFFA0F900598FEF7CE
:10858000BBFA8346DAF80080CAF80070002005992B
:10859000FEF74FFA00EB0B0107913846059AFFF7FB
:1085A00054FBCAF8008007990F98814204DC08F157
:1085B0000208CAF80080D6E0B8F800000B90BDF9B8
:1085C0002C0026F088FC0B902044801ECAF8000086
:1085D000C9E001250598FEF78FFA1F49086028B108
:1085E000DAF80000801CCAF80000BCE0DAF80000ED
:1085F000B0F9000026F06FFC2044801ECAF800008D
:108600000078012801D0FE2800D10025ABE00598B4
:10861000FEF772FA1049086078B1DAF8000010F835
:10862000011BCAF80000E9B1B0F9000026F053FCC4
:108630002044801ECAF8000028E019E0D002006043
:10864000AC02006090E40360D3020060D2020060DC
:10865000D1020060AB020060B80200601C02006042
:10866000AA02006000F8019C801CCAF800000DE01E
:10867000DAF8000000F801BBCAF80000B0F9000009
:1086800026F029FC2044801ECAF800000125DAF8F3
:1086900000000078012801D0FE2864D1002562E0A6
:1086A0000598FEF729FA54490860B0B1DAF80000DD
:1086B00000F8019BCAF80000B0F9000026F00BFC9E
:1086C0002044801ECAF800000125DAF80000007876
:1086D000012818D0FE2846D115E0DAF8000010F87D
:1086E000011BCAF8000029B100F801BC801CCAF8BF
:1086F0000000E9E7B0F9000026F0EDFB2044801E01
:10870000CAF80000E0E700252DE0401CCAF8000090
:10871000B0F9000026F0DFFB2044801ECAF80000FC
:1087200021E0011F09910178A12939D00598FEF7B0
:10873000E3F98046DAF800000068079026F0CAFBEB
:108740002E49896808440790404539D9DAF8000075
:10875000C0F800B015982044A0F801B0DAF8000085
:10876000001DCAF80000DFF898A0DAF800100878B9
:10877000FE2809D0214B9A8802F1010CA3F804C00D
:10878000B2F5FA6FFFF4B2AB1C488088B0F5FA6F0F
:10879000FFF4F0AC1698C1B20120FCF7E5FFE9E464
:1087A000401CCAF80000006826F094FB4FF47A7170
:1087B00000FB01F8DAF80000001DCAF80000B9E774
:1087C000079826F087FB07900D490968086009980B
:1087D000001B00B226F07FFB15992144A1F801008F
:1087E0000120C7E4006800F52A01AB3101D0002068
:1087F0007047012070470000B80200601C02006052
:10880000AC0200602DE9F04107460C465D344FF4A0
:108810006160A17841436078C0EB001001EB8000FB
:1088200021780E1860795D3C00EB8002732007FB15
:1088300000F1FD4800EBC10504F1090128462AF0CA
:1088400087FA463514F85D0FA8706078E870A07854
:1088500028712F7060796870463D06B9012606F0D0
:1088600048F9B0FBF6F0401C704345F85A0F002061
:10887000A880BDE8F08170B506460C46732394F8D5
:10888000611094F86200091A01EB810200EB80008C
:108890000119012000EB46005843E34B093103EB7B
:1088A000800528462AF054FA05F8466F14F8610F3F
:1088B0006178401A68700020288370BD2DE9F04F60
:1088C00085B0054688464FF4616098F85F104143D3
:1088D00098F85E00C0EB001001EB800098F85D1086
:1088E0000844D8F864100844C8F864004FF0000940
:1088F000CD4905EBC502A1F5165002EB051200EBC0
:1089000042177320684301EBC0046AE009EB890059
:1089100026180396B4F85E0018B906F0EAF8C4F811
:108920005A0014F8461F208B07EB001001703178B5
:10893000417171788171B178C171F17801723179C9
:10894000417206F0D6F88DF80400824606F0D1F8A0
:10895000C0F307208DF80500049006F0CAF8C0F3B4
:10896000074B8DF806B006F0C4F8000E8DF807002E
:1089700000EB0B210498020402EB0A600144208BF7
:10898000463C07EB0010C0F8011040F60D21C181F4
:108990000023012202A9304602F078FE01281ED1F0
:1089A000029826F097FAB4F85E1007EB011C8DF8D8
:1089B0000400C0F307228DF80520C0F307438DF8AB
:1089C0000630060E8DF80760120406EB032302EB57
:1089D00000601844CCF80A00491CA4F85E1009F1A4
:1089E000010994F84700484590DCB4F85E6094F8BB
:1089F00047003044192809D9DFF830924FF0000AB7
:108A000099F8000002280BD0A4F85EA005B0BDE8DC
:108A1000F08F07EB0610102200212AF099F9761C3E
:108A2000192EF6DB824C4FF4C871012254F8350040
:108A3000C3B24B43C0F30B20294619F0FDFD0128BA
:108A400046D199F80000022842D105F1B3006946E9
:108A500006461BF01DFF9DF8000054F8351000F08D
:108A60000F02C1F303418A4206D000F0F000014337
:108A7000009130461BF01BFF34F83500C0F307218E
:108A8000542000EB450007461BF011FF552000EB7A
:108A9000450014F8351081461BF009FF54F83500E5
:108AA0006449884203D2401C44F8350010E038463F
:108AB00000211BF0FCFE484600211BF0F8FE9DF84B
:108AC000000000F0F00130461BF0F1FE44F835A044
:108AD00041462846FFF796FE98E72DE9F34F8BB005
:108AE000804652480078022803D153484188491CE7
:108AF0004180012505EB480973204B4909FB00F033
:108B000001EB8004B4F85E0018B905F0F2FFC4F878
:108B10005A000027012000EB4800484900EBC00242
:108B200002EB001040F60D2A01EB0016CEE107EB38
:108B3000870025180023012204A9284602F0A6FD7B
:108B4000012870D1039505F0D4FF3D4951F8281054
:108B5000FA31884276D394F84700401EB84204D1D7
:108B600005F0C7FF364941F82800B4F85E0094F8D4
:108B7000461006EB00100170297841716978817107
:108B8000A978C171E978017229794172049826F0B7
:108B9000A1F988B35E340BFA07FBA08840EA0B000A
:108BA000A08005F0A6FF8DF80800834605F0A1FF20
:108BB000C0F307258DF8095005F09BFFC0F307406F
:108BC0008DF80A000A9005F094FF010E8DF80B1045
:108BD0000A982A0401EB0B6102EB0020014434F8EF
:108BE0005E0906EB0010C0F801104FF08071C0F86C
:108BF0000A10A0F80EA03AE0FFE705F07AFF8DF822
:108C00000800834605F075FFC0F307258DF809506D
:108C100005F06FFFC0F307408DF80A00099005F0DA
:108C200068FF010E0FE050E180F80160A0040060D1
:108C300010D10160FFFF0F002C02006000D3016023
:108C4000AC23026019E08DF80B1009982A0401EB9F
:108C50000B6102EB00200144B4F85E0006EB00104B
:108C6000C0F801100021C0F80A10A0F80EA0B4F856
:108C70005E00401CA4F85E0027E14FF0010BB4F841
:108C800062000BFA07FB1BEA000F7DD0049826F068
:108C900021F950B1B4F86210012041EA0B01A4F8A7
:108CA0006210FE490A78E2B30FE14634A08B20EA55
:108CB0000B00A083218B207806EB0111087005F0D2
:108CC00018FF8DF80800834605F013FFC0F3072551
:108CD0008DF8095005F00DFFC0F307408DF80A002C
:108CE000089005F006FF010E8DF80B1008982A0475
:108CF00002EB002001EB0B61228B014406EB02101A
:108D0000C0F80110A0F80EA003990B7843714B78BE
:108D100083718B78C371CB7803720979417200211A
:108D200000E005E0C0F80A10521C2283463CCCE06B
:108D3000087014F8461F208B06EB0010017029788C
:108D4000417169788171A978C171E97801722979D5
:108D5000417205F0CEFE8DF80800834605F0C9FE8D
:108D6000C0F307258DF8095005F0C3FEC0F3074096
:108D70008DF80A00079005F0BCFE010E8DF80B106F
:108D800001EB0B612A0400E012E0079802EB0020DF
:108D90000A18218B06EB0110C0F801204FF08072F9
:108DA000C0F80A20A0F80EA0491C2183463C8CE0A4
:108DB000049826F08FF8E8B34634A08B40EA0B0005
:108DC000A083208B217806EB001001702978417177
:108DD00069788171A978C171E97801722979417244
:108DE00005F087FE8DF80800834605F082FEC0F38B
:108DF00007258DF8095005F07CFEC0F307408DF87B
:108E00000A00069005F075FE010E8DF80B1006980D
:108E10002A0401EB0B6102EB00200A18218B06EB00
:108E20000110C0F801204FF08072C0F80A20A0F8AD
:108E30000EA000E003E0491C2183463C45E0B4F865
:108E40006210012021EA0B01A4F8621093490A780C
:108E5000DABB087014F8461F208B06EB0010017077
:108E60002978417169788171A978C171E9780172B5
:108E7000297941720021C0F80A1005F03AFE8DF8F8
:108E80000800834605F035FEC0F307258DF809502C
:108E900005F02FFEC0F307408DF80A00059005F09D
:108EA00028FE010E8DF80B1005982A0401EB0B61CA
:108EB00002EB00200A18208B06EB0011C1F80120FC
:108EC000A1F80EA0401C2083463C7F1C94F847006C
:108ED0004FF0010BB8423FF72AAEB4F85E5094F859
:108EE00047002844192804D86C484088B0F5967F7C
:108EF0000AD36A4800274780DFF8A4A19AF8000047
:108F000002280FD0A4F85E70664994F85E0001F85C
:108F100008000DB07BE506EB05101022002129F0BA
:108F200017FF6D1C192DF6DB5F4D55F82900C0F3B6
:108F30000721020E01EB0241C3B28EB24FF4C8709A
:108F4000434300224146304619F076FB012847D1C1
:108F50009AF80000022843D108F1B30001A906469F
:108F60001BF096FC9DF8040055F83830F02100F015
:108F7000F00201EA13418A4206D000F00F000143DB
:108F8000019130461BF093FC35F82900C0F307210E
:108F90006C2000EB480A50461BF089FC6D2000EB6A
:108FA000480B15F8291058461BF081FC55F829008C
:108FB0003E49884203D2401C45F8290010E0504643
:108FC00000211BF074FC584600211BF070FC9DF83A
:108FD000040000F00F0130461BF069FC45F82970D1
:108FE00040460C99FFF747FC8EE770B5304C0025E2
:108FF00094F86300B0B194F8620040B105F079FDD7
:10900000616E884203D3E8B22146FFF757FC94F81B
:10901000610094F86210401A002803DDE8B221468E
:10902000FFF75BFD6D1C68340C2DE1DB70BD2DE995
:10903000FE4F04464FF0010A22791B480126E178D1
:10904000012A12D006EB410350F823506D1C144F37
:109050003B78022B00D00125D4F8120000282DD037
:109060000027022B05D0677408E050F831506D1CC2
:10907000EDE7A84201D2677400E0667404F11A03B8
:109080004FF4C8790293A84223D2401EC3B24F4680
:109090007B43C0F30B2019F014F90BE02C020060A5
:1090A000A0040060A023026010D10160FFFF0F0048
:1090B0008CFE0260012802D04FF0000A6EE04946A3
:1090C000029829F05EFE4A46FE49029829F040FEC9
:1090D00064E0DFF8F483012AA8F5165B1ED0494648
:1090E000029829F04EFEF9480078022843D0E07833
:1090F000732106EB4000484308EB8000A0F85E7047
:10910000E0784A4606EB400000EBC00101EB00109E
:109110000BEB0011029829F01BFE3FE04946029834
:1091200029F02FFEE9480078022812D0E078732158
:10913000484308EBC000A0F85E70E0784A4600EBB8
:10914000C00101EB00100BEB4011029829F000FE6A
:1091500024E0E0787321414308EBC101B1F85E10CF
:109160000A0100EBC00101EB00100BEB401102986B
:1091700029F0EEFD12E0E078732106EB4000414358
:1091800008EB8101B1F85E100A0100EBC00101EBB0
:1091900000100BEB0011029829F0DAFDD4F8120050
:1091A000A0B9D4F8160088B9217904F11600031F7C
:1091B00001290ED0CDE90005E078D4F80D2006EBAA
:1091C0004000D4F80910C0B219F00FF95046BDE8BC
:1091D000FE8FCDE90005E078D4F80D204006D4F8E4
:1091E0000910000E19F001F9F0E730B500EB80022C
:1091F00002EBC002B648002100EBC20080F861100B
:1092000080F8621001EB81028318DA7A82B190F85B
:109210006120521C80F861205A7AAE4D1C7B2D785B
:10922000AC420AD04CB190F86220521C80F8622007
:10923000491CC9B20E29E5D330BD9B7A022B17D049
:10924000012B2AD0032BF3D1C2EBC20303EB421351
:10925000A14A1A4423324418D37884F84F30127844
:10926000012AE5D190F86220521C80F86220DFE7E5
:10927000C2EBC20303EB0213984A02EB430228320B
:109280004418537984F84F301278012AD0D190F8DD
:109290006220521C80F86220CAE7C2EB021202EB85
:1092A00042038F4A1A4423324418537984F84F30CA
:1092B0001278012ABCD190F86220521C80F86220FA
:1092C000B6E72DE9F0410025814FDFF818822846E6
:1092D000FFF78BFF05EB850000EBC50607EBC60427
:1092E00094F85D0028B994F85E0010B994F85F0016
:1092F00098B194F8610080B194F8620018B12146E9
:109300002846FFF77FFA94F8610094F862108842CB
:1093100003D021462846FFF7AEFA05F0EAFB606667
:10932000214608EBC600682229F012FD6D1CEDB243
:109330000B2DCCD30020F3F756FF6B4CE0600020E0
:10934000F3F751FF2061694900200870BDE8F08102
:1093500070B500205B4B664C783B664D03F10C0208
:1093600053F8206054F820108E4201D043F82010AA
:1093700052F8206055F820108E4201D042F820109B
:10938000401CC0B20328EBD3574B5B495C680968AB
:109390008C4200D0596052F8201058480068814231
:1093A00000D0986070BD2DE9FF5F044604EB840097
:1093B0004C4900EBC40001EBC008CDF808804449DB
:1093C00001EBC0060196002505F093FB7066204670
:1093D000FFF70BFF06F1090708F1090081465F223C
:1093E000394629F014FD00285CD006F15D0108F132
:1093F0005D00032229F00BFD18B396F8620000B15E
:10940000012598F8612098F8621096F86130521A98
:109410001B1A9A4202D045F0020543E000EB80009F
:1094200001EB810109300931304408EB01030146A9
:1094300002EB8202184629F0EAFC00B345F002056F
:1094400030E098F8620096F86210884208D100EB8C
:1094500080023946484629F0DAFC10B1012500E0C7
:10946000012598F8612098F8621096F8613096F816
:109470006200521A1B1A9A4202D045F0020511E00E
:1094800000EB800001EB810109300931304408EB29
:109490000103014602EB8202184629F0B8FC08B12C
:1094A00045F00205074FDFF824B004F1B300E907E7
:1094B000A7F16007039075D057F8340001060B0D33
:1094C0001EE0000070D1016080F80160A00400601F
:1094D0008CFE02605B020060F2E802600835056005
:1094E000C84005606C0303602C020060A9020060A4
:1094F0002459046030590460400400604404006052
:10950000C0F30B200122214619F096F8012849D119
:109510009BF80000022841D1694603981BF0B8F976
:109520009DF8000057F8341000F00F02C1F303411A
:109530008A4206D000F0F0000143009103981BF02E
:10954000B6F937F83400C0F30721542000EB440982
:1095500048461BF0ACF9552000EB440A17F83410CC
:1095600050461BF0A4F957F834004349884203D20F
:10957000401C47F8340011E0484600211BF097F9E1
:10958000504600211BF093F99DF8000000F0F00117
:1095900003981BF08CF9002047F834003146204630
:1095A000FFF730F9A8075FD5012000EB440557F815
:1095B0002500C0F30721020E01EB02411FFA81FCD6
:1095C0000006030D00222146604619F035F80128F7
:1095D0004AD19BF80000022842D1694603981BF04B
:1095E00057F99DF8000057F83430F02100F0F002F0
:1095F00001EA13418A4206D000F00F0001430091B6
:1096000003981BF054F937F82500C0F307216C20AC
:1096100000EB440948461BF04AF96D2000EB440A70
:1096200017F8251050461BF042F957F8250012494B
:10963000884203D2401C47F8250011E0484600212B
:109640001BF035F9504600211BF031F99DF8000060
:1096500000F00F0103981BF02AF9002047F82500BD
:1096600031462046FFF707F904B031464046BDE8D1
:10967000F05F682229F06CBBFFFF0F0010B50446B5
:10968000204629F0A5FB401E01B204E0625C202ABE
:1096900003D1491E09B20029F8DA2144002048709C
:1096A000204610BD30B5F849002283788C78A3425B
:1096B00013D144784D78AC420FD104780D78AC4288
:1096C0000BD1CC7814B9C5789D420BD09C4201D106
:1096D000C5783DB1C578AC4204D0521C12B21B31E2
:1096E000802AE3DB802A01DA104630BD4FF0FF30DC
:1096F00030BD182803D2002901DB802902DB4FF09E
:10970000FF307047E14A02EB002030F9110070474A
:1097100030B50021DD4C4A1E002004EB012323F864
:109720001020401C8028FADB491C1829F4DB00209B
:10973000D74B00EB800203EB82014D7B5DB1497892
:10974000491E182907D213F82220802A03D204EBDD
:10975000012121F81200401C1428EADB30BD70B54D
:109760000646CC4D0024687B28B1042229463046A9
:1097700029F04DFB20B1641C24B21C35802CF2DB97
:10978000802C01DA204670BD4FF0FF3070BD2DE90E
:10979000F0410746C04C2078002803D1FFF7B8FFFE
:1097A0000120207078784FF0FF36411E022912D830
:1097B000401E397880290BD2FFF79BFF142807D26F
:1097C000B34A00EB800102EB8101497B002900D103
:1097D0003046BDE8F081AE4D0024022229463846CD
:1097E00029F015FB20B1641C24B21435142CF4DBD1
:1097F000142C01DA2046ECE73046EAE770B5A24ABD
:109800000025867893789E4223D1C378D478A342EA
:109810001FD103781478A3421BD14378547803F006
:109820001F0304F01F04A3421AD0032B01D11B2CE9
:1098300016D01B2B01D1032C12D0032B01D1192CD4
:109840000ED0052B01D11A2C0AD0022B01D1182CD5
:1098500006D06D1CADB21B32802DD3D3002070BD5D
:109860000D70012070BDF8B505460F46894C0026E5
:10987000E978A078884215D1E07898B921786078A5
:109880006A4602F0CBFC69782A7901F0E001C90050
:1098900001EBC2212A78114489B2884202D13E707C
:1098A0000220F8BDA878A178884217D1E878E1783D
:1098B000884213D12878217888420FD1687800F047
:1098C0001F02607800F01F0082420ED0032A01D1EF
:1098D0001B280AD01B2A01D1032806D0761CB6B259
:1098E0001C34802EC4D30020F8BD3E700120F8BD8A
:1098F0002DE9F0418AB00C46DDE91061129D674FF9
:109900003F788DF80E708DF80F0004F01F004FF0B7
:109910000008032909D004F0E004022909D0002737
:1099200082B380328DF810203FE001278DF80D00C2
:1099300074E00127022819D01C2817D0D0B11D28A7
:1099400018D001281AD01E2818D004281BD01F2890
:1099500019D005281BD0162819D003281BD015288C
:1099600019D013281BD0172819D057E01C348DF8B4
:109970000D4053E01D348DF80D404FE01E348DF83E
:109980000D404BE00FE01F348DF80D4046E01634DB
:109990008DF80D4042E015348DF80D403EE017344F
:1099A0008DF80D403AE08DF81080012806D002288D
:1099B00008D004280AD003281CD02FE018348DF8D2
:1099C0000D402BE019348DF80D4027E004F11A000A
:1099D0008DF80D0015B305F1240000F01F0121449E
:1099E0008DF80D109DF8101000F0600001438DF807
:1099F000101013E001292DD0E01C8DF80D006DB181
:109A000005F1200000F01F0121448DF80D109DF894
:109A1000101000F0600001438DF810108DF80C302C
:109A20008DF815803A4602A903A8FFF71CFF00280D
:109A30000ED0184C9FB19DF80800C0EBC00004EB9D
:109A40008000C0F8056016489DF8081020F81180C5
:109A50000AB0BEE604F11B008DF80D00CFE71DB380
:109A60002A46314601A8FCF748FF0E49019829F023
:109A700070FB29F0F7FC9DF80810C1EBC10104EB65
:109A80008101C1F80500DEE71CB10360DC23026040
:109A90009CCC03609CBE0360400200605B020060DF
:109AA00040E3036000007A4402280BD04FF47A7040
:109AB00046439DF80800C0EBC00004EB8000C0F8EE
:109AC0000560C0E79DF80800C0EBC00004EB800013
:109AD000C0F80560817A6429B5D1012EB3D14FF465
:109AE0007A71C0F80510AEE72DE9F0418AB00D4655
:109AF000DDE91061129C00278DF810708DF80E00C2
:109B00008DF80F50501CC0B28DF80D005B1E8DF803
:109B10000C308DF8157002293AD002F01F0302F0C4
:109B2000E000012B38D0172B36D0022B38D0182B61
:109B300036D0042B38D0192B36D0012946D0C11C81
:109B40008DF80D1054B104F1200101F01F021044F2
:109B50008DF80D0001F060008DF8100000252A46F8
:109B600002A903A8FFF74AFE002810D0DFF8F4830B
:109B70008DB39DF8080000EBC00000EB40004044AE
:109B8000C0F80560F8489DF8081020F811705FE7EC
:109B900001258DF80D00E2E718308DF80D00DDE7A6
:109BA00019308DF80D00D9E700F11A018DF80D106C
:109BB000002CD3D004F1240202F01F0108448DF8D8
:109BC0000D0002F060008DF81000C7E700F11B01E6
:109BD0008DF80D10B6E7FFE7A4B12246314601A883
:109BE000FCF78BFEE149019829F0B3FA29F03AFC21
:109BF0009DF8081001EBC10101EB41014144C1F89E
